:020000040800F2
:1000000000500020A92C0108492D01089116010873
:10001000492D0108492D0108492D01080000000063
:10002000000000000000000000000000492D010851
:10003000492D010800000000492D01087D860008B7
:10004000492D0108492D0108492D0108492D0108B4
:10005000492D0108492D0108559E0008519E0008B0
:10006000492D0108492D0108492D0108492D010894
:10007000492D0108492D0108719E0008492D0108EC
:100080002DD50008492D0108492D0108492D0108E9
:10009000492D0108492D0108492D01084D9E0008F0
:1000A000492D01083D9C0008492D01084D9C000880
:1000B0002D9C00081D9C00080D9C0008E7520008BC
:1000C000EB520008E1520008E5520008492D0108F2
:1000D000492D0108659E0008599E0008492D010818
:1000E0008D860008492D0108492D010800000000F7
:1000F0000000000000000000000000000000000000
:0C01000000000000000000005FF808F1A3
:100110002DE9F04F684B694EA1B033600023736046
:1001200010F080F918B910F09FF907F029FA07F0DC
:10013000F1FA634A634C1378634D43F00103137083
:100140000023089309930A934FF4E0130B93236859
:10015000A87B43F480332360A36943F01003A361B9
:10016000236803F400330993089B01330893099B28
:100170001BB9089BB3F5A06FF2D12368514913F462
:10018000003301D0022315E00A6842F001020A6040
:100190000893236803F002030993089B0133089333
:1001A000099B1BB9089BB3F5A06FF2D123689A078E
:1001B00039D501230A93454B45491A6842F010028C
:1001C0001A601A6822F003021A601A6842F00202EA
:1001D0001A606368636063686360636843F48063A4
:1001E00063603C4B1A68043B22F070425A603A4A02
:1001F0001160616821F47C116160596841F000412F
:100200005960D96821F40041D9609B681B0449BF3B
:10021000324B4FF4E01313604FF480130B930A9B9F
:10022000012B01D117E0FEE7022B18D168B10B9B1F
:10023000B3F5801F02D14FF4A01305E00B9BB3F57B
:10024000E01F02D14FF400130B930B9963680B432B
:1002500043F4803302E0636843F46013636023680F
:1002600043F0807323602168164B8F01FBD55968DA
:1002700021F003015960596841F002015960636837
:10028000104903F00C03082BF9D14B68DFF85480B8
:1002900003F00C03042B03D0082B03D00C4B29E0F4
:1002A000136827E04B684868C3F38343C00303F136
:1002B000020319D40A4A1CE0936D0008C80000200C
:1002C0006C3000200010024054100020002002403A
:1002D00000127A000410014034000020001BB70017
:1002E00000093D005400002049681268890348BF96
:1002F00052085343C8F800306368DFF870A3C3F3B3
:10030000031353441A7BD8F80030DFF874B3D3409A
:10031000C8F80030C04B0DF18009CBF80C30A36950
:10032000002743F00103A361636ABC48B360636ABA
:1003300043F080736362A36943F01C03A3614FF62B
:10034000FF7329F82C3D49468DF856700DF0E4F9FD
:10035000B34849460DF0E0F94946B2480DF0DCF9E2
:10036000B14A4846536843F0007353600DF086FE6F
:10037000159BAE4A6420B3FBF2F3AD4A1360AD4B5C
:100380004FF47A721F60D8F80030DFF8F882B3FBC0
:10039000F2F3A94A013B5360F0238BF82330072383
:1003A00097601360AB68C8F8003008F034F939463C
:1003B000A248A02214F0BFFDE369394643F00703C9
:1003C000E361A36943F4006343F00C03A361544663
:1003D0009B4B4FF0000A03F10C0201F802A001311F
:1003E0000E29F5D1FF229A76DA761A775A77954B4D
:1003F000954A51461A6095483022D8F8008014F08A
:100400009AFD5146C8F380170423914ADFF83CE275
:10041000885C0C224A4302F80E0047B91E380128B6
:100420009FBFFF2003F1FF3302F80E00DBB2013162
:100430000429EAD1874A95F805B01370864B87499D
:1004400083F800B0864B7E4A3362C0330B60854B25
:1004500018F0200F03EBCB035B7818BF0123536226
:10046000002340F2DC51804A22F813100133082B9C
:10047000F7D10EA800211C2214F05DFD18F4007ABB
:100480001DBF7A4BCDF850900393CDF80CA0BBF173
:100490000E0F03D00BF0EF03082B02D101238DF8D0
:1004A0004A30012007F08CFE18B14088003018BF98
:1004B0000120C8F340038DF83E30C8F340338DF877
:1004C0003830C8F3C03300F001008DF83B3018F429
:1004D00000638DF83D008DF8407004D095F88631AA
:1004E0005F1E7B427B418DF83C30C8F300438DF8A2
:1004F0004130736A1AF1000A18BF4FF0010A003345
:1005000018BF01238DF84330C8F300538DF84430F1
:10051000B5F84A31B5F8480118F4805FADF84830B5
:10052000B5F85631ADF84E0018BF5148ADF8463019
:10053000C8F3804318BFB0F850018DF83F30B5F8CC
:10054000543118BFADF84E00B3F5FA7FADF84C301A
:1005500084BF0023ADF84E3095F8D631454886F873
:100560002830002386F8293043709DF84A3008F07F
:100570000101002BC8F3C0028DF839108DF83A2024
:100580008DF842A00CBF0023022301B902B1013350
:1005900004EB8304E3694FF00008A3F102091A3366
:1005A00005934FF6FF7339F8026F9E4200F09C816D
:1005B0009DF83D20F3B21AB19A1E012A40F29081B3
:1005C0009DF8402032B12C491A0189582B4A91429A
:1005D00000F086819DF8412032B127491A018958DF
:1005E000264A914200F07C819DF83E2052B1224A79
:1005F0000A4802EB03125168814203D11289102A82
:1006000000F06E819DF83B20002A44D01A4A03482E
:1006100002EB031238E000BF0005FA0500080140B4
:10062000000C0140001001400000014040420F005A
:10063000601900206419002010E000E0282C002040
:10064000C8000020342A002048120020382A002048
:100650001AA301082910002070080020442D002052
:1006600068100020649A0108940F002000750108AA
:1006700054100020F1000020C09401080004004044
:1006800000ED00E0742E00205168814203D11289F0
:10069000022A00F025819DF83C2052B1B74AB848A3
:1006A00002EB03125168814203D11289022A00F041
:1006B0001781149A7AB1B14C116804EB0314606885
:1006C000884208D121899088884200F00981D28827
:1006D0008A4200F00581360A022E02D19DF83820A8
:1006E00003E0012E04D19DF83920002A00F0F880A3
:1006F000DFF888A29DF844101F010AEB0704524658
:1007000031B19DF84A1019B9043B032B40F2D08057
:10071000012EF0B246D19B4D3A44FF23517B85F820
:10072000703085F87130506802F1080312894FF07B
:10073000000BADF854208DF85610022215A985F84B
:1007400074B0C5F8804004938DF8572085F82CB01C
:10075000C5F830B0C5F834B0C5F838B0C5F86CB0DD
:1007600085F872B085F873B00CF0D6FF049B5AF888
:10077000070099785A460CF083FE204659463246C7
:1007800009F0C0FA804BC5F88CB0C5F884307F4BB7
:100790002046C5F8883005F1840105F1880209F08A
:1007A000F9FA9DE002284BD15FFA88F34FF01C0C58
:1007B0000CFB03FC714ADFF8CCA1D1194B680692FF
:1007C00001F1080209890AEB0C0692F805E0002500
:1007D0004FF0010B86F87580ADF854108DF8570076
:1007E00015A9184686F8765086F87E5086F874B0BB
:1007F000C6F88040CDF81CC08DF856E004920CF08D
:100800008BFF049B069A9978D0592A460CF038FE43
:10081000204629465A4609F075FA5D4ADDF81CC0A3
:10082000C6F88420E2445B4A0AF18401C6F88820B5
:10083000C6F88C5020460A1D09F0ACFAD8444FE0A7
:10084000032833D19DF83F304E4D534E3BB195F8C0
:100850002A70204608214FF6FF7200231AE0BDF8E7
:100860004C2095F82A70B2F5FA7FBDF84E300BD9BE
:100870004A492046B1FBF2F2082192B20DF040F84D
:10088000474B46F827000AE046492046B1FBF2F202
:10089000012192B20DF034F8434B46F82700C360B3
:1008A00095F82A30013385F82A3019E0042817D149
:1008B000BDF846203B4B334D93FBF2F22046BDF88A
:1008C0004830012192B295F829600DF019F895F899
:1008D000293005EB86060133C6F8540185F8293026
:1008E000059B99457FF45DAE264C304F94F8292046
:1008F000002384F874212E4A3B701678A6F1170263
:10090000022A1AD81D46236A0021585903EB05080C
:1009100011F07AF918B1636A002B51D126E0254B0A
:1009200005EB030E98E80F008EE80F003B781035BA
:100930000133C02D3B70E6D1EDE71F4A12F836E0D7
:1009400002EBC602D2F804C087F800E0BCF1000F49
:10095000E1D01D467545DEDA164A2B0103EB02088D
:1009600063440FCB013588E80F00F3E7134B1A6897
:10097000984612F4805F49D142E000BFC09401085C
:10098000000C0140C800002071D2000851D30008BB
:10099000BDD4000849D20008F82B002000127A00CC
:1009A00071D3000840420F0061D30008F72B0020EC
:1009B00070080020AC070020649A0108742E002003
:1009C000B64BB74A13F8360003EBC6035D681070E8
:1009D000002DCBD000238342C8DAC3EBC3016A18D1
:1009E000D2F80080DFF8F0C2013341F80C8001EB4F
:1009F0000C0E9188AEF8041092798EF80620EAE782
:100A000006F0EF03082BA74B24D125E03B78012B00
:100A1000F6D9A54D05EB031303F110071035BD42C0
:100A2000EED055F8100C4FF07C5110F059FF4FF0FC
:100A30007C5145F8100C55F8140C10F051FF4FF094
:100A40007C5145F8140C55F80C0C10F049FF45F892
:100A50000C0CE3E70E2E08D11A78182E42F0100283
:100A60001A7008D10EF0CEFB05E01A78192E22F08C
:100A700010021A70F5E70EF0A9FBD8F8003001203B
:100A80005E035EBF894B01221A70894A894D137833
:100A90004FF0100A43F00403137004F093F8D8F8F1
:100AA0000060284606F4006300215246049314F0C7
:100AB00042FA022306F4004900271E408DF8363022
:100AC0008DF837700CD07C480DA9ADF834A00DF02E
:100AD00049FC04232B70012607236F70AE70EB7066
:100AE000202375480DA9ADF834304FF0010B0DF0FF
:100AF00039FC4FF007080523DFF8B8A12B72771CEB
:100B00006E7285F80AB085F80B80B9F1000F0FD02E
:100B1000022269480DA9ADF834200DF023FC8AF8B3
:100B200005708AF804B08AF806B08AF80780B71C06
:100B3000049B7BB1022361480DA9ADF834300DF060
:100B400011FC092301222B73AA737B1C07226F73EC
:100B5000EA73DFB25A4A5B485368002643F44043C5
:100B600053605369DFF85C8143F00103536193697B
:100B700043F4007393610DF009FA534B012F159361
:100B8000524B15A916930CBF334680231A934FF48A
:100B900080731B934FF480631C9320231D93404666
:100BA0004FF400531E931796189719961F960DF041
:100BB000CFF9D8F80030464943F00103C8F80030B7
:100BC0004A68012F22F4702294BF0023012322F4EB
:100BD000807242EA03224A608B683E4A1A4042F41D
:100BE000602242F002028A60CB6A23F470027B1E0C
:100BF000DBB242EA0353CB620123AA1991780029A0
:100C00007CD0A85D591C0928C9B2D278DFF8C0E0B1
:100C100011D9A0F10A07DEF80C8007EB47074FF067
:100C2000070C0CFA07FC28EA0C0CBA404CEA02024A
:100C3000CEF80C200EE0DEF8107000EB40084FF00C
:100C4000070C0CFA08FC27EA0C0702FA08F23A43F0
:100C5000CEF81020062B1E4F0ED8013B7A6B03EB0B
:100C600083034FF01F0E0EFA03FE22EA0E0200FA73
:100C700003F313437B6340E00C2B2FD8DA1FD7F824
:100C800030C002EB82021F2393402CEA030E00FACD
:100C900002F34EEA03033B632FE000BF84820108A6
:100CA000D02C002048180020B4070020D80C0020C9
:100CB0006C300020942A002000080140000C014004
:100CC00000100240080002404C240140A42A0020E9
:100CD00000240140FDF7F1FFD12C0020A3F10D020B
:100CE000D7F82CC002EB82021F2393402CEA030E9C
:100CF00000FA02F34EEA0303FB620B460436102EA1
:100D00007FF47BAF7E4B9A6842F480729A609A6857
:100D100042F001029A609A6842F008029A6099686B
:100D2000774A0D07FBD4936843F004039360744B38
:100D30009A6812F00408FAD19A6842F4A0029A6004
:100D4000704BB3F85C019A46002840F0B287BAF9BC
:100D50005E31002B40F0AD87BAF96031002B40F0D6
:100D6000A887694B00211B680C22B3F856306748EE
:100D7000BAF864519AF863B19AF86B719AF86C6199
:100D80000493BAF80C909AF80FA014F0D4F8604BC2
:100D9000002118461422059314F0CDF85D49002275
:100DA0000A70C4F8782104F0A1FA059B002800F02D
:100DB0006587594AB5F5807F1A60584A5A60584A83
:100DC000DA60584A1A61584B01D1002216E0BB2D57
:100DD00001D9012212E0612D01D902220EE0292D54
:100DE00001D903220AE0132D01D9042206E0092DBE
:100DF00001D9052202E0002DE7D006221A70012356
:100E00004A4A13704A4A136843F0010313605A4672
:100E1000092A4FF0000101D90A46F9E74FF0010B0A
:100E20000BFA02F313F04D0005D113F46C7357D095
:100E3000404B18704AE03F4BC4F87811197004F029
:100E400055FA002842D006210A4615AB682004F066
:100E500009F89DF8591001F001029DF8571001F0B2
:100E600001014B0043EA82019DF8552002F0010385
:100E70000B430AD05BB2012B01D1002302E0022B0D
:100E80000ED1012384F87C3111E00DAB68200C21D8
:100E90005A4603F0E7FF9DF8343013F00F0303D1F7
:100EA000032007F0C2FB02E0042BEAD1E5E7174B71
:100EB000214A1A60214A5A6094F87C21002A0CBF0A
:100EC0006F226E221A72032300F0E1BE0F4B1C4A00
:100ED0001A601C4A5A6000221A72092300F0D7BE19
:100EE000012A9B4693D8134A1370042E00F2018105
:100EF000DFE816F02A0008012A002A00C90000BF16
:100F00000024014054100020A40F0020402E002097
:100F1000982300203406002075520008BB4F0008BB
:100F2000954F000890C1793D00000020500000203E
:100F30004418002090300020994B0008FD4F000815
:100F4000DDDB0008F9DB000894F87D31BB4E002B97
:100F500040F0CF86142007F05EFB7720D0210122DD
:100F60000DAB03F07FFF002800F08D809DF834303A
:100F70000322552B86F89731A6F8A02140F08380F4
:100F8000D12101220DAB772003F06CFF9DF83430A6
:100F9000772003F00F021B0986F8982186F8993113
:100FA000162215ABAA2103F05DFF9DF854209DF891
:100FB000553043EA0223A6F880319DF856209DF86B
:100FC000573043EA0223A6F882319DF858209DF855
:100FD000593043EA0223A6F884319DF85A209DF83F
:100FE0005B3043EA0223A6F886319DF85C209DF829
:100FF0005D3043EA0223A6F888319DF85E209DF813
:101000005F3043EA0223A6F88A319DF860209DF8FC
:10101000613043EA0223A6F88C319DF862209DF8E6
:10102000633043EA0223A6F88E319DF864209DF8D0
:10103000653043EA0223A6F890319DF866209DF8BA
:10104000673043EA0223A6F892319DF868209DF8A4
:10105000693043EA022341F27072A6F89431784B6A
:101060001A8046F678125A80764A5A60764A9A6012
:10107000764ADA60764A1A61764A5A61012386F81E
:101080007D3100F036BE94F8A4B16C4EBBF1000F78
:1010900040F00686142007F0BEFA06F2A51376206B
:1010A000D021012203F0DEFE96F8A531582B29D17C
:1010B00006F5D47388211822762003F0D3FE31225E
:1010C0007620F42103F0BBFF0123634A86F8A431A4
:1010D0005B4B9A60614AA3F800B05A6045F6D8129B
:1010E0005A805F4ADA605F4A1A615F4A5A6100F0CB
:1010F000D7BD012E06D05D4B5D4A9E70136843F04C
:10110000040313605A4E3368980702D5594B1B6885
:101110009847EDB2584ABAF1000F29D033684DB95B
:1011200040F2596113F0020F40F2712318BF0B46D1
:101130007D2108E0990759BF4FF47A7319464FF49F
:10114000FA634FF47A71994505DBB9F57A6FA8BF58
:101150004FF47A6900E099464B1E4B44B3FBF1F320
:10116000013BDBB203FB011184F8C431116003E0E1
:1011700084F8C4A1C2F80090404D2B689847404ABB
:1011800000231370914617B1022F40F08C854FF069
:10119000000A20AB03F82CAD1E200A210122C4F85E
:1011A000C8A103F05FFE002800F0A6859DF854302A
:1011B000482B0CD1334B344A1A60344A5A602B4BBB
:1011C0000222DA70336843F00803336002E05046CD
:1011D00000F092BD2E4C94F858310BB12D4A13708B
:1011E00094F859310BB12C4A137094F85A310BB161
:1011F00089F800303368DFF8ACB013F0080F53D033
:10120000BDF910A04FF064099AFBF9F7384610F0C9
:1012100013FB049009FB17A000B210F00DFB1F494F
:1012200010F05EFB049B0146184610F051FA1C4971
:1012300010F056FBCBF8000039E000BFC8000020DA
:10124000D41B00206D5200086D4F00085552000855
:101250002D4F00086D4A0008694A00086B4A0008D3
:101260004D520008E14E00080548000850000020DB
:1012700044180020402E0020241D00209823002028
:1012800093300020B01B0020C550000895D3000803
:101290005410002034060020903000208988883CBB
:1012A00000002041502D00200023CBF80030A54F36
:1012B0004FF00A093B78049743F002033B70192072
:1012C00007F0A9F909F1FF39192007F0A4F919F07D
:1012D000FF09F4D133681B0705D59B4B1B68984762
:1012E0009A4B01221A709A4B9A4F1B68187B10F088
:1012F000A3FA994910F0F4FA06F01EF882463888ED
:1013000010F09AFA514610F0EBFA14F021F8934BD2
:101310001880388810F090FA0146914810F094FB3C
:10132000904910F091FB904B8B491860286910F0A0
:10133000D7FA8E4910F0D4FA8D4D8E4BFF211860EC
:101340001B22284613F0F7FD28460021297031683A
:10135000894B012211F0020F18BF6A701A701FBF6B
:1013600003221A700222AA704F0741BF1A78551C37
:101370001D70032548BF855411F00A0F0CD01A7850
:1013800004218154511CC9B205254554D11C023297
:101390001970D2B206218154784D29688E0641BF5A
:1013A0001A78561C1E70072648BF86540A0608D5B0
:1013B0001A7809268654961C01321E70D2B20A266B
:1013C00086546679082E01D00E2E08D11A7802F1C3
:1013D000010E83F800E04FF00B0E00F802E01A78DF
:1013E000CF0302F1010E4FF00C0C48BF624F00F822
:1013F00002C05FFA8EFE48BF023283F800E041BFB0
:101400003A705B4A4FF00E0C02F80EC04A0748BF14
:101410001A784FF0120C41BF02F1010E83F800E080
:101420004FF0100E00F802E01A784F0502F1010E9D
:101430005FFA8EFE83F800E000F802C00AD594F847
:1014400018723FB14C4F02323A70494A4FF0130CB8
:1014500002F80EC01A788F0502F1010E4FF0140C3D
:1014600048BF454F00F802C05FFA8EFE48BF023207
:1014700083F800E041BF3A703D4A4FF0150C02F886
:101480000EC0182E13D11A784FF0160E00F802E095
:1014900002F1010E5FFA8EFE4FF0170C00F80EC03D
:1014A00002F1030E0232D2B283F800E086540F0339
:1014B00041BF1A78561C1E70192648BF8654CE05A7
:1014C00041BF1A78511C19701A2348BF8354002158
:1014D00098222B4813F02FFD0CF025FC294A2A4BAB
:1014E000B4F852111A60294BB4F8980119802849B0
:1014F00000230B808B7027490A6081B2264A22F8AC
:1015000013100133122BF9D12B68D9045CBFB4F846
:101510009E1111801B0740F1EA8094F89241062C3D
:1015200000F2DF80DFE804F004073C6782A2A2003B
:1015300045F2F05201E042F6F822184B1A800CF006
:101540008CFCCDE06C300020B01B0020C81B0020BC
:10155000C00600201600002035FA8E3CDC06002074
:101560000AE81C4100401C46FC1C0020BD378635A3
:101570006D0F0020BC0600206C0F0020742E002090
:1015800090290020DE1100200C0E0020100E0020FB
:1015900044300020383000206C2F00201C07002031
:1015A00042F6F8227A4B1A8010F046F9794910F089
:1015B00097F9794910F08AF810F07EFB0023774AFA
:1015C00042F823000133122BF9D1754A75494020A6
:1015D0001160754A137006F0CDFE002800F081807E
:1015E00001234FF0070990F9000040218DE808021F
:1015F0006E4A6F4B6FE042F6F822654B40201A802E
:101600006C4A674B1A60684B10221A7006F0B2FEE3
:10161000002866D001234FF0000C90F90000402113
:101620008DE80810644A4FF4E13354E042F6F822A2
:10163000574B40201A80614A594B1A605A4B082276
:101640001A7006F097FE00284BD001234FF0000ED1
:1016500090F9000040218DE80840594A4FF4E133E9
:1016600007F01FF8574BC3F8CC0136E042F6F822DA
:10167000474B0C261A804C4B53485449544A1E7011
:10168000062C4FF00003DFF87CC1524F03700B7043
:10169000137009D01B238CF800304F4B05223E708D
:1016A0001A704FF4E13406E021238CF800304A4BE5
:1016B0003E701C70494C4A4A394B40201A6006F073
:1016C00059FE70B10123002790F900008DE88800D1
:1016D0002346444A402106F0E4FF003018BF0120B1
:1016E00028B9082005F01AFF3F4A2D4B1A602A68D6
:1016F0002D4912F4804F1FBF08230B703B48284B25
:1017000018BF186042F2010313409BB144F62060F9
:101710001F4B9604188041BF08230B703448204BA0
:1017200048BF1860D40741BF0C230B7031481C4BD5
:1017300048BF18600B781006A3F104034B7040F10A
:101740009B8020482C4E0024DFF8BC90C0F8D0616C
:1017500021461522294F00F5EA7089F80140C9F8A1
:101760000440C9F80840053E13F0E5FB20463E6002
:1017700008F0E0F8224B02201B68BA46C9F80C308A
:1017800006F0F8FD002841D1802005F0C7FE6BE08F
:101790001C070020CDCCCC3F0000B044242F0020FB
:1017A00030000020251301082C2A0020CD14010848
:1017B000A08601001113010821140108FD1201087F
:1017C000D5130108C800002034300020692900200A
:1017D00068290020333000208C29002090D003009D
:1017E000E5DB000815DC0008851301085513010826
:1017F0007513010865130108481200202C0600200B
:10180000982E00208B2900200C060020447999F89E
:101810000130BC490C2202FB03125278A24204D0D0
:101820000133DBB2042BF4D9002389F80130DAF854
:10183000003099F801201B7890F90000002B4FF040
:101840000C0303FB021314BF0324012400225B7862
:1018500000940192022106F024FFAB4B186000288F
:1018600092D0012008F066F8A84B1868A84B00F544
:10187000C5721A6008F006F92B6899056CD5A54A5F
:10188000A54C039BA548236093690DA943F0010370
:101890009361039B1B88ADF8343010238DF83630EC
:1018A00002238DF837300BF037FF23689B485B88A5
:1018B0000DA9ADF8343004238DF836300BF02CFF31
:1018C00020680F21037A03F0030203F0FC0303F105
:1018D000804303F580339C689200914024EA010123
:1018E00099609968012404FA02F20A439A604368F5
:1018F0008B4AD943536116680E40166056680E40F5
:10190000566016681E43166096680E409660D6684C
:101910003140D160916819439160D1680B43D36025
:10192000437A15A88DF8543003238DF855300023E1
:101930008DF856308DF857400FF0E6F8794B7A4A1B
:101940001B683C3B1360794A136843F01003136033
:10195000774B4FF0FF321A60764B774A774C136023
:10196000774A803313602B680026DA03267040F133
:10197000AA8040F22A3ADFF8F4B1664F0DF084FDF8
:101980004FF0010952465846314684F8009013F052
:10199000D2FABB696B4843F00403BB614023ADF846
:1019A000303018238DF833300CA903238DF83230F2
:1019B0000CF0D8FCFB69644943F00203FB61634B04
:1019C000634C1B68A7F69477B3FBF1F32188013BC6
:1019D00021F45C710904090C21809BB21D21A185B1
:1019E0002385A4F81490238C23F001031B041B0C03
:1019F0002384238CA088218B23F0020321F0730120
:101A000009041B04090C1B0C41F0600180B243EA7D
:101A10000903A0802183A6862384238B23F0080357
:101A20001B041B0C43F008032383B4F844306FEA13
:101A300043436FEA53439BB2A4F84430D7F8A83F1E
:101A400043EA0903C7F8A83F38460CF09FFA414B18
:101A5000CDF858B0159380231A934FF480734FF04C
:101A6000100B1B9338464FF4005315A91E9319967B
:101A70001C961D961F96CDF85CB0CDF860A00CF0BA
:101A800067FAA3890DA89BB243F40073A3813B6856
:101A900043F002033B608DF834B08DF835908DF83B
:101AA00036608DF837900FF02FF82B4B1A682B4BC0
:101AB00043F8282008F10108B8F1200FF5D10BF008
:101AC0004DFD0BF04BFD2B685B0540F19180DFF87D
:101AD000A090234BD9F814A50420C3F800A006F069
:101AE00049FC0421C9F8180506F020FC1D4B89F8B3
:101AF0001C050820C3F800A006F03CFC1A4B082186
:101B000038E000BF9C750108EC1E0020A40F0020E7
:101B1000680E0020001002401C1D0020000C014037
:101B200000040140982E0020181D002044180020B9
:101B3000C40F00207C120020281F0020D90C002098
:101B4000241F00200008014000366E0154000020D0
:101B500000040040340400402C750108DA0C002019
:101B60003818002090180020DC180020B102002056
:101B7000C8000020186006F0D9FB634C89F81D05E9
:101B8000002120462C2213F0D6F98E2363704FF0EB
:101B90007C08E0237D26E37084F8008084F82B60C5
:101BA0005A4C2C220021204613F0C5F98A23637079
:101BB0001020A023E37084F8008084F82B60C9F81B
:101BC00020A506F0D7FB1021C9F8240506F0AEFBCE
:101BD00089F828052020C9F82CA506F0CBFB202188
:101BE000C9F8300506F0A2FB89F834050FF072FA47
:101BF0002B68474A13F4002318BF0123137006F023
:101C0000E3FC444B1860444B5A791946052A02BF3D
:101C1000424B4FF4C8721A80414B4FF47A721A80CB
:101C2000404BC8221A80404A137843F008031370CF
:101C30003E4A137823F00203137040F602032A6829
:101C400013406BB13A4A3B4B1A603B4B03221A706C
:101C50003A4B01221A703A4A00231380394A138002
:101C60008B6801222B60384B1A70049B049A1B78F6
:101C700063F07F03137021B0BDE8F08F334A1A6020
:101C8000334A5A60334A9A600823FFF7B9B8324A98
:101C90005370324A136843F002031360FFF725B90B
:101CA0000426FFF728BA012F7FF694AA1F46FFF7F4
:101CB00066BA2B4B00221A7000B20FF0BDFD294905
:101CC0000FF00EFE1590BAF95E010FF0B5FD254933
:101CD0000FF006FE1690BAF960010FF0ADFD214934
:101CE0000FF0FEFD2049179015A805F02FFBFFF718
:101CF00038B80226FFF7FFB9012F7FF66BAA00273D
:101D000089F80000FFF743BA6018002095180020FA
:101D1000211D0020FC060020541000201E0E002073
:101D20008A3000208830002048180020923000209F
:101D3000D01100203018002094180020440000200A
:101D4000080F00200A0F0020D80C0020E3DB000859
:101D500007DC0008DFDB00085000002044180020EA
:101D60003800002035FA8E3C702A0020954A2DE973
:101D7000F04F1568944C05F59C43944E2033236036
:101D8000336889B013F4804F059205D10FF066FCDB
:101D900010B92379013323718D4A13784BB18D49E2
:101DA00009688D4240F2E58003F1FF3882F8008037
:101DB000DFE09846884B5FFA88F51F78DFF83892A5
:101DC000AF4231D9D9F80030072D98BF595D834B08
:101DD00088BF29461B6880489847032D1ED8D9F82C
:101DE000002005F10E0302EB83039988DA88A8B17D
:101DF0004FF47A73401A5843531A90FBF3F040F6AD
:101E0000C90300F57A70984205DC40F2EE2398424F
:101E1000B8BF184601E040F6CA0080B204EB4505A1
:101E2000E88008F10108C5E794F804800325B8FBB1
:101E3000F5F50F2384F82A3094F82B3005EB45058F
:101E4000019394F82C30C5EB08050393D9F80030C2
:101E5000DFF8ACA10293EBB204930025BD4255DA42
:101E60005F4B4FEA450933F815B0019B53B90FF0AA
:101E7000F5FB28B1039B002B08BF4FF0000B01E0DE
:101E8000DDF804B0029B988A584502D8D88A584594
:101E90000ED2E8B20FF08EFB032D8346DFBF94F81D
:101EA0002AE00120A8402EEA0000D8BF84F82A00CA
:101EB0000FF0D4FB18B14B4829F800B022E0049B86
:101EC00094F876002AF813B030B9B8F1020F15D99A
:101ED0003D4B012083F87600BAF80000BAF80230D2
:101EE0000344BAF8040003443F489BB229F8003089
:101EF0001BB2032093FBF0F39BB200E05B46394832
:101F000029F8003001350AF1060AA7E794F82A20DB
:101F10003648A2F10F014A424A4184F89020344BDE
:101F20006AB1344A1268520109D40268D9689A60C9
:101F3000521AC82A1DD9012283F8212019E002680B
:101F40009868DA605B68121A9A4288BF284B4FF093
:101F5000000184F82B1088BF83F821100025BD42B2
:101F600007DAE8B20FF026FB1E4B23F81500013507
:101F7000F5E73368DD0405D51E4B1B68D80701D48F
:101F800008F0FEFC059B1F681B4B1A68907A00281E
:101F900038D01449137B013831F810001BB1C0F55B
:101FA0003B60083080B200B2A0F57A70B0F57A7F5D
:101FB000A8BF4FF47A7020EAE0700FF03DFC0F49A3
:101FC00055E000BF70300020600D0020742E00200E
:101FD000403000203C3000202C2A0020300000201F
:101FE000660D00206C2F0020D80D0020982E0020B8
:101FF00044300020680F00203830002000007A4470
:102000008E0D0020336819043AD5D4F89430934DDE
:10201000FB1A002B34DB07F59C432033C5F89430C2
:102020008F4BD27A59798F4B33F8113095F898103D
:102030009BB293FBF2F3013101F00F0285F8982077
:102040002A4482F899300346874A825C013013445F
:1020500010289BB2F8D11BB293FBF0F000B26428B9
:10206000A8BF642020EAE0700FF0E6FB7F490FF084
:10207000EBFC7F490FF034FC0FF01EFE7D4B188007
:1020800033687D4D13F4807F00F00F817B4BDFF8C8
:10209000F0919F4205D999F8022012B9012289F8DE
:1020A000022099F80220002A00F0FF80744A95F877
:1020B000008092F82170C8F380087A1E5742574179
:1020C000704A002F9246116818BF4FF0000BC1F301
:1020D0008063019308BF4FF0030B99F82020052A75
:1020E00000F2DD80DFE802F0034E537988A5B8F1F5
:1020F000000F3AD0D4F8AC00B4F8B01006F0D7F91D
:10210000012809D16049614A09681268C9886420B8
:1021100000FB0122C9F81020019B6BB15A4A1268DA
:1021200012794AB10BF070F8032289F820204FF49D
:102130007A72C9F81C20D0E7002F40F0B080534AD3
:10214000D9F8101010684E4A88420AD902920BF052
:102150005BF8029A032182F8201040F6B831D16171
:10216000BBE7012182F82010B7E7019B4FF48060A4
:1021700013B105F0C3F901E005F0AFF90022C9F889
:1021800010208CE0002F49D10BF03EF8A5E727B1D5
:10219000052289F82020012000E03846B8F1000F20
:1021A0000CD0D4F8AC204FF0020BD189384A118002
:1021B00051809180344909684988D180334A116837
:1021C000D9F81420914202D8B8F1000F64D147F237
:1021D0003052C9F81C20032221E02A7842F0020282
:1021E0002A7008F0CDFB294AD9F81C1012680A445D
:1021F000C9F81820042212E0244A9FB11168D9F8C6
:10220000182091424BD9234A12781AB9DAF80020E3
:10221000D30744D42A7822F002022A70052289F8D2
:1022200020205AE71268D9F81C100A44C9F818206F
:1022300035E01549154A09681268C988642000FB11
:1022400001224FF48060C9F81020002289F8202074
:1022500089F8032005F041F93FE700BF600D002039
:10226000942A0020A42A0020F90D00200000C84272
:1022700000C07F44C80F002092300020404B4C002B
:1022800044300020680F0020D0230020982E00202A
:102290006C2F00201400002000287FF41EAFBBF13B
:1022A000000F02D0584606F055F9934F07F5C57058
:1022B000B7F8521106F0FBF80197834668B90AF0A7
:1022C00095FF8E4B0022C3F800B0C3F804B0C3F8EA
:1022D00008B08B4B1A605A609A602B785F0736D52E
:1022E0003368D80633D5874B1B78D9062FD4864B55
:1022F0001B789BB1019B93F8E231BBF1000F15D124
:102300007BB1824B1A68D4F8B4309B1A002B08DAE0
:1023100008F036FB7E4B83F8B8B018E0BBF1000F35
:102320000DD1102006F016F901230EE03BB1774ADB
:102330004FF47A71126801FB0323C4F8B43094F8A7
:10234000B83023B106F0F6F8002384F8B830019BCA
:1023500093F8E0A193F8E111B3F89AE1B3F89CC1C6
:10236000002318466B4F800837F91320013372455C
:10237000C4BF60F07F00C0B26245B8BF40F040000B
:10238000042BB946EED194F8B930614A834205D1A5
:1023900092F8BA30F92B04D8013300E0002382F818
:1023A000BA30594B84F8B9001A785B4F9846E2B9B5
:1023B0003B68DA0708D5BBF1000F16D12B78DB0795
:1023C00013D508F033F910E02B7858070DD5504B92
:1023D00093F82B304BB1514BDB7833B911B108F086
:1023E000CFFA02E0BBF1000FF9D094F8BA30484AB6
:1023F000142BDFF83CB140F0AD8098F800301AF1B2
:10240000000A18BF4FF0010A6BB392F8B9305F2B86
:1024100011D12B7803F0040303F0FF0113B108F08E
:10242000AFFA08E00B200391029206F093F8029AAB
:10243000039982F8BA10BAF1000F14D094F8B930A9
:102440007D2B10D12B7803F0040303F0FF0213B1AE
:1024500008F096FA07E00B20029206F07BF82C4B6E
:10246000029A83F8BA202B7803F0040303F0FF01EB
:10247000002B6FD194F8B930254A572B15D1284B32
:102480004FF47A721A803368190601D507F04AFBB7
:10249000244B1B685A0742BF234A0A21118013F0BC
:1024A000080357D1214A138054E03068400717D5FC
:1024B0005A2B15D192F8BB302BB1012382F8BB10F7
:1024C00082F8BC3046E092F8BD3083F0010382F818
:1024D000BD300BB10C2000E00D2006F03BF839E0D8
:1024E0005D2B00F012855B2B00F011855E2B21D156
:1024F000032000F00DBD00BF54100020582B002019
:10250000D42B00204818002014000020982E002012
:10251000600D00206C2F0020680F00204430002048
:102520008A30002044180020883000204410002009
:10253000A40F0020562B03D1029305F0BFFA029B93
:1025400098F80020002A00F0F9846F2B40F0F08406
:1025500008F06CF833685B0736D594F8BD30B64A9E
:1025600093B12B7858070FD5019BB9F90610B3F832
:102570009A31994208DD3B6813F0010302BF322112
:10258000A2F8C01082F8BD303B68D9030DD594F88D
:10259000C220A94B2AB993F8BB2012B93222A3F862
:1025A000C020012384F8C2300EE094F8BB30A24A68
:1025B00053B12B7803F0040303F0FF0123B9012387
:1025C00082F8BB1082F8BC30DBF8009000233B603F
:1025D00009F17B0809F1CB0A98F8002098F801303E
:1025E00018F8010C9A420BD2414605F02BFF38B186
:1025F00018F8022C012303FA02F23B6813433B60F4
:1026000008F10408D045E7D18C4B1B784BB18C4BBB
:10261000DFF844921A68984612F0020F40F03183B6
:1026200029E309F1CA0709F589783A787B7817F820
:10263000010C9A4225D2394605F004FF08B397F8F9
:1026400004E00C21BB7801FB0E417E4A013B03EB09
:1026500043031344D1F8C82097F803909A42764870
:102660000FD0C1F8C830002390F8F420C1F8CC3066
:10267000012303FA0EF322EA030381F8C49080F8E1
:10268000F43006374745D0D16F4BDFF8D0A1D3F8EF
:1026900000806E4B4FF0000B1B68029394F82B30B8
:1026A0000393DAF80030002B00F0DC8293F80090FE
:1026B000B9F1000F00F0D682DAF8042002998A1AE4
:1026C000002A0CDB01F5FA72CAF8042094F8F41021
:1026D000012202FA0BF221EA020284F8F420039AA2
:1026E000002A00F0BF821AF8042C59780432D2B2C2
:1026F000002940F07882564931F91210554AB2F853
:10270000982102F1C800814201DD9F7814E0C83AA7
:10271000914202DA99784F420EE094F8F4200123B6
:1027200003FA0BF322EA030384F8F430029B03F567
:10273000FA73CAF8043095E294F8F43043FA0BF3D4
:10274000DA0700F18F82002FCCBF0220012005F0B4
:1027500023FF09F1FF32384B132A00F27B82DFE8B6
:1027600012F0140023003200440061007F00E400F6
:102770004901AE01E30112027902440055007F00D5
:10278000E4004901B6001B01800198F800104046A2
:102790000F44FA2FA8BFFA2727EAE77788F80070D6
:1027A00005F036FE01201EE098F8011040460F4467
:1027B000642FA8BF642727EAE77788F8017005F03F
:1027C00027FE02200FE098F8031040460F44642FC4
:1027D000A8BF642727EAE77788F80370D3F8F810D2
:1027E00005F0CEFD03203946CAE198F805100D200A
:1027F00039446429A8BF642121EAE17188F80510F1
:1028000005F084FEB9F10D0F00F0248298F8041051
:102810000E2039446429A8BF642121EAE17188F8B7
:102820000410ADE198F806100520394481F3080141
:1028300088F80610A4E100BF600D0020943000204D
:10284000680F002094790108CC0F0020982E0020FA
:102850006C2F00205410002044180020280E002067
:10286000D3F8FC301A78022A22D1384604930EF0AD
:10287000E3FFA9490FF0E8F8049B596A05930EF0AD
:1028800027FF002104900FF0C9F9059B48B9049A6D
:10289000A24910460FF0E0F9049A059B10B19F4A37
:1028A00000E000225A620F20114605F01BFE0AE0EC
:1028B00099780F203944C829A8BFC82121EAE171BD
:1028C000997005F023FEB9F10F0F00F0C381944B0E
:1028D000D3F8FC9099F80030022B1AD138460EF04C
:1028E000ABFF8D490FF0B0F8D9F820100EF0F0FED4
:1028F000002107460FF092F930B9384687490FF0AA
:10290000ABF910B1854F00E00027C9F82070122004
:1029100059E199F8011012203944C829A8BFC821EB
:1029200021EAE17189F801102AE1D3F8FC301A7824
:10293000022A22D1384604930EF07EFF77490FF029
:1029400083F8049B196B05930EF0C2FE00210490DE
:102950000FF064F9059B48B9049A704910460FF0CE
:102960007BF9049A059B10B16C4A00E000221A63BF
:102970001020114605F0B6FD0AE0197B10203944FD
:10298000C829A8BFC82121EAE171197305F0BEFD6D
:10299000B9F1100F00F05E81614BD3F8FC9099F80B
:1029A0000030022B1AD138460EF046FF5B490FF07B
:1029B0004BF8D9F82C100EF08BFE002107460FF0D3
:1029C0002DF930B9384655490FF046F910B1534F3B
:1029D00000E00027C9F82C701320F4E099F80B10E0
:1029E00013203944C829A8BFC82121EAE17189F818
:1029F0000B10C5E0D3F8FC301A78022A22D13846F1
:102A000004930EF019FF47490FF01EF8049BD96B91
:102A100005930EF05DFE002104900FF0FFF8059B7A
:102A200048B9049A3D4910460FF016F9049A059BDF
:102A300010B13A4A00E00022DA631120114605F095
:102A400051FD0AE0997D11203944C829A8BFC82149
:102A500021EAE171997505F059FDB9F1110F00F006
:102A6000F9802F4BD3F8FC9099F80030022B1AD143
:102A700038460EF0E1FE2B490EF0E6FFD9F838108B
:102A80000EF026FE002107460FF0C8F830B9384690
:102A900022490FF0E1F810B1204F00E00027C9F8FB
:102AA000387014208FE099F8151014203944C82983
:102AB000A8BFC82121EAE17189F8151060E0D3F8B8
:102AC000FC9099F80030022B1AD138460EF0B4FE73
:102AD00011490EF0B9FFD9F828100EF0F9FD0021C8
:102AE00007460FF09BF830B938460C490FF0B4F8A0
:102AF00010B10A4F00E00027C9F82870092062E0F1
:102B000099F8031009203944C829A8BFC82121EA2F
:102B1000E17189F8031033E0000020410000C84251
:102B2000600D002000007A44D3F8FC9099F8003042
:102B3000022B1AD138460EF07FFEBB490EF084FFFF
:102B4000D9F834100EF0C4FD002107460FF066F8E6
:102B500030B93846B4490FF07FF810B1B24F00E0F9
:102B60000027C9F834700A202DE099F80D100A20CA
:102B70003944C829A8BFC82121EAE17189F80D109C
:102B800005F0C4FC66E0D3F8FC9099F80030022B05
:102B90001DD138460EF050FEA4490EF055FFD9F86D
:102BA00040100EF095FD002107460FF037F830B9C0
:102BB00038469D490FF050F810B19B4F00E00027B8
:102BC000C9F840700B20394605F08CFC42E099F8BA
:102BD00017100B203944C829A8BFC82121EAE17188
:102BE00089F81710CCE7012934D19878904B33F944
:102BF0001230B3F5617F05DB40F633029342A8BF84
:102C0000134601E04FF46173B9F10C0F22D14FF478
:102C1000966292FBF0F0A3F5617393FBF0F3854AA3
:102C2000DFB21378BB4215D0042F34BF3B460223DA
:102C30001370019A09FB03237F4A03F2B2731360F6
:102C400004F044FD4846394605F060FC781CC0B2EB
:102C500005F0A2FC94F8F420012303FA0BF31343CC
:102C600084F8F4300BF1010BBBF1040F0AF10C0AEC
:102C70007FF417ADCBE43368DB0511D56F4BDB7800
:102C800073B1D9F800309F070AD56D4B1B8813F03C
:102C900001070AD10AF0AAFA012004F02FFC04E08F
:102CA000012004F01AFC012300E00023D8F80020E2
:102CB00050070DD563B1012004F00FFC604B1B8859
:102CC000990708D40AF092FA022004F017FC02E0F7
:102CD000022004F002FCD9F8003013F00A0F29D0CA
:102CE000D8F80030DA060BD5554B1B885B070AD4A1
:102CF000042004F003FC534B1B88A4F8003102E0CD
:102D0000042004F0EAFBD8F800309F0607D54C4BAE
:102D10001B88580606D4402004F0F0FB02E0402057
:102D200004F0DBFBD8F80030590642BF454B1B8846
:102D3000A4F80231D9F800309A0609D4D8F8003046
:102D40001B0540F1B2804FF4807004F0D7FBB0E077
:102D50003D4BDFF8EC901B7813F0020F53D03B4B48
:102D60001B78042B4FD9D8F8003013F4007A0FD019
:102D7000B9F80030DF063AD4102004F0BFFB202061
:102D800004F0ABFB3248011D06F036FE02232AE0B8
:102D9000B9F8007007F01007BFB22FB1102004F08F
:102DA0009CFB012784F804A1D8F80030580512D5FF
:102DB000D4F8083127495A89B1F90030002BB8BF3F
:102DC0005B42934207DAB1F90230002BB8BF5B4295
:102DD0009342C0F2F380B9F80030990608D520205C
:102DE00004F07BFB002384F80431012700E0002776
:102DF00094F80C3193BB0E2005F0ACFB164B01226E
:102E000083F80C212AE0B9F8003003F03003002BDE
:102E100094D0102004F061FB202004F05EFB00231E
:102E200084F804311DE000BF0000C84200007A446D
:102E30006C2F0020202E0020CC0F002044300020DA
:102E40000C19002044100020481800204E180020C3
:102E5000D40F00204C100020600D0020002F3FF404
:102E60006DAF00221446624B002023F81400614B22
:102E7000191D03F10A0721F814000021D15117444C
:102E80007860B96023F8140003F132075A33D15146
:102E9000D150174413447860B96058609960143277
:102EA000002C7FF44BAF0124DDE74FF4807004F079
:102EB00014FB514B5A791C46082A01D00E2A02D124
:102EC000402004F00AFB33685A0540F18D8094F8E5
:102ED00018321BB92B7813F0040F03E0D8F8003038
:102EE00013F4002F0AD0454B00221A703C200AF040
:102EF000FDFF002878D00CF09BFFF7E70EF0EAF812
:102F000009B0BDE8F04F0AF00EBF012000E002203A
:102F10005FFA80F8019A08F1FF3382F8B03704F0C5
:102F20002FFB04F0F7FB404605F036FBFFF712BB22
:102F3000BAF1000F02D07E2B3FF40AAB972B05D1DC
:102F40004FF4C873A4F8BE30FFF704BBA72B06D11B
:102F50002B4A137843F004031370FFF7FBBA0022E7
:102F6000BB2B079201D1022303E0B72B04D14FF60C
:102F7000FE73ADF81E300AE0BE2B01D1022304E03F
:102F8000BD2B7FF4E7AA4FF6FE73ADF81C30DBF8DB
:102F90000030BDF81C10B3F858200A44A3F858209C
:102FA000BDF81E10B3F85A200A44A3F85A2004F0C2
:102FB00085FD002384F8BA30FFF7CCBAB9F80030A9
:102FC0009B063FF515AF202004F098FA0D4B0E48F4
:102FD0001A685B68011D4360026006F00DFD0B4B33
:102FE000012783F8047103E709B0BDE8F08F00BF43
:102FF0008C3000206E0E002054100020312A00205A
:103000004818002050180020DC0F0020600D002020
:10301000B54B2DE9F04FB3F90610B44B85B01F68DE
:1030200001937A8991420EDBB1F5FA6FFC79BFBF4B
:103030008B1A6343A2F5FA6493FBF4F4ACBFC4F1BA
:103040006404643400E06424A94BAA4AB3F898B13C
:1030500093F9623112689BB20292154603930022E3
:1030600040F2E630A04B4FEA420C33F912E0CBEBD2
:103070000E0303F2F316864203D8002BB8BF5B425F
:1030800001E04FF4FA73022A2ED0029E96F81161E5
:103090001EB1B342CCBF9B1B0023642093FBF0F80E
:1030A000954E6FF0630A36F818900AFB083A08F15B
:1030B000010836F918600FFA89F8C8EB060606FB16
:1030C0000AF696FBF0F68D484E4420F80C60BE18C8
:1030D0003679642073438A4E93FBF6F364339BB2D4
:1030E000634393FBF0F02CE0029890F812611EB15C
:1030F000B342CCBF9B1B0023642093FBF0F0DFF8AE
:103100002C926FF0630808FB003A39F91060013027
:1031100039F91000002BA0EB060000FB0AFA9AFB1D
:10312000F8FA0398C6EB0A0A0AFB00FA7348B8BF1C
:103130005B42A0F804A0B8794343714893FBF0F0D8
:1031400064306B784FF06408434393FBF8F36D4EA3
:10315000022AB354EB7A6C4E00FB03F393FBF8F3B3
:10316000B3546B7D654E00FB03F090FBF8F0674BAA
:103170009854674B0ED1DE4583F802800DDB5C4C22
:10318000B4F89A21914214DBB1F5FA6FA8BF4FF45D
:10319000FA610FE0DE459C5404DA36F80C305B42ED
:1031A00026F80C300132032A05F101057FF458AFEF
:1031B000E5E71146891A4FF47A735943C2F5FA626A
:1031C000B1FBF2F1642391FBF3F2DFF874E16FF0ED
:1031D00063073EF8120007FB021101323EF912208C
:1031E00007B2D21B514391FBF3F30344F380494BE5
:1031F000424D1B885F063BD5474A484B10881B88C9
:10320000181A00B20EF018FB45490EF069FB07468C
:1032100004F092F88046384604F01BF80746B5F9EA
:1032200002000EF009FB8146B5F900000EF004FB28
:10323000414682460EF054FB3946834648460EF01E
:103240004FFB014658460EF041FA0EF00FFD414685
:10325000288048460EF044FB3946804650460EF022
:103260003FFB014640460EF033FA0EF0FFFC68804B
:103270002C4D2B68980740F19E8045F207212A4B80
:103280002A4F1A687B69D31A8B4240F394807A6183
:103290000BF0B0F9264BDFF8AC901A789846032A69
:1032A000B9F8003050D10A2B58D90023282088F8CB
:1032B000003005F0B0F90BF09DF91E4B18880BF0AB
:1032C00083F91D4B1A68D37890FBF3F0013008287E
:1032D0001A4BA8BF08201870537980B243433B8330
:1032E00013795843788339E06C2F0020CC0F0020ED
:1032F00054100020A40F0020421900204C10002080
:103300000CFEFFFFE02B0020FE0E0020F42B00201F
:10331000382B00200C190020620E002044100020E1
:1033200035FA8E3C742E002070300020F00E002004
:1033300094180020AC2A00203018002044000020FF
:103340002A190020341800200A2B07D803238E4A9C
:1033500088F80030002313703B837B8398F800309B
:103360008A4A012B0CD002D3022B1BD023E03A8BCC
:10337000B9F800309A421EDD012388F800300FE0D2
:10338000B9F800107B8B8B4202DD022313700FE033
:103390007F4B1B8B0133994202DD002313700AE03F
:1033A000082006E07B8BB9F8002001339A42E3DC69
:1033B000072005F0CFF82D68290577D5754B744F98
:1033C0001A68FB69C3EB020845F2072398456DDDD7
:1033D000714BB6F906B0D3F800904FF47A7099F8B3
:1033E0000A30FA61012B98FBF0F8B4F85211ABF5F2
:1033F0007A7B6A4E03D042D3022B20D041E0684B47
:10340000396A5A7B674B4FF0080E33F8122091FB54
:10341000FEF392B2C91A8B183B6293FBFEF3BA8497
:1034200040F6E4429BB25343B9F80820C2EB133391
:103430005843B9F9063090FBF3F0306021E05A4B65
:10344000B9F808A01B78C6F800A05A0719D5574844
:1034500005F02DF820B915F0100F18BF4FF0000B34
:103460000BFB0BF3322293FBF2F3B9F906205B441A
:103470005A434FF47A7392FBF3F3534400E0002372
:1034800033603368D7E90A0103FB08F84FF47A7315
:1034900098FBF3F810EB080041EBE8710023C7E953
:1034A0000A01434A0EF028FC424B1860424E336832
:1034B000DB0427D52F0622D5404B1B789D071ED550
:1034C0003F4B187804281AD900223E4B0521D71803
:1034D000951C4FF00A0E122AD154E9B287F801E088
:1034E00004D0B0EB510F2A46EFD800E014215A184F
:1034F000322002F8010CFF225A540F2000E00A206B
:1035000005F028F8304D2A68002A73D02F4B304F31
:1035100018683968984681426CD82E4BDFF8C09005
:1035200018785168B0B901221A70B9F80030CB5C34
:10353000D3B1294B1A700EF09DF8B9F800309BB941
:103540002B681B78053B012B0ED805F03DF8234B6B
:10355000186009E000221A70B9F80030CB5C1BB18A
:103560001D4B1A700EF086F82B68B9F800205B68C6
:103570001B499B5CFE2B02D100230B803AE0FF2B02
:1035800030D104F0D7FF35E044000020941800202B
:10359000F00E002070300020301800203C18002071
:1035A000942A0020A42A002092300020DE1100205E
:1035B000407E050040180020680F002048180020B9
:1035C0004E1800204C2E00205C190020982E002060
:1035D000541900205119002050190020DC1E002031
:1035E00058190020D8F800000A2505FB0303013212
:1035F0003B600A809D4D2B7858073DD43268D10737
:103600005CBF43F001032B70994B1B781F075EBF13
:103610002B7823F001032B70D60248BF2B78954AF4
:1036200044BF23F001032B70934B1B6813F0040F6E
:1036300002D09249098851B99149098809B198077E
:1036400005D4904B1B88003318BF012333B10223EC
:1036500013702B7823F001032B7004E02978C9073D
:1036600058BF0223137004F0AFFF874B1B68C01ACA
:10367000002801DB0DF0FEFF0DF02CFD834B1E78C2
:103680009846002E00F0AB80814E3368002B00F08E
:10369000EE8630680BF0F5FB002800F0E8867C4BE6
:1036A0007C4C18680BF0EAFB092801D03F2850D168
:1036B0004FF0000A5746D4F80090774DB9F1000F4B
:1036C00005D0764829684A4611F082FC10B9AA460E
:1036D00007B92F46724B10359D42EFD3C7B1D7F8CB
:1036E00000E0DAF800C023681EF803501CF803005D
:1036F000A8420DD15A1C694938B92D2B05D8654D02
:103700002A602025CD54885402E0CD542260EAE797
:1037100023680BB1574511D062480CF079FC57452E
:1037200007D857F8100B0CF073FC09200CF068FC5C
:10373000F5E75D480CF06CFC4FF0000923689945F3
:10374000A7D2564B13F809000CF05AFC09F10109F5
:10375000F4E72368002B40F06F86042840F0A88629
:103760004E4807F069FA00F082BED9F80000DFF891
:1037700048A10BF086FB40B3DAF800000BF07EFBAB
:10378000DBF80030024693F84810002935D1242890
:1037900040F09480012283F84820DBF80030DFF805
:1037A00014A193F84820062ADFD193F8490001F0CC
:1037B000B3FD8146002800F0AC803B6898790CF09E
:1037C00074FB3B68002283F84820384B93F835306F
:1037D000002B40F01F864C36982E00F04886344B64
:1037E000F21892F84A100129F5D1324FF3583A6095
:1037F000314ABB4613609146B7E7012904D14D28F1
:1038000014BF00220222C6E7022904D13C2814BFBB
:1038100000220322BFE703290CD140284FF000010A
:1038200002D983F84810B8E758711971D9719871A5
:103830000422B0E7042906D1997983F849004A4067
:103840009A710522A7E70529A7D1587919798842E5
:10385000987906D950409871481C18710B441A7217
:103860009BE790420CBF0622002294E79230002092
:1038700048180020501900204418002088300020EB
:103880001E0E00208A300020683000209430002076
:103890003C2E0020201F00207C800108F01E00200C
:1038A0002C820108C7980108CC980108F00E00206E
:1038B00090290020EC180020F01800202B78D8491F
:1038C00058073FF56AAF232ADAF8003014D10120F7
:1038D00088F80000D34803910360D3480292036341
:1038E000D2480CF095FBD2480CF092FB0399029A57
:1038F0000B7843F002030B70CE4B1B681B7893428E
:1039000001BFCD4ACD4B1A60CD4A04BFCD4BDA6022
:1039100043E7DAF8002092F849304C2B00F0698434
:103920005DD8332B00F0A08421D8292B00F02D8402
:1039300009D8252B00F00484272B00F00884232BC2
:1039400040F0B2852FE22D2B00F0308407D82B2BCE
:1039500040F0AA850CF08CFA607100F03EBD2F2B70
:1039600000F0EE84312B00F0008500F09DBD3E2B71
:1039700000F0F2801DD8372B00F0AA8404D8352B34
:1039800000F04A8200F090BD392B00F0ED833C2B13
:1039900040F08A85DFF8B092D9F800A00CF068FA00
:1039A0008AF80000D9F8003018780BF0D9FC00F044
:1039B00014BD432B00F0698406D8412B40F0748578
:1039C0004FF0000900F055BC442B00F002854A2B53
:1039D00040F06A850CF056FAA08100F0FEBCD02BB6
:1039E00000F0108355D8CA2B00F0C08009D8C82B2E
:1039F00000F0858000F23E834E2B00F0078400F03B
:103A000053BDCD2B00F0098304D8CC2B00F02C82C1
:103A100000F04ABDCE2B00F00983CF2B40F0448547
:103A20000CF030FA6FF4AF6283189BB2C62B98BFCC
:103A3000A4F898010CF026FAA4F844010CF022FA3C
:103A4000A4F846010CF01EFAA4F848010CF01AFA8A
:103A5000A4F8DA010CF00CFA84F8EF010CF008FA83
:103A60000CF006FA84F8F0010CF002FA84F88701F1
:103A70000CF0FEF984F894010CF0FAF9724BD3F8CB
:103A800000900CF0FFF900EB80004000A9F8560010
:103A90006AE3D62B00F03B820AD8D22B19D0C0F0B3
:103AA0001083D32B25D0D42B00F03C8200F0FCBC3B
:103AB000EF2B41D005D8D82B40F0F6844FF0000909
:103AC00004E1F22B00F07682FA2B00F0B88200F0CD
:103AD000EBBC2B78590700F180840CF0C9F902285F
:103AE00084F8B00740F29482584B002283F8B02744
:103AF0008EE20CF0C7F9564B188000F06EBC92F8BD
:103B000005904FEA5909B9F1120F03D90AF0EAF901
:103B100000F063BC4FF0000ACA4507D20CF0B2F9BE
:103B20004C4B23F81A000AF1010AF5E73E4B01223B
:103B300083F8342000F051BCDFF80C91D9F800A0D4
:103B40000CF0A0F9AAF85A00D9F800900CF09AF9F4
:103B5000A9F8580000F041BC0CF08AF984F8E201A1
:103B60000CF086F984F8E10100F037BC364B1A6896
:103B70009A461278022A40F08E80DAF8003009F175
:103B8000080B02930CF074F90DF052FE32490DF05F
:103B90005BFF029B43F82B00DAF800B00CF068F9E9
:103BA00009F10A030BEB830B0DF042FE2B490DF0DC
:103BB0004BFFDAF80030CBF8040002930CF058F910
:103BC0000DF036FE26490DF03FFF09F10E0B029B6A
:103BD00009F10109B9F1030F43F82B00CDD1B9F177
:103BE000070FDAF800B03DD10CF042F90DF020FEDD
:103BF00019490DF029FFCBF84400DAF800B00CF0B9
:103C000037F90DF015FE14490DF01EFFCBF84800F2
:103C1000DAF800B00CF02CF98BF84C0035E000BF5E
:103C2000923000203C2E0020F00E0020FC9801086D
:103C3000CC980108342A0020EFBEADDEF04F002002
:103C40000400FA0500ED00E0A40F0020541000204D
:103C5000600E00206C2F0020000020410000C842B0
:103C600000007A440CF004F9CB448BF80100DAF838
:103C700000B00CF0FDF8CB448BF80B00DAF800B084
:103C80000CF0F6F8CB448BF8150009F10109B9F1F5
:103C90000A0FA4D1A1E3DAF800B00CF0E9F8CB44A4
:103CA0008BF80100DAF800B00CF0E2F8CB448BF8A6
:103CB0000B00DAF800B00CF0DBF8CB4409F1010995
:103CC000B9F10A0F8BF81500E5D186E3DFF890A370
:103CD00009F1080BDAF8003002930CF0D3F80DF07C
:103CE000A7FDD9490DF0B0FE029B43F82B00DAF88E
:103CF00000B00CF0C7F809F10A030BEB830B0DF0D1
:103D000097FDD1490DF0A0FEDAF80030CBF80400A1
:103D100002930CF0B7F80DF08BFDCB490DF094FE3B
:103D200009F10E0B029B09F10109B9F1030F43F8E8
:103D30002B00CBD1B9F1070FDAF800B01AD10CF093
:103D4000A1F80DF075FDC0490DF07EFECBF84400E2
:103D5000DAF800B00CF096F80DF06AFDBA490DF0F3
:103D600073FECBF84800DAF800B00CF08BF88BF853
:103D70004C0012E00CF086F8CB448BF80100DAF826
:103D800000B00CF07FF8CB448BF80B00DAF800B0F1
:103D90000CF078F8CB448BF8150009F10109B9F162
:103DA0000A0FC7D119E30CF063F8132883463FF6D6
:103DB000ADAEDFF8ACA2DAF800900CF059F80023B1
:103DC000A2490C2202FB0312117A814220D11378FE
:103DD00009EB8B0989F879300CF04AF889F87A00F8
:103DE0000CF046F889F87B000CF042F8984A994BA1
:103DF00089F87C001A60DAF80000974B00211860FF
:103E0000793004F043FB954B80F001001870E4E238
:103E100001331C2BD4D179E60CF02AF80B2882460A
:103E20003FF674AE8E4BD3F800900CF021F80328C7
:103E30003FF66CAE062303FB0A9989F8CE000CF01E
:103E400017F889F8C9000CF013F889F8CA000CF0CB
:103E50000FF889F8CB000CF00BF889F8CC000CF0C7
:103E600007F889F8CD00B8E25379092B7FF64EAEFA
:103E7000019BD3F800900BF0FBFF019B89F8000039
:103E8000D3F800900BF0F4FF89F801000BF0F0FF7D
:103E9000019B64281B68A8BF642018710BF0E8FF21
:103EA000019B64281B68A8BF642058710BF0E0FFD9
:103EB000019BFF281B68A8BFFF2098710BF0D8FF5B
:103EC000019B6428D3F8009028BF642089F807007C
:103ED0000BF0CEFF019B89F80200D3F800900BF0A5
:103EE000C7FF019B89F80300D3F800900BF0CAFFCD
:103EF0003B68A9F80A005B790A2B40F26E82594BA5
:103F0000D3F800900BF0B4FF89F8080065E20BF0DD
:103F1000B9FF554B23F8190009F10109B9F1080F50
:103F2000F5D15AE253790F2B7FF4F0AD0BF0A0FFDF
:103F3000072881463FF6EAADDFF824A1DAF800B0A1
:103F40000BF0A0FF0E2303FB09F9CB44ABF81901DA
:103F5000DAF800B00BF096FFCB44ABF81B01DAF8AF
:103F600000B00BF08FFFCB44ABF81D01DAF800B0C6
:103F70000BF07EFFCB448BF81F01DAF800B00BF09A
:103F800077FFCB448BF82001DAF800B00BF070FF1C
:103F9000CB448BF82101DAF800B00BF069FFCB4479
:103FA0008BF82201DAF800A00BF076FFD144C9F8B3
:103FB000230112E20BF05CFF0F2881463FF6A6AD0D
:103FC0000BF056FFC9EBC909A14489F8D4000BF0E6
:103FD0004FFF89F8D5000BF04BFF89F8D6000BF0A6
:103FE00047FF89F8D7000BF043FF89F8D8000BF0A2
:103FF0003FFF89F8D9000BF03BFF89F8DA000BF09E
:1040000001F9EAE12B785B0700F1E7810CF02CFA6B
:1040100003F0B6FA03F07EFBDFE12B78580700F1DE
:10402000DC81124B4FF4C8721A80D6E12B78590705
:1040300000F1D3810E4A137843F004033FE02B785C
:104040005A07E5D530E200BF00007A44287A01081B
:1040500098110020580E00205C0E00201400002053
:10406000A40F0020CC0F0020222E00201E0E0020C6
:10407000481800200BF0FCFEDA4B1A7810B142F021
:10408000020201E022F002021A700BF0F1FED64BA0
:10409000DFF8789318700BF0FFFEC9F800000BF002
:1040A000FBFEC9F804000BF0EDFED04B18800BF0BE
:1040B000E9FECF4BCF4A1880137843F00203137008
:1040C0008BE10BF0D5FE02900BF0E6FE83460BF081
:1040D000E3FE82460BF0E0FE81460BF0D3FE0BF0D0
:1040E000D1FE0BF0C5FE029BA3B9C34B1020C3F851
:1040F00000B0C3F804A003F0F0F9BA4A137843F013
:1041000001031370B9F1000F00F06781BB4BC3F8D6
:10411000009062E1102B40F06081B94BC3F800B011
:10412000C3F804A0B9F1000F02D0B44BC3F800905B
:10413000B348B44B0222011D1A7005F05DFC4CE13E
:10414000A0600BF0A9FEA3681843A06045E10BF046
:1041500099FEA4F85C010BF095FEA4F85E010BF04B
:1041600091FEA4F8600138E10BF082FE84F87C0136
:104170000BF07EFE84F880010BF07AFE84F87F015C
:104180000BF076FE84F8810127E10BF07BFEA4F8AA
:1041900082010BF077FEA4F884010BF069FE84F82D
:1041A00086010BF06FFEA4F8880116E10BF060FEAB
:1041B00084F892010BF066FEA4F89C010BF062FEFD
:1041C000A4F898010BF05EFEA4F89A010BF050FEE3
:1041D000DAF8003084F893015B79082B40F2FD8017
:1041E0000BF050FEA4F89E010BF04CFEA4F8A001C9
:1041F000F3E00BF03DFE84F8D8010BF039FE84F8B3
:10420000D9010BF03FFEA4F8DA01E6E092F8059040
:104210000323B9FBF3F9B9F1120F3FF677ACDFF8DE
:10422000F0A14FF0000BCB4580F0D7800BF020FEC3
:104230008AF8A2010BF026FE40F2ED23984205DD3C
:1042400040F6CA039842A8BF184601E040F2EE20AB
:10425000A0F2EE20192390FBF3F00BF1010B8AF88A
:10426000A3010AF1020ADEE70BF002FE84F89401D2
:10427000B3E00BF0FDFD04EB090309F10109B9F10D
:10428000080F83F88A01F4D1A7E00BF0F1FDC4F820
:10429000089060710BF000FEA3681843A0600BF05B
:1042A000E7FD84F892010BF0EDFDA4F85C010BF042
:1042B000E9FDA4F85E010BF0E5FDA4F860010BF048
:1042C000E1FDA4F882010BF0DDFDA4F8840184E097
:1042D00053794FF0070AB3FBFAF2C2EBC2029A1A03
:1042E00012F0FF0F7FF412ACB3FBFAFA0AF1FF3AB7
:1042F0005FFA8AFABAF1FF0F6FD00BF0B9FD5FFADF
:1043000080FB4FFA8BF003F05BFF814600283FF4FF
:10431000FDAB80F800B00BF0B5FDA9F802000BF082
:10432000A7FD89F804000BF0A3FD89F805000BF048
:104330009FFD89F807000BF09BFD89F80600D5E783
:10434000DFF8CC9009F1400A0BF09CFDA9F8A80217
:104350000BF08EFD89F8AA020BF08AFD09F1040921
:1043600089F8A702D145EFD137E00BF081FD1F2876
:1043700081463FF6CBAB3B685B79082B7FF4C6AB3D
:104380000BF080FD09F18A0904EB890A00F03F0077
:10439000AAF802000BF076FDBAF80230800100F4B2
:1043A000FE501843AAF802000BF062FD000104F869
:1043B00029000BF05DFD14F8293000F00F001843C0
:1043C00004F829000BF054FD8AF801000BF05CF8AA
:1043D00003E00D4B012283F8352000200BF094FD03
:1043E000FFF7EBB9481800204E1800204C180020A9
:1043F0004A180020D20F0020D40F0020E40F002024
:10440000DC0F0020640E0020F00E00205018002069
:1044100054100020584B985904F08CF918B93220E8
:1044200004F0F9F8F6E70AF0ADFE03F07FF8534A1E
:10443000534BDA60FFF7CFB90C283BD00A2842D1A2
:10444000504D51480BF0E4FD2846232110F0A9FD02
:1044500008B1401B20602368002B57D14948002138
:104460003022236010F067FD98F800302BBB474BDB
:104470001B689B060FD5464B46491B688A6B9A1AE8
:10448000002A08DB444A1278042A82BF03F512335B
:1044900003F5F8738B63414B9B68002B69D0404850
:1044A00005B0BDE8F04F184709F01CFDFFF785B9CE
:1044B0000C2804D13B480BF0ABFD3B480DE07F28B6
:1044C00012D1FFF7E6B80D28BAD07F2809D12D4ABE
:1044D000013B002135482360D1540BF099FDFFF7D3
:1044E000D8B82F2B3FF6D5A8A0F12002D2B25E2A71
:1044F0003FF6CFA813B920283FF4CBA85A1C22605E
:10450000204AD0540BF07CFDFFF7C3B85A1EA95CBB
:10451000202901D113469FE71A4A00212360D15474
:10452000234B244DD3F800A0D5F800B0DFF8549009
:10453000584610F044FD074659463A46484610F0A2
:1045400047FD1D4A28B919F8073053445B785B07CB
:1045500003D010359542E7D306E0954204D2781C8B
:10456000EB684844984702E014480BF051FD0023E3
:1045700074E705B0BDE8F08F902900200400FA052B
:1045800000ED00E0F01E002073A401084418002094
:1045900070300020F00E00204E18002098230020DC
:1045A0002C0F0020D1980108CC980108F898010838
:1045B000580000207C8001082C820108DC9801084A
:1045C0008F4A70B51368988A80B2C1B2CE072ED5D3
:1045D000198821F400610904090C1980198889B22D
:1045E00041F48061198000211171517999B191795B
:1045F00011B9D179FF290ED101219171117A0229C6
:1046000001BF198889B241F400611980517A41F0E3
:1046100001011982DFE0517A01F0FE011982D3799C
:10462000FF2B00F0D880764BFF211971D3E08D0766
:104630003AD5BFF35F8F107AC0B2012813D15179F8
:1046400089B1917979B1198821F480610904090C43
:104650001980BFF35F8F198B1988907289B241F46A
:10466000007119801BE0198BBFF35F8F107A6449CA
:1046700002280AD1487940B1897931B1198821F4E9
:1046800080610904090C19809FE0107A5C490328B5
:1046900005D1487918B18979002940F09680998828
:1046A00089B241F4806195E04C0754D501219172A3
:1046B0005179002936D09179002933D0117A1888A0
:1046C000022911791CD920F480600004000C1880A4
:1046D0001C8AD568C8B2E4B249B26C54198889B250
:1046E00041F400711980811C1171198A0130C9B21D
:1046F00040B22954998889B241F48061998026E0BA
:1047000080B240F4007018801C8AD568C8B2E4B248
:1047100049B26C541C8A411C49B2E4B203306C5457
:10472000107114E09179364809B9017C41B11988BA
:1047300089B241F40071198011790131117106E0DB
:10474000198889B241F48071198001218171198819
:10475000C905FCD43FE001F0400101F0FF04E1B1E4
:1047600010791E8AD568C4B2611C40B2F6B22E54CC
:10477000C9B2157A117149B2C81C854201BF988827
:1047800020F480600004000C08BF9880137A8B42EC
:1047900021D11B4B02341C711DE006061BD511797B
:1047A00048B2451C0AD054690131205CC9B2188254
:1047B000107A117149B288420DD106E0D179147195
:1047C0001982517909B9117A29B9998821F480613E
:1047D0000904090C9980117A92F904000131884288
:1047E000074B0CD100219971997A31B119688B88E6
:1047F00023F440731B041B0C8B800023137670BDC5
:10480000300F00202DE9F04FDFF8589285B00746B1
:10481000D9F81C000E460DF00FF88E4C804620880B
:104820000DF006F84FF05C51054640460DF058F883
:104830004FF06451824628460DF052F8014650462A
:104840000CF044FF4FF06251824640460DF048F8AC
:104850004FF06A51804628460DF042F80146404626
:104860000CF034FF0546B4F902000CF0E5FF0146F8
:1048700028460DF035F85146054650460DF030F803
:104880008046B4F904000CF0D7FF014640460DF015
:1048900027F8014628460CF01BFF80460DF0E6F98C
:1048A0006D490546A06140460DF0CEF8D9F820309C
:1048B0008046284601930CF0BFFF4FF07C510DF06D
:1048C0000FF866490CF002FF0546E389B4F90A00C7
:1048D00002930CF0B1FF29460DF002F829460CF0C6
:1048E000FFFF4FF058510CF0FBFF8146B4F9080070
:1048F000B4F810B0B4F80CA00CF09EFF29460CF0F0
:10490000EFFF014648460CF0E3FE4FF058510CF023
:10491000E7FF4FF060510CF0E3FF4FF07E510CF0D9
:10492000D7FE8146E0880CF083FF014648460CF034
:10493000D7FF002181460DF067F900287BD1294679
:1049400028460CF0CDFF03900FFA8BF00CF074FFAB
:10495000039B014618460CF0C3FF4FF060510CF06A
:10496000BFFF8346BDF908000CF066FF01462846EC
:104970000CF0B6FF01460CF0ABFE014658460CF0B9
:10498000A7FE4FF07A510CF0ABFF834601980CF074
:1049900053FF01464FF093400CF098FE05460FFA86
:1049A0008AF00CF049FF4FF08F410CF099FF01465F
:1049B00058460CF08DFE4FF066510CF091FF014609
:1049C00028460CF083FE26490CF08AFF49460DF07C
:1049D0003BF80546B4F916000CF02EFF29460CF002
:1049E0007FFF29460CF07CFF4FF040510CF078FF20
:1049F0008146B4F914000CF01FFF014628460CF064
:104A00006FFF4FF060510CF06BFF014648460CF011
:104A10005FFE8146B4F912000CF00EFF01464846D5
:104A20000CF056FE4FF076510CF05AFF0146284626
:104A30000CF04EFE00E0002017B10DF017F93860C1
:104A40002EB140460DF012F964235843306005B092
:104A5000BDE8F08F700200200000A04500007A47FA
:104A60000050C345300F0020704770472DE9F041DA
:104A7000324C334D6289AB8CB4F904809A1A238985
:104A8000B4F902E05A43B4F91230D613B4F9142041
:104A9000DB02324493FBF2F232440A26E2615643CF
:104AA000A2F57A6202FB02F3B4F90EC002FB0EFE1D
:104AB00002FB08F2B4F90C801B130CFB03FC03FB94
:104AC00008F31B1403EB62320232E388921002F502
:104AD000004253434CF25032B4F920704FEAEE2EAC
:104AE000B4F900400EEBEC2C0CEB8404BC40AD6A36
:104AF0000234A5EBA4043A4162434FEAD3384EBFD7
:104B0000B2FBF8F35400B4FBF8F340F6DE3448BFD0
:104B10005B001A12524362430A4C08365C43241469
:104B200004EB224202F6CF62361103EB221300B1EE
:104B3000036001B10E60BDE8F08100BF48020020B3
:104B4000300F002043E3FFFF104B13B593F82C20E8
:104B50001C46CAB90E4B1B68B3B11A681AB10D498D
:104B6000886902438A619A889868ADF80420022215
:104B70008DF8072004220DEB02018DF8062008F0C5
:104B8000CBFD012384F82C3002B010BD300F002083
:104B9000400200200010024008B5FFF7D5FF074B88
:104BA0001B7813B1012B03D008BD4FF4006201E064
:104BB0004FF48052024B1A8008BD00BF440200200F
:104BC00016000020012828BF01202DE9F04F0646DD
:104BD000142000FB06F3704F89B0F918FC586F4B96
:104BE0000A691C6083F82D606D4BB1F80880DD699F
:104BF000B1F80AA02A43DA61A2884D6822F4407213
:104C00001204120C4AEA0809A28003A9C5F8109000
:104C100002228DF80E0028460193ADF80C908DF815
:104C20000F2008F079FD019B00971F464FF0080BFD
:104C3000AA6818EA020F03D10A2003F0E1FCF7E7A3
:104C40000A20C5F8148003F0DBFCC5F810800A20A8
:104C500003F0D6FCBBF1010BEAD1C5F814A00A2081
:104C600003F0CEFCC5F814800A2003F0C9FCC5F897
:104C700010800A2003F0C4FC0222C5F810A02846C8
:104C800003A98DF80F201C228DF80E20ADF80C9092
:104C900008F042FD434A03A894423A690BBF42F42C
:104CA000001242F480023A613A610BBF3A693A69F4
:104CB00022F4001222F480023A61A38823F44073A4
:104CC0001B041B0CA38023889BB243F001032380A9
:104CD000A58809F0D3F90599334B25F03F05B1FBC1
:104CE000F3F32D042D0C1D43ADB2A58022880025C1
:104CF00022F001021204120C22802C4A03A8B1FBFC
:104D0000F2F100298AB208BF012242F400414FF4B7
:104D1000967253434FF47A7293FBF2F301339BB2D2
:104D20002384A1832388009A9BB243F0010323804C
:104D3000238823F4816323F002031B041B0C2380CC
:104D40004FF480432381142303FB0626737B012445
:104D50008DF80C308DF80D508DF80E508DF80F40F9
:104D60000BF0D2FE337B9DF80F208DF80C308DF8C0
:104D70000D508DF80E501AB103A80BF0C5FE08E0D7
:104D80005A0903F01F039C4002F12003084A42F82D
:104D9000234009B0BDE8F08FD0790108300F002022
:104DA000001002400054004040420F00804F1200AB
:104DB00000E100E010B5214C2368998A89B211F412
:104DC000706F1CBF012284F82E2011F4E06F2BD0ED
:104DD0001A8B9A88890522F480624FEA02424FEAD0
:104DE00012429A8020D41A8892051DD41A88D005C0
:104DF0000FD51A88D105FCD41A8892B242F40072F9
:104E00001A801A889205FCD494F82D00FFF7DAFE78
:104E10000AE01A8892B242F400721A809A8822F448
:104E200040721204120C9A802268938A23F47063F1
:104E30001B041B0C93820023237610BD300F00202F
:104E4000064A08B5138801339BB21380044B93F8CC
:104E50002D00FFF7B7FE002008BD00BF660F002041
:104E6000300F002010B540001C4CC0B26072E171E0
:104E70000120002121746071227220762068E36095
:104E8000636184F82E1040B383889B0515D4038892
:104E9000D9050DD447F230530288920502D5013B63
:104EA000FAD112E08BB103889BB243F48073038084
:104EB00083889BB243F44073838047F23053227E51
:104EC00012B1013BFBD100E013B9BDE81040B7E7D8
:104ED000024B93F82E0080F0010010BD300F00202F
:104EE00007B5F7216B4606227620FFF7BBFF9DF83A
:104EF00000309DF801101B0343EA01139DF80210D6
:104F0000094A43EA111313629DF803309DF8041017
:104F10001B0343EA01139DF8051043EA1113D36103
:104F200003B05DF804FB00BF300F002007B5F62189
:104F300001AB03227720FFF795FF9DF805309DF820
:104F400004201B0243EA02439DF806201343054A4E
:104F5000B2F92020C2F10802D340034A936203B0A1
:104F60005DF804FB48020020300F002007B5F62151
:104F700001AB02227720FFF775FF9DF804209DF812
:104F8000053043EA0223024A938403B05DF804FB30
:104F9000300F002013B501220DF107033A2104461A
:104FA0006820FFF75FFF052003F02AFB9DF807301C
:104FB00003B10123237002B010BD13B506220446CD
:104FC000432168206B46FFF74DFFA8B19DF80020F4
:104FD0009DF80130012043EA022323809DF802203E
:104FE0009DF8033043EA022363809DF804209DF876
:104FF000053043EA0223A38002B010BD13B5062298
:1050000004463B2168206B46FFF72CFFA8B19DF8B2
:1050100000209DF80130012043EA022323809DF8FF
:1050200002209DF8033043EA022363809DF80420A8
:105030009DF8053043EA0223A38002B010BD13B5EA
:105040001F4B4000C0B2587202AC1868D97104F806
:10505000012D002101221A745C615971DC601A7201
:105060001A7683F82E1040B38288920515D40288F0
:10507000D4050DD447F230520188890502D5013A92
:10508000FAD112E08AB1028892B242F480720280B0
:10509000828892B242F44072828047F23052197E86
:1050A00011B1013AFBD100E012B9FFF7C9FE04E0EB
:1050B000034B93F82E0080F0010002B010BD00BF3A
:1050C000300F00202DE9FF415B4B1B689BB11A6834
:1050D0001AB15A49886902438A619A889868ADF87A
:1050E000042002228DF8072004220DEB02018DF826
:1050F000062008F011FB322003F08DFA0021112266
:105100001E20FFF79CFF012160221E20FFF797FF62
:10511000642003F080FA002402A808F03BF9274637
:1051200026460A25022101221E20FFF788FF322091
:1051300003F071FA02A808F02DF9BDF90820BDF9B5
:105140000A1014448A42A8BF0A46BDF90C300F4425
:1051500093421E44A8BF134613F5805F04DD013D52
:10516000E0D14FF0010801E04FF000081E200021BF
:105170001222FFF764FF0A25022101221E20FFF7F9
:105180005EFF322003F047FA02A808F003F9BDF9E8
:105190000820BDF90A10A41A8A42A8BF0A46BDF920
:1051A0000C307F1A9342A6EB0306A8BF134613F5F3
:1051B000805F02DD013DDFD101E04FF000082046B5
:1051C0000CF03AFB01461E480CF03EFC1D4D20F051
:1051D0000040286038460CF02FFB014618480CF0C0
:1051E00033FC20F00040686030460CF025FB01469F
:1051F00015480CF029FC20F00040A8600021702226
:105200001E20FFF71CFF012120221E20FFF717FFA1
:105210001E2002210022FFF712FF642003F0FBF999
:10522000B8F1000F04D14FF07E532B606B60AB6080
:1052300004B0BDE8F08100BF9002002000100240E1
:1052400000406F462400002001C05E467620F42115
:105250003122F4E6044B772093F82020F4219201C8
:10526000343202F0FC02EAE6480200207720F42102
:105270002E22E4E608B5FFF767FC6B218022682048
:10528000FFF7DDFE642003F0C6F96B2103226820DE
:10529000FFF7D5FE0F2003F0BEF90F4B19211A7846
:1052A0006820FFF7CCFE0F2003F0B5F90B4B1A2155
:1052B0001A786820FFF7C3FE1B2118226820FFF729
:1052C000BEFE1C2110226820FFF7B9FEBDE8084091
:1052D000682037210022B2E68C0200200000002066
:1052E000FFF76EB966E5FFF76BB963E507B52320F5
:1052F00003F091F96820752101220DF10703FFF7F2
:10530000B1FD28B19DF80700A0F16803584258414B
:1053100003B05DF804FB00BF4D282DE9F0470446BB
:1053200000F0548600F2B980302800F0B48651D8DD
:10533000222800F0908423D8032800F0058214D896
:10534000012800F0F581022840F0F48604200AF0DC
:10535000DBFD43200AF0A9FD4C200AF0A6FD462003
:105360000AF0A3FD4C2000F056BE042800F0F581A1
:10537000052840F0DF861A200AF0C6FD0024FCE173
:10538000282800F0E28515D8242800F0C9852628B1
:1053900040F0D086DA4C06200AF0B6FDB4F85C0185
:1053A0000AF0B5FDB4F85E010AF0B1FDB4F8600191
:1053B00000F0B3BD2C2800F0DB852E2800F05586C8
:1053C0002A2840F0B78601200AF09EFDCC4B587980
:1053D00000F021BE3D2800F0F8821ED8362800F0EB
:1053E0002B860BD8322800F01086342840F0A28695
:1053F00048200AF089FD002500F04FBC3A2800F053
:10540000B9823B2800F02084382840F0938604209D
:105410000AF07AFDBA4C00F089BD452800F0768686
:1054200027D8402800F0FA85422840F08386B44C03
:1054300010200AF069FD60790AF037FDA0680AF0D3
:105440006FFD94F892010AF030FDB4F85C010AF0A7
:105450005EFDB4F85E010AF05AFDB4F860010AF08E
:1054600056FDB4F882010AF052FDB4F8840100F050
:1054700054BD492800F0B4824B2800F09885462896
:1054800040F058860D200AF03FFD00200AF00DFD87
:1054900000200AF045FD00F044BE702800F0F082C4
:1054A00000F2E180692800F0458200F2B2806628AF
:1054B00000F0A08100F2A280642800F077816528C6
:1054C00040F038868F4C0B200AF01EFD20880AF031
:1054D0001EFD608880B20AF01AFD8B4B1B68C3F377
:1054E000C000C3F38002800040EA4200C3F34002E0
:1054F0001043C3F3401240EAC20003F01003184304
:105500000AF005FD814B1A88636802F0080103F474
:10551000475949EA010903F4804149EA010903F4C2
:10552000004149EA010903F4803149EA010903F421
:10553000003149EA010903F4802149EA010903F431
:10554000002149EA010903F4801149EA010903F045
:10555000007349EA0303DFF8D49112F0010F99F8C0
:10556000009018BF4FF00208C9F3800908BF4FF040
:10557000000843EA090312F0020F43EA080314BFCC
:105580004FF0040C4FF0000C12F0040F43EA0C0C27
:1055900014BF4FF0100E4FF0000E12F0400F14BF6A
:1055A000202700274CEA0E0E12F0100F14BF4FF404
:1055B000007600264EEA070712F0200F14BF4FF4C2
:1055C000806500253E4312F4807F14BF4FF40060D5
:1055D0000020354312F4007F14BF4FF40011002166
:1055E000284312F4806F41EA000114BF4FF080633A
:1055F000002300201943247A0346E7E0672800F0DF
:105600002181682840F0968510200AF07DFC002456
:1056100088E16C2800F0A18117D86A2800F0038483
:105620006B2840F0878505200AF06EFC384B1888FF
:105630000AF06DFC374B18880AF069FC314B93F87F
:105640006E0000F0010000F0E6BC6E282D4D00F069
:10565000978100F2CB8106200AF056FCE86D0AF033
:105660005FFC2D4B84E1782800F0F98018D874286D
:1056700000F034830AD8722800F09583732840F034
:10568000598508200AF040FC0124C5E3762800F083
:10569000EA8300F25C832F200AF036FC1F4CCBE239
:1056A000A42800F0068414D87B2800F06B82A02880
:1056B00040F040850C200AF027FC194B18680AF0CE
:1056C0002FFC184B18680AF02BFC174B186800F0D9
:1056D0002CBDF12800F0FF80FE2800F01184F02896
:1056E00040F02885074C04200AF00EFC236CB3F828
:1056F0005A000AF00CFC236CB3F8580000F00DBC03
:1057000054100020640F0020441800200C190020C1
:10571000C2180020C41800203C100020F7790108AE
:10572000E8F7FF1FECF7FF1FF0F7FF1F9230002094
:1057300003200AF0E9FB00200AF0B7FB20460AF03C
:10574000B4FB0D2000F067BC0AF0DEFB01200AF07C
:10575000ACFB0A200AF0A9FBA9E306200AF0D4FB5F
:105760004F200AF0A2FB4C200AF09FFB49200AF0D0
:105770009CFB31200AF099FBCEE3B04B185D01345D
:105780000AF093FB0B2CF8D10024AD4B185D0134CB
:105790000AF08BFB082CF8D10024AA4B185D0134C9
:1057A0000AF083FB072CF8D100F0C1BC07200AF0F7
:1057B000ABFBE7200AF079FBA34B58790AF075FBA5
:1057C00000200AF072FB042000F0AFBCA3420AD212
:1057D0009E4A9D5C012202FA05F50D421CBF9A40CB
:1057E00010430133F2E70AF09BFB974B93F8B007A5
:1057F00000F011BC12200AF087FB954B00241B8897
:10580000B3F5806F8CBF08250125924B33F9140046
:10581000013490FBF5F080B20AF079FB032CF4D14F
:105820008D4CA08C0AF073FBE08C0AF070FB208D8D
:105830000AF06DFB608D0AF06AFBA08D0AF067FB31
:10584000E08D6AE310200AF05FFB0024834B185DB3
:1058500001340AF02AFB102CF8D100F068BC70204B
:105860000AF052FB00260E2474437B4D01362B6C4C
:105870002344B3F819010AF04AFB2B6C2344B3F814
:105880001B010AF044FB2B6C2344B3F81D010AF002
:105890003EFB2B6C234493F81F010AF006FB2B6C94
:1058A000234493F820010AF000FB2B6C234493F867
:1058B00021010AF0FAFA2B6C234493F822010AF032
:1058C000F4FA2B6C1C44D4F823010AF029FB082EAF
:1058D000C9D100F02CBC70200AF016FB5A4C04F120
:1058E000700594F8D4000AF0E0FA94F8D5000AF0B4
:1058F000DCFA94F8D6000AF0D8FA94F8D7000AF047
:10590000D4FA94F8D8000AF0D0FA94F8D9000AF042
:10591000CCFA073494F8D3000AF0C7FAAC42E0D1CD
:1059200000F005BC4E4B185D01340AF0BEFA102C95
:10593000F8D1FCE34B4D00242878400000F0FE0035
:105940000AF0E2FA2B789C4280F0F183464B33F860
:1059500014000AF0DCFA0134F4E7444C06200AF0A3
:10596000D3FA20880AF0D3FA60880AF0D0FA404BC4
:105970001888D2E204200AF0C7FA374B186ED4E335
:1059800007200AF0C1FA3B4B1888FF28A8BFFF2068
:10599000C0B20AF08AFA384B186880F3100080B25F
:1059A0000AF0B5FAB5F864000AF0B1FA264B93F89C
:1059B0008721324B186822B10A23584380F3100024
:1059C00001E000F30F0080B2A7E21F4C02200AF0B2
:1059D0009BFA94F8E2010AF068FA94F8E1011AE3FC
:1059E00002200AF091FA184B988996E20B200AF0EF
:1059F0008BFAAB6E002618780AF057FAAB6E58781F
:105A00000AF053FAAB6E144C3344187901360AF09D
:105A10004CFA032EF6D1A36ED8790AF046FAA36E9B
:105A200098780AF042FAA36ED8780AF03EFAA36E8C
:105A300058890AF06CFAA36E187AECE2F89501081E
:105A400004960108D9950108541000206D0F00201C
:105A50001600002036100020640F0020940F002054
:105A6000A80F00202C2A00206C2F00206A2E002076
:105A70004410002034180020401800203C1800205A
:105A8000C04C1E200AF040FA236C00251B78022B24
:105A900065D1236C05F1080253F82200BA490BF0D6
:105AA0001FFF0FF055FC80F30800C0B20AF0FDF9AB
:105AB000236CB64903EB8503D86A0BF011FF0FF096
:105AC00047FC80F30800C0B20AF0EFF9236C05F13F
:105AD0000E0253F82200AE490BF002FF0FF038FC23
:105AE00080F30800C0B201350AF0DFF9032DD0D1F0
:105AF000072D236C21D1586CA3490BF0F1FE0FF058
:105B000027FC80F30800C0B20AF0CFF9236C9E494D
:105B1000986C0BF0E5FE0FF01BFC80F30800C0B2A0
:105B20000AF0C3F9236C93F84C000BF081FE0FF0E0
:105B30000FFC80F30800C0B20BE02B4458780AF049
:105B4000B4F9236C2B44D87A0AF0AFF9236C2B44B8
:105B5000587D01350AF0A9F90A2DC9D1E7E2236C75
:105B60002B4458780AF0A1F9236C2B44D87A0AF018
:105B70009CF9236C2B44587D01350AF096F90A2DC7
:105B8000EDD1D4E23C200AF0BFF900247D4D04F1B0
:105B900008022B6C7E4953F822000BF0A1FE0FF097
:105BA000D7FB80B20AF0B3F92B6C794903EB84037D
:105BB000D86A0BF095FE0FF0CBFB80B20AF0A7F984
:105BC0002B6C04F10E0253F8220071490BF088FE91
:105BD0000FF0BEFB013480B20AF099F9032CD5D145
:105BE000072C2B6C16D1586C69490BF079FE0FF01D
:105BF000AFFB80B20AF08BF92B6C6549986C0BF007
:105C00006FFE0FF0A5FB80B20AF081F92B6C93F8C0
:105C10004C000BE0234458780AF079F92B6C2344AC
:105C2000D87A0AF074F92B6C2344587D01340AF0B9
:105C30006EF90A2CD4D17AE214F8010F002800F092
:105C400076820AF032F9F7E701200AF05DF94D4B50
:105C50001B6C1878DFE150200AF056F90025494BFB
:105C60000C211C6C4B4B04EB850494F87920013516
:105C700001FB023393F838000AF017F994F87A0020
:105C80000AF013F994F87B000AF00FF994F87C00FD
:105C90000AF00BF9142DE2D149E23A4B1C6C0623B1
:105CA00003FB054494F8CE000AF0FFF894F8C9000D
:105CB0000AF0FBF894F8CA000AF0F7F894F8CB0061
:105CC0000AF0F3F894F8CC000AF0EFF8013594F8F4
:105CD000CD000AF0EAF80C2DDFD128E24FF00008E1
:105CE00001260027274B1A7A974227DA0933FA5CF4
:105CF00000240C236343274D05F13001595C914288
:105D000007D12B44586B0FF05AF982462EB9B14691
:105D100005E001341C2CECD10EE080440CE0D145B0
:105D20000ADA0C2303FB04535B6B13F809000AF037
:105D3000BCF809F10109F2E70137D3E7002E00F0C2
:105D4000F6815FFA88F00AF0DFF80026C9E70D4D0A
:105D50000024287A0AF0D8F82B7A9C4280F0E78158
:105D60000D4B0021E65C0C2202FB01F3094800F117
:105D70003007DA5DB24211D1034493F838000AF0DB
:105D800094F80EE0640F0020000020410000C8429B
:105D900000007A44F87901086D0F002001311C29B8
:105DA000E1D10134D8E7CE4C16200AF0ADF8B4F8B2
:105DB00098010AF0ACF8B4F844010AF0A8F8B4F875
:105DC00046010AF0A4F8B4F848010AF0A0F8B4F8C3
:105DD000DA010AF09CF894F8EF010AF066F8002066
:105DE0000AF063F894F8F0010AF05FF894F887017C
:105DF0000AF05BF894F894010AF057F800200AF0D2
:105E000054F8B84B0A201B6CB3F9563093FBF0F0F2
:105E100080B20AF07CF889E0E0B201340AF045F87B
:105E2000092CF9D183E110200AF06EF8AE4BAF4C8B
:105E3000187800F002000AF038F8AD4B18780AF034
:105E400034F820680AF06CF860680AF069F8A94B29
:105E500018880AF05CF8A84B18880AF058F8A14B8B
:105E6000B3F86C0059E00AF003F8074612200AF074
:105E70004BF89C4C17B9266F656F05E0102F19BFC2
:105E800000252E46A66FE56F38460AF00EF830461C
:105E90000AF046F828460AF043F8D4F880000AF0E1
:105EA0003FF800200AF033F800200AF030F8002014
:105EB000B1E08C4D002495F884002E46800001301E
:105EC000C0B20AF021F895F8840009F0EEFF96F8C8
:105ED00084309C4280F02B81884D285D09F0E5FFDD
:105EE00005F11003185D09F0E0FF05F12003185DCE
:105EF000303509F0DAFF285D09F0D7FF0134E6E715
:105F000008200AF001F800200AF001F8002009F04A
:105F1000FEFF002009F0FBFF002009F0F8FF06E17A
:105F2000042009F0F1FF6E4B9868FEE094F87C01C4
:105F300009F0BBFF94F8800109F0B7FF94F87F01E6
:105F400009F0B3FF94F8810165E0654C072009F082
:105F5000DBFFB4F8820109F0DAFFB4F8840109F03C
:105F6000D6FF94F8860109F0A0FFB4F88801D4E7C1
:105F70005B4C0C2009F0C8FF94F8920109F095FFE2
:105F8000B4F89C0109F0C3FFB4F8980109F0BFFF11
:105F9000B4F89A0109F0BBFF94F8930109F085FF6A
:105FA000B4F89E0109F0B3FFB4F8A001B5E74C4C7A
:105FB000042009F0A9FF94F8D80109F076FF94F8BD
:105FC000D90109F072FFB4F8DA01A6E74C4C4D4D47
:105FD0002078002600EB4000C0B209F095FF23783E
:105FE00002359E4280F0A38015F8020C09F05DFF97
:105FF00015F8010C013600EB800000EB800000F288
:10600000EE2080B209F083FFE9E7012009F07CFF70
:10601000334B93F8940109F048FF88E0082009F019
:1060200073FF00242E4B234493F88A01013409F0B6
:106030003CFF082CF6D17AE02A4B294C93F8C50096
:1060400004F12005C0EBC000C0B209F05DFF94F878
:10605000F60100232C4AD25C90426ED00C33302BD8
:10606000F8D10834AC42F2D161E0402009F04CFF95
:106070001B4C04F14005B4F8A80209F048FF94F85D
:10608000AA0209F012FF043494F8A70209F00DFFE8
:10609000AC42F0D14BE0E02009F036FF104C04F1A7
:1060A0008005B4F82A02043400F03F0009F02FFF05
:1060B000B4F82602C0F3861009F029FF94F82402F0
:1060C000000909F0F2FE94F8240200F00F0009F034
:1060D000ECFE94F8250209F0E8FEAC42E1D126E09E
:1060E00054100020640F0020481800205018002091
:1060F0004E1800204C1800204A180020E90F0020FC
:106100002C2A0020F6110020382A0020132009F044
:10611000FBFE0024144B185D013409F0C6FE0B2C65
:10612000F8D1002009F0FCFE002009F0F9FE012062
:10613000BDE8F0870020BDE8F08709F0B6FEB4F8AE
:10614000F80109F0E4FE94F8FA0109F0AEFE94F8C3
:10615000FB0109F0AAFE94F8FD0109F0A6FE94F8EF
:10616000FC0109F0A2FE7CE7F89501082DE9FF4744
:10617000CC4C07462378CC4E002B00F001823268CD
:106180006368D31A7C2B40F2FB81237A626001336F
:1061900023724FF0000808F12400C24DC0B20AF08B
:1061A0004DFF05F10A0333F918000BF045FBBF4B17
:1061B000814618880BF040FB014648460BF044FC32
:1061C000BB490BF08DFB0BF051FD08F1010800B24B
:1061D0000AF022FFB8F1030FDDD130200AF02EFFC4
:1061E000B5F910000AF018FF0AF020FF2B7A9A0781
:1061F0002CD141F288336A689A4218D910200AF0EB
:106200001DFF68694FF0640890FBF8F000B20AF0D7
:1062100003FF21200AF012FF686990FBF8F308FBE6
:1062200013000028B8BF404200B20AF0F5FE142067
:106230000AF004FFB4F918000AF0EEFE1C200AF080
:10624000FDFE00200AF0E8FE0AF0F0FE237ADFF8F7
:1062500054825B0740F0718102200AF0EFFED8F80B
:106260001C006423323090FBF3F000B20AF0D4FE3D
:10627000B8F926504FF0050A95FBFAF503200AF00D
:10628000DDFE8C4BADB21B78DFF83C9213F0040FAF
:106290000DD008F5D970394602F009F928B9D9F8B6
:1062A000003013F0100F18BF002528B205E0D8F811
:1062B00004389889B0FBFAF000B20AF0ADFED9F8C4
:1062C00000309F0740F18780DFF80092B4F808287B
:1062D00099F800304FF0640808FB02325B00B2FB13
:1062E000F3F3B4F80A7806203F01BFB247EA032768
:1062F000BFB2C3F303231F430AF0A0FE38B20AF073
:106300008BFEB4F80A3899F8001001339BB293FB66
:10631000F1F201FB1233A4F80A38D4F80C38614DBD
:106320009B7B012B05D139200AF088FEB5F90808BE
:106330001AE0B5F808586E235D43152795FBF7F56D
:106340003A20AFB20AF07AFEB7FBF8F528B208FBA4
:1063500015750AF061FE3B200AF070FEA8B2451DDB
:106360000A2095FBF0F000B20AF056FE28200AF051
:1063700065FED4F810380A2093FBF0F000B20AF062
:106380004BFE04200AF05AFED4F80438454F9D898C
:106390004FF6FF73D7F814089842A8BF1846ADB15E
:1063A0000028ACBF281A28460BF046FA42490BF0E9
:1063B00097FA074628460BF03FFA014638460BF09D
:1063C00043FB0BF053FC6428A8BF642020EAE07074
:1063D00000B20AF021FED4F81838324F9D0640F181
:1063E000A18097F81C3898071DD511200AF026FEC9
:1063F000B7F81E084FF4F3656843304B90FBF3F099
:1064000000B20AF009FE19200AF018FEB7F81E08BB
:106410004543642095FBF0F595FBF0F300FB13502A
:1064200000B20AF0F9FD94F81C38B4F8205813F0C3
:10643000020F08BF002501200AF000FE28B20AF072
:10644000EBFD09200AF0FAFD00200AF0E5FD1C4BE7
:1064500094F822581A88B2F5967F0AD9114B1B7A04
:1064600003F00F03072B04D842F20F75954228BFA3
:10647000154605200AF0E2FDD4F80C385B7B0BB919
:1064800028B22DE0A5F120000BF0D6F90D490BF054
:10649000DBFA002105460BF0C1FBC8B94FF07C5177
:1064A00018E000BF2C100020982E002016000020BD
:1064B00000007A44923000200000C842A08601000B
:1064C000460000206666E63F742E0020440000204F
:1064D0004FF03F4128460BF0FBF80BF0C7FB00B232
:1064E0000AF09AFD94F81C28C74B910703D493F83F
:1064F0002328012A04D1012384F82338C34818E053
:10650000D3F80C58C24968680BF0EAF90BF0AEFBFF
:10651000BF490290A8680BF0E3F90BF0A7FB0390CA
:1065200002A806E0BB4A02AB92E8030083E803003E
:1065300018460AF093FD0AF079FD237A282B1FD123
:10654000B14B00221A7233684FF47A70B3FBF0F843
:106550003C2717200AF072FDB8FBF7F5B5FBF7F002
:1065600007FB1050000200B20AF056FD18200AF096
:1065700065FD07FB158000B20AF04EFD0AF056FDDE
:1065800094F82C38A04D002B00F0638102F01CF829
:10659000D5F83038A04AC31A9342074640F2C78064
:1065A000002385F8363885F83838B5F80838DAB277
:1065B0001B0A85F8522885F8533885F8482885F84D
:1065C0004938D5F8602833689A1AD5F86438D97BE9
:1065D0004FF47A734B439A420ED3904B1B68C5F825
:1065E000603895F86838013B012B9FBF102385F870
:1065F0003638022385F83838D4F810280A20D4F821
:10660000143892FBF0F293FBF0F384F85028121246
:1066100084F8512884F8543894F81C281B1284F804
:10662000553894F822389207774984F8833803D490
:106630002D2381F8843878E0D4F824987848DFF85E
:10664000ECC199FBF0FA0CFB0A924FF0060E042BFA
:106650000EFB02F28CBF3323322381F88438714B56
:10666000D4F8286892FBF3F196FBF0F003FB1122BB
:10667000642592FBF5F20CFB006C0EFB0CFE84F81B
:106680007528121284F876289EFBF3F203FB12E3BE
:1066900093FBF5F30AEB8A0A4FFA81F80AEB8A0AB0
:1066A00008EB8A0189B284F8731800EB8000090AAC
:1066B00084F8741800EB800051B201EB800292B2B2
:1066C00084F87828120A84F8792884F87A38B4F89B
:1066D0001E281B1284F87B382423534393FBF5F5C3
:1066E000B4F896380A2284F87C381B0A84F87D387E
:1066F000B4F820384FEAD979B3FBF2F303F5FA7313
:106700009BB284F87E381B0A84F87F38B4F8983836
:10671000F60F84F87058C5F3072584F8729884F84A
:10672000776884F8715884F88538C4F8307894F81C
:106730009A88354DB8F1000F0DD1D5F8A00808F0B2
:10674000A0FB012807D90228374E00F0608202F032
:1067500067FD0123B370D4F8A4282B4D002A78D00C
:1067600095F89A683EB140F6B731D5F8AC38FB1AC7
:106770008B4219D86DE00123D5F8A00885F89A3826
:1067800001F00AFDD5F8B038082193F90000022382
:106790008DE8480032464FF4964301F082FF85F8B9
:1067A000B468C5F8A00852E095F8A868CEB9D5F845
:1067B000A008C5F8A46885F89A6801F0EDFCD5F842
:1067C000B038082193F9000001238DE848003246D3
:1067D0004FF4964301F065FFC5F8A00802F020FDD4
:1067E00035E0013EF6B285F8A86895F8B41895F83A
:1067F000B538EEB94A1C013385F8B42885F8B538A8
:10680000D5F8A00821E000BF2C100020501800206F
:106810008096184B847B01083F0D0300982E0020C2
:106820008096980040420F0016000020806967FFA4
:1068300012F8016B01337018314685F8B408D5F8A9
:10684000A008C5F8A42885F8B53808F01DFBC4F8E1
:10685000AC7894F8B638A14DF3B1D5F8B838DBB1BF
:10686000D5F8BC38C3B1C5F8C0381B689C4AC5F818
:10687000C438D5F8C8381344187AFEF74DFDD5F85A
:10688000C038987909F011FBD5F8C8380133092BC5
:1068900088BF0023C5F8C838924D94F8CC282E68DC
:1068A0008E4B002A00F0EE81D3F8D028002A00F0A9
:1068B000E98193F8D438013B012B00F2E381D4F84D
:1068C000D008864F08F0DDFAE0B1D7F8D00808F01C
:1068D000D5FA97F8D53880467E2BD5F800900ED1A2
:1068E00002231B2887F8D43809D1D7F8D00808F03C
:1068F000C8FA20B90123C7F8D89887F8DC3884F89B
:10690000D588DCE7D7F8D8282B689B1A41F658328F
:1069100093421ED9032387F8D438B3E1724A32F880
:10692000130010B903464FF403600133B0F5C06F94
:10693000DBB279D01ED9B0F5006F7FD032D9B0F577
:10694000036F3FD184F8DD38D4F81838634F9906C7
:106950003FD494F8DC1894F8DD38002900F0548115
:106960002A68921B012AD9D984F8DD38002384F8DB
:10697000DC3887E1B0F5007F43D007D8B0F5807FE1
:1069800049D0B0F5887F00F08B80E6E7B0F5806FE6
:1069900000F0AE80B0F5826F00F0F380B0F5047FB8
:1069A000DBD123E0B0F5E26F00F08B80B0F5E46F4F
:1069B00000F08C80B0F5E06FCFD184F8DD38B4F909
:1069C0000A1087E0B0F5046F74D0B0F5026FC4D13F
:1069D00003E197F81C389A07BBD5B7F81E18242393
:1069E0004B436421123393FBF1F107E184F8DD3866
:1069F0003E4B3A4F1B689B07ABD5B7F808380A21C6
:106A0000FBE084F8DD38394B344F1B681905A0D5FD
:106A1000D7F81018F2E084F8DD38D4F818382F4F82
:106A20005A0796D57969E9E084F8DD382F4B2B4F6A
:106A30001B681B058DD5D7F81418DFE0D4F818189B
:106A4000264A8F0684F8DD3883D592F81C1888070B
:106A50007FF57FAFD90711D5D2F82838192283EAFC
:106A6000E371A1EBE37101EB5101B1FBF2F1002BFA
:106A7000ACBF41F0004141F040410EE0D2F8243873
:106A8000192283EAE371A1EBE37101EB5101B1FB40
:106A9000F2F1002BB8BF41F080414FF400608BE071
:106AA00084F8DD38D4F818380C4F5B077FF551AF08
:106AB0003969A3E084F8DD38B4F91830642159430A
:106AC0007AE084F8DD38B4F90C1003E0B4F90E1064
:106AD00084F8DD382C2391FBF3F16DE02C100020BD
:106AE000847B0108982E00201A9A0108742E002039
:106AF00084F8DD3894F8DE38644A0133DBB2032BC6
:106B000088BF012382F8DE3842F2107394F8DE1851
:106B100059435F4B1B78D80748BF01319A0748BFDC
:106B200002315F07B4F8E03848BF0431D80748BFE6
:106B30000A319A0748BF14311F0648BF2831D805CB
:106B400048BF28315A0748BF64311F0748BFC831C2
:106B5000980548BF01F5C8719A0648BF01F57A71DA
:106B6000DF0648BF01F5FA61580648BF01F57A61B2
:106B70004FF4806002F020FB444B002283F8DC28B5
:106B8000E7E6D4F81818DFF8048111F0200784F83C
:106B9000DD3817D098F81C2812F0020F14BF4FF4FC
:106BA0007A71002112F0010F14BF4FF4FA63002331
:106BB0000B4494F82218194402F0FEFA002384F8DA
:106BC000DC38C6E6334B1B6819067FF5C2AE394682
:106BD00002F0F2FA88F8DC78BBE684F8DD38D4F805
:106BE00018382A4F9A067FF5B4AE97F81C389B07E1
:106BF0007FF5AFAEB7F820386421594302F0DCFAD4
:106C0000002387F8DC38A4E684F8DD383AE0B3786E
:106C100023B1C5F89C7886F802809CE5D5F89C38AD
:106C2000FB1AB3F57A6FFFF496AD0123D5F8A008EF
:106C3000B37008F023F90646D5F8A00808F01EF94D
:106C400076067FF488AD8A2802D08E280DD082E5A2
:106C5000D5F8183898067FF57EAD95F89A38002B50
:106C60007FF479AD05F6690306E095F89A38002BB4
:106C70007FF471AD05F63403C5F8A4382D2385F8EB
:106C8000A83868E504B0BDE8F08700BF2C100020EC
:106C900092300020742E0020F0B50124B0FBF4F5F2
:106CA0008D4201D34C43F9E70026D4B1B0FBF4F593
:106CB00004FB1500B4FBF1F41EB9002D01DC002C1F
:106CC000F3D1092D03F1010EEFB204DD002A14BF48
:106CD0003725572500E030253D441D7001367346A9
:106CE000E3E71C70F0BDF0B50124B0FBF4F58D4274
:106CF00001D34C43F9E70026D4B1B0FBF4F504FB13
:106D00001500B4FBF1F41EB9002D01DC002CF3D109
:106D1000092D03F1010EEFB204DD002A14BF37255F
:106D2000572500E030253D441D7001367346E3E7EA
:106D30001C70F0BD03685A1C0260197070472DE981
:106D4000F843089E002B074688461446334614BF76
:106D50004FF030094FF0200913F8012B0AB92546EE
:106D600003E0002CFBDD013CF6E7002D04DD384696
:106D70004946C047013DF8E7354624EAE474A01BC4
:106D8000284415F8011B11B13846C047F7E7BDE8A4
:106D9000F883024B186808F077B800BF200F002076
:106DA000F8B507460C464868002115461E460AF00D
:106DB0002BFF58B128460AF03FFD10490AF090FD1C
:106DC00001464FF07E500AF03FFE60606168304639
:106DD0000AF07EFC014630460AF036FE256806467B
:106DE000294638460AF072FC014630460AF078FD22
:106DF000014628460AF06CFC2060F8BDDB0FC94054
:106E00002DE9F04102780346202A00F10100F9D073
:106E1000092AF7D02D2A02D10346414D04E02B2A3E
:106E200008BF03464FF07E551C460026234614F843
:106E3000012BA2F13007F9B209290DD839493046A2
:106E40000AF04EFD064638460AF0F6FC014630468A
:106E50000AF03EFC0646E9E72E2A17D1314F2346B9
:106E600014F8010B3038C2B2092A0FD80AF0E4FC3A
:106E700039460AF0E9FD014630460AF029FC294965
:106E8000064638460AF02CFD0746E8E71A7802F075
:106E9000DF02452A39D15A782D2A02D1023301273F
:106EA00004E02B2A14BF013302330027013B0024E6
:106EB00013F8012F303AD1B2092903D80A2101FB76
:106EC0000424F5E7B4F59A7F28BF4FF49A74A046DE
:106ED0004FF07E53B8F1070F07D9184612490AF050
:106EE000FFFCA8F108080346F4E704F0070434B1F6
:106EF00018460C490AF0F4FC013C0346F7E7194632
:106F00002FB130460AF0A0FD04E04FF07E5130462C
:106F10000AF0E6FC014628460AF0E2FCBDE8F081F2
:106F2000000080BF0000204120BCBE4C30B50546AB
:106F300087B00C4603A800210C220DF0FCFF284668
:106F400000210AF089FE20B1284628490AF0C0FB3A
:106F500003E0284625490AF0B9FB25490AF0C0FCA0
:106F60000AF084FE054680EAE0706946A0EBE57011
:106F700006F062FF002DACBF20232D2368468DF85C
:106F80000C300EF01CF8012807D130238DF80D309D
:106F90008DF80E308DF80F300CE0022805D130232B
:106FA0008DF80D308DF80E3004E0032804BF302337
:106FB0008DF80D30694603A80DF0E4FF03A80DF02D
:106FC000FEFF0338C5B22A4603A920460EF022F878
:106FD00000236355204607490DF0D4FF03AB20463C
:106FE00059190DF0CFFF204607B030BD6F12033A9C
:106FF00000007A443A9A010870B50646B6FBF2F4EE
:107000000846154614B12046FFF7F6FF05FB146449
:10701000024B1B5D00F8013B70BD00BF3C9A0108AC
:107020002DE9F04F81468A4616461C4689B0002558
:107030003178002900F0DB80252902D0013648464E
:1070400074E072784FF00008302A0CBFB278B71C99
:10705000A2F1300312BF4FF0000BF71C4FF0010BF1
:10706000092B19D8A2F13003D9B2092905D80A226F
:1070700002FB083817F8012BF4E7A2F16103052B96
:1070800002D8A2F1570305E0A2F14103052B03D872
:10709000A2F137030A2BEADD6C2A30D13A787E1C44
:1070A000642A00F083800BD8252A3DD003D8002A1B
:1070B00000F09D80BCE7582A0CD0632A19D0B7E7AE
:1070C000732A22D002D86E2A37D0B1E7752A5CD055
:1070D000782AADD1271D2068A2F1580462424FF0F2
:1070E0001001624155E02CD9582A32D0632A2AD1A6
:1070F0003E4648462178271DD04701350FE0642AD7
:1071000063D00ED9732A14D13E46236848460093B3
:10711000514642460023FFF712FE271D05443C4618
:1071200086E7252ADFD13E4648462521D04701354E
:107130007EE70AD86E2A06D13E46236804341D60D5
:1071400076E7002A53D03E4672E7752A26D0782A81
:10715000F9D1A2F1580304F1040C5A422068CDF889
:107160000CC04FF010015A4105ABFFF795FDDDF85B
:107170000CC03E46644605AB009348465146424625
:107180005B46FFF7DCFD054452E72068271D0A2116
:10719000002205ABFFF7A7FD3C46ECE704F1040C29
:1071A000CDF80CC020680A210022DDE72068271DE9
:1071B000002808DA2D238DF8143040420DF1150314
:1071C0000A210022E6E705ABFAE7206804F1040C87
:1071D00000280ADA2D238DF8143040420DF11503F2
:1071E000CDF80CC00A210022BFE705ABF8E728461E
:1071F00009B0BDE8F08F0FB413B50B4904AB0868B4
:107200000A4953F8042B09680193FFF709FF044664
:10721000074B186801F08EFA0028F9D0204602B01A
:10722000BDE8104004B07047CC000020C80000202A
:10723000200F002080EAE073A3EBE0738B4206DBB3
:10724000002801DD401A704702D008447047002032
:10725000704770B504460AF009FD2030402857D821
:1072600020462C490AF0F8FC28B120462A490AF0A9
:107270002DFA0446F4E7204628490AF0CFFC28B14D
:10728000204625490AF024FA0446F4E7204624491A
:107290000AF0E2FC30B1224920460AF017FA014612
:1072A0001F480AE020461F490AF0B8FC40B11C49BB
:1072B00020460AF00DFA01461A480AF007FA044679
:1072C000214620460AF00CFB0546204629460AF0D6
:1072D00007FB1549064628460AF002FB13490AF047
:1072E000F5F9014628460AF0FBFA11490AF0F0F9CF
:1072F000014628460AF0F4FA0E490AF0E7F9014679
:1073000030460AF0EDFA014620460AF0E1F970BD78
:10731000002070BDDB0F4940DB0FC940DB0F49C0C7
:10732000DB0FC93FDB0FC9BF9A7C2E36FAAF4F394E
:107330003587083CA4AA2A3E08B503490AF0C8F9D3
:10734000BDE8084085E700BFDB0FC93F2DE9F04FDE
:10735000056885B0814628460C46FFF7EDFF80465C
:107360002846FFF776FFD9F8045006462846FFF76F
:10737000E3FF07462846FFF76CFFD9F8089005465B
:107380004846FFF7D9FF82464846FFF762FF41466D
:10739000814650460AF0A4FA4146834648460AF020
:1073A0009FFA5146019030460AF09AFA49460290F7
:1073B00030460AF095FA3946039050460AF090FAA2
:1073C0004946206007F100400AF08AFA29466060C9
:1073D000A56002980AF084FA014601980AF078F94B
:1073E0002946E06003980AF07BFA014658460AF005
:1073F0006DF93946206106F100400AF071FA29461C
:10740000606158460AF06CFA014603980AF05EF98A
:107410002946A06101980AF063FA014602980AF031
:1074200057F94146E06138460AF05AFA206205B041
:10743000BDE8F08F2DE9F04107688AB0466885689D
:107440000446084601A9FFF781FF019938460AF072
:1074500047FA0499804630460AF042FA014640460F
:107460000AF036F90799804628460AF039FA0146AB
:1074700040460AF02DF90299206038460AF030FAA9
:107480000599804630460AF02BFA014640460AF03C
:107490001FF90899804628460AF022FA014640461C
:1074A0000AF016F90399606038460AF019FA06994D
:1074B000074630460AF014FA014638460AF008F941
:1074C0000999064628460AF00BFA014630460AF0AA
:1074D000FFF8A0600AB0BDE8F081074B10B51A882C
:1074E0001C4622EA00009042188002D0012001F0E0
:1074F00053F8208810BD00BF0C190020064B10B5B2
:107500001A881C4610439042188002D0012001F0D6
:1075100043F8208810BD00BF0C190020024A936870
:1075200023EA0000906070475410002008B5104B0B
:107530001A780023D9B2914207D20E49002051F89F
:107540002310013309680880F4E7322001F063F862
:10755000094B1B685A0309D5084B9B685B0305D48C
:10756000BDE8084040F2DC5001F055B808BD00BF4E
:10757000F72B0020F82B0020742E00205410002040
:107580002DE9F3410AF054F84B4A6923137040F295
:10759000DC735380BE231371EF2382F8D9370023A5
:1075A0001946164682F8DA37F25C0133514040F250
:1075B000DC729342F8D1404B404A83F8DA17404BD3
:1075C00004275A6002F188325A600020013F17F008
:1075D000FF075ED03A4B34223A4CDA6004F1784827
:1075E000A8F5FC38C8F3090353B100234FF4005049
:1075F00056F80880019306F091FD0428E6D11CE0BE
:107600004FF4302006F08AFD0428DFD12C4D4FF4D2
:1076100030202B6943F002032B616C612B6943F02E
:1076200040032B6106F07AFD41F6FD732A690428B8
:1076300003EA02032B61D8D0C8E7214D4FF4005074
:107640002B6943F001032B611FFA88F3238006F0B6
:1076500065FD042813D1A31C0193019B4FEA184830
:10766000A3F800804FF4005006F058FD41F6FE7379
:107670002A69042803EA02032B6106D0A6E741F633
:10768000FE732A6913402B61A0E70F4B04349C4220
:10769000A4D10B4A0428136943F08003136102D17B
:1076A00008F0C0FE10B9052000F0BFFF09F0AAFFE6
:1076B00002B0BDE8F08100BF5410002023016745EF
:1076C0000020024000F80108DCFF010810B50E4C54
:1076D000206800F09DFE20680022047A02FB02F37D
:1076E000193B634303F6C4135343192193FBF1F38E
:1076F000064921F812300132072AEFD1BDE81040C7
:10770000034900F03DBE00BFCC0F0020F00E00206A
:10771000981100202DE9F04108F084FE10B90420F2
:1077200000F083FFBF4C09F083FFBF4940F2DC72D9
:1077300020460DF0F5FB94F8B0374FF4CC71022BD6
:1077400084BF002384F8B03794F8B027B74D01FB0D
:1077500002F303F53A7020442344286093F83C0375
:1077600001FB0242022803F54E7384BF002018710A
:1077700092F83C33AE4A13700C2202FB0343AD4A2D
:1077800003F2B273136046F20902A3681A401AB9F1
:10779000A44A43F400539360A368DE0703D54FF473
:1077A0000050FFF7BBFEA368580409D50820FFF777
:1077B000B5FE4FF40050FFF7B1FE0120FFF7AEFE1B
:1077C000A368190706D54FF40050FFF7A7FE012064
:1077D000FFF7A4FEA3689A0413D54FF40040FFF707
:1077E0009DFE904B93F88631012B03D14FF400603E
:1077F000FFF794FE4FF48030FFF790FE4020FFF734
:107800008DFEA3685B0603D54FF48030FFF786FE3C
:10781000894B1B6803F42063B3F5206F07D194F8FC
:107820008631012B03D14FF40060FFF777FE94F807
:10783000E0217C4B2AB193F8E42112B1002283F8B5
:10784000E4214FF0000C67467C4E7D4B1E6004EB3C
:107850000C03B3F8F8E14FEA5E0101F077314FEA2B
:107860009E0303F03333C1EB0E00C11A4FEADE036F
:1078700003F01133CB1A03EB231303F00F32FF2372
:1078800092FBF3F31EF00108C3EB032318BF01378B
:10789000A2EB030318BFFFB2012B0ADD022B40F05D
:1078A000BE80B8F1000F00F0BA801EF0BC0F00F0EF
:1078B000B6800CF1080CBCF1200FC8D1013F012F9C
:1078C00000F2AD80FFF702FF302200215D480DF08D
:1078D00032FB5D4F5D4BD5F800801F605C4B002193
:1078E00008F17900C3F8008000F0D0FD594B80F01A
:1078F00001001870584B07F126021A60574B07F128
:10790000D4021A6098F8000007F02AFD2868544B4A
:1079100000F5C5721A6002F0B5F8524B94F8D81110
:1079200007F194021A6064224A434F4BC8325A60EE
:1079300000229A60DA601A615A619A61DA6183F80A
:10794000202083F82120494B2D6807F12C021A6072
:10795000474B05F219121A60464B05F289121A605C
:10796000454B07F108021A60444BDFF84C811F6059
:10797000434B07F1A0021A6007F1AA03C8F80030D0
:10798000404BB4F866011E6009F052FFC8F80800C9
:10799000B4F8680109F04CFF95F85C3008F1040276
:1079A00088F8043095F87830C8F80C0088F805306D
:1079B00094F8E331286E88F81030334BC8F814502F
:1079C0001A60324B05F164021A60314909F088FFF0
:1079D00001464FF07C500AF037F8B5F816412D4BB0
:1079E0001860204609F028FF01462B480AF02CF8C1
:1079F0002A4909F075FF2A4A2A4B15602A4A18605D
:107A000005F168031360294A05F211151560284A2B
:107A10001760284ABDE8F041136009F0F3BD06F095
:107A2000C3F94FE75410002000F80108A40F00200C
:107A3000202E0020CC0F0020742E0020DE1100200C
:107A400038300020240E002098110020580E00200D
:107A50005C0E00201400002038060020DC05002009
:107A6000680E0020D0230020443000209006002023
:107A70002C1F002094080020C82C0020CC2C0020B3
:107A8000A80700206C080020C0060020F80600208F
:107A9000DB0F4940F4060020000061444C3D0F44D8
:107AA0000C1D0020A4070020001D002098070020C6
:107AB000A0070020F81B00201019002008B5FFF7D0
:107AC0005FFDFFF727FEBDE80840012000F064BD20
:107AD000F8B504460E4617460025204620210DF035
:107AE00060FA0446D0B1013420460DF0BDFAB0F57D
:107AF000617F05DB40F634039842A8BF184601E0D9
:107B00004FF46170A0F56170192390FBF3F00DB98B
:107B1000307000E070703B7801333B700DB9012587
:107B2000DBE72046F8BD30B505460C46134629462E
:107B30002246BDE830400148FFF75DBB349B010899
:107B40007FB504780646E4B9354B1921186800EB77
:107B5000840090F87B5090F879204D4305F56175CD
:107B600090F87A30009590F87C00414301F56171FE
:107B700001912C4821460134FFF73DFB142CE3D141
:107B80004BE00DF071FA1328054641DC244B701CC4
:107B90001C68202100238DF80F300DF002FA1E35ED
:107BA000064670B1013630460DF05EFA1A289FBFC6
:107BB00004EB850358709DF80F30013398BF8DF8A2
:107BC0000F30304620210DF0ECF9064670B1013639
:107BD00030460DF049FA0D289FBF04EB85039870DD
:107BE0009DF80F30013398BF8DF80F3004EB8504FA
:107BF0003046E11C0DF10F02FFF76AFF9DF80F30D0
:107C0000042B0AD0601C002104220DF094F904E03A
:107C1000054800211322FFF786FF04B070BD00BFA6
:107C2000A40F0020539B0108689B0108014808F03D
:107C3000EFB900BF6E9B0108F8B50478064674B929
:107C4000304D2146B5F8C621B5F8C8312E4801346B
:107C5000FFF7D1FA042C05F10405F2D1F8BD2B4948
:107C60000DF072F9A8B9274B4FF47A714FF4FA620C
:107C7000A3F8C611A3F8C821A3F8CA11A3F8CC2110
:107C8000A3F8CE11A3F8D021A3F8D211A3F8D421E0
:107C9000F8BD30460DF0E8F9032805462BD83046EC
:107CA00020210DF07EF9044630B1013420460DF05C
:107CB000DBF90126074600E00646204620210DF0AC
:107CC00070F910B9BDE8F840B0E701300DF0CCF91B
:107CD000012EF7D140F2DC53A7F2EE229A42F1D8FE
:107CE000A0F2EE229A42EDD8064B703503EB8503E5
:107CF000DF801881F8BD064800210322BDE8F84066
:107D000011E700BF541000207C9B01088F9B0108E5
:107D1000A1A601082DE9FF4104780546002C34D1C5
:107D20006D4808F075F96D4D6869002109F06CFF28
:107D3000002840F0CE8021466948FFF75CFA686968
:107D40006946FFF7F3F801466648FFF754FAA86959
:107D50006946FFF7EBF801466248FFF74CFAE8691D
:107D60006946FFF7E3F801465E48FFF744FA286AE0
:107D70006946FFF7DBF8013401465B48FFF73BFA41
:107D80000C2C05F11005CFD1A3E0584905220DF0C8
:107D90001FF938B9514B002203441030C0285A61F2
:107DA000F8D196E02846524904220DF011F9044614
:107DB0002846002C3FD120210DF0F3F8002800F0D8
:107DC0008880451C28460DF0FAF80746494B53F8C1
:107DD00024601EB9484808F01BF97AE0284631466D
:107DE000FAB20DF0F5F801340028EFD13B4B002139
:107DF000C2181030C02851619E46F7D13F4B03EBAB
:107E0000C402D2F804C09846BCF1000F04D1314638
:107E10003B48FFF7F0F953E0002718F834309F4251
:107E2000F5DA3B010EEB0305143563440FCB013744
:107E300085E80F00F1E70DF017F90B28064643DC43
:107E4000284620210DF0ADF8054648B101352846F9
:107E5000FEF7D6FF214B012403EB0613586100E027
:107E60000446284620210DF09CF8054640B1013516
:107E70002846FEF7C5FF194B013403EB0613986142
:107E8000284620210DF08DF8054640B101352846E1
:107E9000FEF7B6FF114B013403EB0613D8612846F9
:107EA00020210DF07EF810B9FFF7C0FE11E001307F
:107EB000FEF7A6FF094B032C03EB06163062F3D145
:107EC0001048FFF727FF04E00F4801210C22FFF7BD
:107ED0002AFE04B0BDE8F081959B010854100020F3
:107EE000B09B0108B69B0108B5A301088F9B010850
:107EF000BA9B010820930108BF9B0108649A0108FE
:107F0000CE9B0108FB980108689B0108F0B5047836
:107F100087B0064614BB514B19201968062303FB92
:107F2000041191F8CA5091F8CE20454305F56175CA
:107F300091F8C930009591F8CB50C831684300F5ED
:107F40006170019008790290497945480391214672
:107F50000134FFF750F90C2CDDD17CE00DF084F8F2
:107F60000B28044672DC3D4B701C1D682021002349
:107F70008DF817300DF015F8064680B10136304601
:107F80000DF072F803289FBF062303FB045383F808
:107F9000CE009DF817309CBF01338DF81730304666
:107FA00020210CF0FEFF074680B1013738460DF066
:107FB0005BF80D289FBF062303FB045383F8C90019
:107FC0009DF817309CBF01338DF8173006266643A5
:107FD000A9193846CA310DF11702FFF779FD2021A2
:107FE0000CF0DFFF074670B1013738460DF03CF862
:107FF00014289FBF9DF817307619013386F8CC00FE
:1080000098BF8DF81730384620210CF0CAFF78B1A0
:1080100001300DF029F80D289FBF062303FB045300
:1080200083F8CD009DF817309CBF01338DF81730D1
:108030009DF81730062B0ED0062202FB04500021BB
:10804000C9300CF078FFFFF7F1FD04E0054800218E
:108050000B22FFF768FD07B0F0BD00BFA40F0020A2
:10806000DA9B0108689B01082DE9F347047806466E
:108070004CB9204601A905F0DFFE0134FFF7F4FFFB
:10808000122CF6D17AE00CF0EFFFC5B2112D70D8AA
:108090003C4C05F1D00704EB4703701C202193F8FA
:1080A00002800CF07EFF384E034630B9A8F1020280
:1080B000D2F1000848EB020845E000F1010A5978C6
:1080C00030460CF06EFF60B1032D8CBF03230023FC
:1080D000801BC0B23344184490F80490B9F1030FE8
:1080E00002D1FFF7A3FD49E0A9F10203D3F1000893
:1080F00050464FF0200148EB03080CF052FFD8B176
:10810000B8F1000FEDD001300CF0AEFF40F2ED23DE
:1081100080B2984205DD40F6CA039842A8BF1846CF
:1081200001E040F2EE20A0F2EE20192290FBF2F0E6
:1081300004EB4703D87002E0B8F1000FD1D104EB93
:10814000470383F8029004EB4704A378F25CB8F18C
:10815000000F09D0E17819234B430C48294603F25C
:10816000EE23FFF748F809E029460948FFF743F8EE
:1081700004E0084800211122FFF7D5FC02B0BDE859
:10818000F08700BF54100020987B0108FA9B01087B
:108190000C9C0108A1A60108002208490C2303FB3E
:1081A00002135968814204D10022C2621A725A60D5
:1081B00070470132042AF0D1704700BF382A0020EE
:1081C00010B5084B0022196801EBC20393F9024075
:1081D000844201D1981C10BD0132042AF4D1002040
:1081E00010BD00BF342A0020F0B5027887B08AB9EC
:1081F0004A4C04F1200694F8F6210023484950B275
:10820000595681426DD00C33302BF7D10834B4422B
:10821000F1D180E0002204920592451C0CF024FF6D
:10822000C4B260B2FFF7CCFF074618B18DF810401A
:10823000012400E00446284620210CF0B2FE054649
:1082400038B1013528460CF00FFF0134ADF81200AB
:10825000E4B20026284620210CF0A3FEB0B3451C52
:1082600028460CF001FF00222E495FFA82FE51F8E9
:108270002230834204D00132082AF5D1002300E0E5
:10828000734651F82320824220D1022E0FD0032EB4
:1082900012D05A1E012ED2B204D0042A13D88DF85F
:1082A00014300EE0042A0ED88DF8153009E0052BA5
:1082B00009D88DF8173004E09A1E052A03D88DF8E6
:1082C00016300134E4B20136042EC3D1052C03D894
:1082D00007B0BDE8F040A9E404AB03CB3860796097
:1082E00019E094F8FB010F4B94F8FA5153F8200071
:1082F000B4F8F821009094F8FD0153F820000190A3
:1083000094F8FC0153F8200053F8253002900648F9
:10831000FEF771FF7AE707B0F0BD00BF54100020F0
:10832000382A00208C8401081B9C010838B143883E
:1083300011EA030003D08B420CBF012002207047DA
:1083400030B50A4B0A491C680A78032A0AD8134632
:10835000551C04EBC303EAB29D882842F5D00A708D
:10836000981C30BD0A70002030BD00BF342A0020A8
:1083700028190020014B00221A70E1E7281900207B
:108380002DE9F047877890F803C0BBB2C7F1640EBF
:1083900003EB83065C42C3F178001C4D5FFA8EFE4E
:1083A0007600CCF16408A4B280B2A3B20FFA83F9CC
:1083B000B9F1000F04DC002B14BF3B46012300E0A1
:1083C000734609FB09F25B4302FB0CF292FBF3F3E9
:1083D000434403FB09F30A2293FBF2F333449BB2B9
:1083E00025F8023FB1F800904A880A34C9EB020A26
:1083F0001AB202FB0AF24FF47A7392FBF3F3A4B2BF
:108400004B4484422B80D0D1BDE8F087281900204E
:1084100010B544780078002240F6C41102FB02F344
:10842000193B634303F6C4135343434393FBF1F3F4
:10843000034921F812300132072AEDD110BD00BFE7
:1084400042190020104B043033F91000B0F5617F61
:1084500005DB40F633039842A8BF184601E04FF40D
:1084600061700A7819235A4302F28332824208DA91
:108470004A78534303F283338342B4BF0020012080
:1084800070470020704700BF6C2F002010B500F12E
:10849000500302788A4203D18478C278944204D38C
:1084A00004309842F5D1002010BD012010BD0B4BC7
:1084B0001B6813F4805F0A4BB3F9063005D0C089FE
:1084C000421A934207DD084400E0008A8342B4BFA9
:1084D0000020012070470120704700BF742E00204B
:1084E0006C2F00201FB5084B1B681B0309D58DF8A6
:1084F0000400039101230D2001A98DF8053000F03F
:10850000B7FA05B05DF804FB742E00201FB5084BC8
:108510001B681B0309D58DF80400029100230D2070
:1085200001A98DF8053000F0A3FA05B05DF804FB51
:10853000742E002038B5064C002584F8285009F028
:1085400099F884F82950E5622586656338BD00BF37
:108550002819002010B510B9BDE81040EAE7002343
:108560000C225A430A4C1119125D824203D0013386
:10857000102BF5D110BD074B586B18B14A784078D5
:10858000824203D2002259631A86DA6210BD00BF0C
:10859000C48401082819002010B540001428A8BF81
:1085A00014200023074A022199540B4499181424DB
:1085B000834201F8014CF5DBFF21D1540F20BDE8C7
:1085C0001040C7E74C2E002010B50A4A0A4B11682C
:1085D0009B6800BF12689142F7D1084A4FF47A7045
:1085E000946B00FB04F2D31AB3FBF4F300FB0130ED
:1085F00010BD00BF982E002010E000E028190020D8
:1086000038B50446FFF7E0FF0546FFF7DDFF401BE6
:10861000A042FAD338BD10B504462CB14FF47A709D
:10862000FFF7EEFF013CF8E710BD2DE9F041804671
:108630000B25013D19D008F10106322705243846E3
:10864000FFF7E9FF3846FFF7E6FF3CB1013CF6D102
:108650004FF4FA70FFF7DFFFFA27F0E7013EEED1A3
:108660004FF47A70FFF7D7FFE3E7024A024BDA6074
:10867000BDE8F0810400FA0500ED00E0024A13684D
:1086800001331360704700BF982E0020024BDB6B54
:1086900003B11847704700BF2819002003685B69C1
:1086A00018472DE9F743064689469DF8288011466C
:1086B0001A469DF82C3000250C2068431A4FC41927
:1086C000C057B04202D1207A20B126E00135042DF6
:1086D000F2D122E0012E0AD003DCF6B90093134850
:1086E00007E01E2E0AD01F2E17D1012006E01048E9
:1086F0000093434603F06DFA044605E005F03EF8AA
:1087000041460446FFF7CAFF4CB10C2303FB057535
:10871000267185F808906C6001E0002000E020469A
:1087200003B0BDE8F08300BF382A002000380140C4
:108730000044004003681B69184710B504462046F2
:10874000FFF7F8FF18B90A20FFF765FFF7E710BD3C
:108750000368DB68184700BF344B354A1B68126852
:1087600010B51A60334A116859605168926899606F
:10877000DA60314A116819615168926859619A61E9
:108780002E4A1168D9615168926819625A622C4A5E
:1087900011881985518859859188D2889985DA85FB
:1087A000284A118819865188598692889A86264ABD
:1087B0001188D986518892881987194621F83A2F4D
:1087C000224A10780022824206DA214C34F8124004
:1087D000013221F8024FF6E71E4A1288A3F86420FE
:1087E0001D4A1288A3F866201C4A1188A3F86C1051
:1087F00051889288A3F86E10A3F87020184A3B2184
:1088000012689A66174A126892FBF1F2B2F5967FE7
:10881000C8BF4FF0FF325A67134A1288A3F8782076
:10882000124A5289A3F85E2010BD00BF441D0020EB
:1088300070300020A82B0020B42B0020C02B00207B
:108840004C100020880F002036100020F72B00204D
:10885000A80F0020AC2A0020140F00208E0F00204B
:10886000401000201C000020C80F0020940F0020A2
:108870002DE9F84305460E460D4B002493E880038E
:10888000B44213DA7B1933F9140008EB050333F90A
:10889000142009EB050333F9143001341344022288
:1088A00093FBF2F3C01A08F029F9E9E7BDE8F88371
:1088B000441D002070B5472008F070F8174B1B6866
:1088C0001B0307D5164B174A5B6810681B68C01A54
:1088D00008F005F9144E154C154D307808F0FFF8E6
:1088E00023682868C01A08F009F963686868C01A24
:1088F00008F004F90F4B188808F0F1F80E4B1888AF
:1089000008F0EDF80D4B188808F0E9F83378237477
:108910002B68A3606B68E36070BD00BFC81E0020B9
:10892000441D0020703000204E180020301D002013
:10893000501800204C1800204A180020D00F0020AA
:108940007FB5264C264E274D2749284A284B20B173
:1089500028480088B0F5805F31D2308891F8201027
:108960001278ADF8040028781C4D1B788DF80600AD
:108970008DF807108DF8082001A8294606228DF8E9
:1089800009300CF0BDFA30B30198BDF8083028600A
:10899000AB80532008F002F8208808F0A0F8A078F7
:1089A00008F09DF8E37801A8019323790293637995
:1089B000039307F0FBFF0F4B00221A800BE0308877
:1089C00091F820102080127828781B78A070E17030
:1089D00022716371DDE704B070BD00BF681900202B
:1089E0000C19002048180020443000208B0D002076
:1089F000F00D0020E81E0020A0F17D03012B70B5D2
:108A000004460D460A4E05D830687D2106F03CFA32
:108A100084F020043068214606F036FA35B12B8800
:108A20001C4404EB142404F0FF042C8070BD00BF30
:108A3000FC1800200A4A138801331380094A13687E
:108A400001331360084A138801339BB2202B01BF06
:108A500000231380054A138808BF01331380704731
:108A6000E81E0020D01E0020D41E0020D61E0020AC
:108A700038B53A4B05461B780C46083B012B6BD8A2
:108A8000452007F08BFF284607F088FF0C2D23D0E8
:108A900004D80A2D0AD014D835B138BD0E2D4BD0CC
:108AA0002ED3FF2D50D038BD206849E0207807F044
:108AB00075FF62796378002A14BF80200020184374
:108AC00000E0207807F06AFFA07807F067FFE07801
:108AD00007F064FF20793BE0B4F9000007F0F5FFF0
:108AE000A07807F05BFFE07807F058FFB4F90400C6
:108AF00007F0EBFFB4F90600BDE8384007F0E5BF2A
:108B0000637820788BB180F0800007F047FFA4687D
:108B1000E0B207F043FFC4F3072007F03FFFC4F3C0
:108B2000074007F03BFF200E12E007F037FF6068B8
:108B3000BDE8384007F0E2BF206807F0D0FF60686A
:108B4000BDE8384007F0CBBF054807F005FF00201F
:108B5000BDE8384007F022BF38BD00BF211D00200E
:108B60003A9C01082DE9F04FBE4B8BB01A88019357
:108B7000BD4F002A40F0A98042F20103B7F8D607A2
:108B8000BA4EC21A50425041FFF7DAFEFFF7E4FD39
:108B900034684920254607F001FFB54B04F11C0954
:108BA000186807F09CFF55F8040B07F098FF28465B
:108BB00005F0ACF804F1100005F0A8F84FF010082B
:108BC000AC4D01232A6803FA08F3134203D0D9F805
:108BD000000007F093FF08F10108B8F1130F09F145
:108BE0000409EDD104F1280005F080F8B7F844310C
:108BF000B4F92E00C01A07F072FF2B68DB0408D509
:108C00009D4BB4F864001B88181AC0F30D0007F0E0
:108C100066FF2B68980403D5B4F8660007F05FFF81
:108C20002B68590503D504F16C0005F05FF82B683B
:108C30001A0502D5A06E07F061FF2B685B0402D510
:108C4000606F07F05BFF2B68180403D5B4F8780059
:108C500007F045FFA04604F1300005F047F804F1A5
:108C6000360005F043F8B7F8443138F93C0F0127D6
:108C7000C01A07F034FF814B1B789F4208DA38F99D
:108C8000020FB4F93C300137C01A07F037FFF2E7A2
:108C90002B68990505D5B4F95E00A0F2DC5007F009
:108CA0002DFF326876487260B260121A9110754AD0
:108CB0004A43531C032293FBF2F202EB42029A1A3C
:108CC0007C2303FB02033360D6E16F4B6F4A1B68C2
:108CD00011688B4206D00AA941F8203D002013609C
:108CE000FFF7C6FE019B97F8D6171B8897F8D707A2
:108CF0000B44013BB3FBF0F200FB12338B4280F0DC
:108D000086815A4F0120FFF71BFEFFF725FD5020FB
:108D10003E687D6807F042FEBA683B6810681B68D1
:108D20007A680344106806F11C0BA3EB400007F0BF
:108D3000E5FE6A68736802A89B1A0293AA68B36882
:108D400005F11C089B1A0393EA68F36810249B1A28
:108D5000049304F0DBFF2A69336902A89B1A02938B
:108D60006A6973699B1A0393B369AA699B1A04938E
:108D700007F01CFE3F4901220B68A2401A428A46B6
:108D800006D0DBF80000D8F80030C01A07F0B6FEB5
:108D90000134132C0BF1040B08F10408EAD106F19D
:108DA000260005F12601002331F9024F30F9022F88
:108DB000121B02AC44F823200133042BF4D103210D
:108DC0004FF000094FEA89035FFA83F902AB53F8C9
:108DD00021206AB102F108000F2802D849F00109E8
:108DE00006E08032FF2A94BF49F0020949F00309E6
:108DF00011F1FF31E6D24846002407F0CFFDA0462E
:108E00000DF1080B09F00302022A16D0032A1DD027
:108E1000012A4ED1B8F1000F05D1DBF80040904691
:108E20002401E4B245E0DBF800004FF0000800F058
:108E30000F00204307F0B2FD3BE0B8F1000F0CD06B
:108E4000DBF80000C0F3031020432CE0B8F1000F62
:108E50001ED19BF8010007F0A1FD9BF8000007F070
:108E60009DFD26E0D41E002054100020441D00204B
:108E7000D01E0020C81E0020C41E0020F72B00209A
:108E8000501D0020DF7BEFBDDC1E0020D81E00201F
:108E9000DBF80000C0F30330204307F07FFDDBF870
:108EA0000000C0F3071007F079FDDBF80040240153
:108EB000E4B20BF1040B06AB9B454FEA9909A1D133
:108EC000B8F1010F02D1204607F068FDDAF8003052
:108ED00013F480541FBFB6F86420B5F86410012461
:108EE000521A18BF02929A040AD50AAA02EB840108
:108EF000B5F86600B6F866200134121A41F8202C45
:108F0000580513D502AA02EB840C06F16A0E05F18E
:108F10006A0000223EF9021F30F9028FC8EB0101FE
:108F20004CF822100132032AF4D10334190508D574
:108F30000AAA02EB8400A96EB26E0134521A40F8FC
:108F4000202C5A0408D50AAA02EB8400696F726FBC
:108F50000134521A40F8202C18040BD50AAB03EB4D
:108F60008402B5F87810B6F8783001345B1A42F80C
:108F7000203C00E0FCB1012C03D1029807F0BEFDBB
:108F800019E0631E002002AA52F823204000C0B25C
:108F90000AB140F00100013BF5D507F0FFFC4FF0AE
:108FA000000802AB53F8280008B107F0A7FD08F14C
:108FB0000108A045F5DB30200321FFF759FC3620DE
:108FC0000321FFF755FC2F4B3C201978FFF750FC8D
:108FD000DAF80030990506D5B6F95E00B5F95E30CD
:108FE000C01A07F08BFD3A6827487B687A60121A2E
:108FF0009110264ABB604A43531C032293FBF2F2B2
:1090000002EB42029A1A7C2303FB02033B60204BD3
:109010001B681A0630D51F4C1F4D22682B689A42D8
:109020000BD162686B689A4207D1019B1B88102B99
:1090300011D11A4B1B885B060DD1482007F0AEFCFE
:10904000206807F05BFD606807F058FD23682B601F
:1090500063686B600EE0124A0F4B11782A7C9142D4
:1090600008D1104A99681068884203D15268DB68B9
:109070009A4201D0FFF71EFC07F060FC0BB0BDE880
:10908000F08F00BFF72B0020501D0020DF7BEFBDCD
:10909000742E0020D40F0020301D0020D61E00208A
:1090A0004E180020501800202DE9F84F0C9EC2EBFE
:1090B000030B394C0B9B002914BF4FF0060A4FF0ED
:1090C000040AF61A636805460133904613D12368F3
:1090D00053455ED2314A032B98BF294652F82320CC
:1090E0002F4807F049FC63680022013363602D4B71
:1090F00005469A7113E0002511E02B4A127895423B
:1091000040DA0B9BE3B109FB06F2995C01228A402D
:10911000264909680A4213D1636801336360D4F8B1
:1091200004900A9B1C4F9945E7DB2BD10A2007F0DE
:1091300035FC3B6801333B604FF0FF337B6021E03F
:10914000184A917921B12C2007F028FC013501E063
:109150000121917109FB0BF3226808EB030752B957
:1091600058F8030007F0F8FB97F9041005444B1C6E
:10917000D2D00F4802E03A440E48117907F0FCFBC8
:109180000544C9E7206850452CBF00200120BDE8F8
:10919000F88F0020BDE8F88FE01E002064800108F1
:1091A000459C01086819002048000020C81E0020C6
:1091B000549C0108CDA3010830B585B004AC00254E
:1091C00024F8025D0091ADF8060021461020FFF75B
:1091D00013FC9DF806002146FFF70EFC9DF80700E2
:1091E0002146FFF709FC9DF800002146FFF704FC2B
:1091F0009DF801002146FFF7FFFB9DF80200214684
:10920000FFF7FAFB9DF803002146FFF7F5FB9DF8F9
:109210000E002946C043C0B2FFF7EEFB05B030BDDB
:1092200010B5054C206805F02CFE18B1206805F03B
:1092300025FEF6E710BD00BFCC18002010B508F0E1
:10924000FBFA0021044608F007FD08B1204601E0C2
:1092500004F10040054908F0F7FB054908F040FB20
:10926000FEF76AF8034B186010BD00BF8096184BDC
:1092700035FA8E3C3C0000202DE9F04105460E46B3
:10928000078A83899BB21F40002F37D0B7FA87F235
:109290004FF00043D340DB4399B21F40A2F11B03C0
:1092A0002982042BF0D8DFE803F0221F1C190300E9
:1092B000746A24B1013C0023A4B2736201E0AC8D56
:1092C000A4B2D6F82080B8F1000FDDD0D8F8003075
:1092D000404621469847D8F80480F4E73068A98EC4
:1092E00008E07068298F05E0B068A98F02E0F06897
:1092F000B5F84010036889B29847C5E7BDE8F0812A
:1093000038B50D4B0D4D99680D4B1A681C465288A7
:10931000114203D0FFF758F9286007E0FFF754F92E
:109320002B68984282BFC01A064B186023685A689F
:10933000054B5A6138BD00BF000C01407019002078
:109340001C1D00201C00002000040140F8B59C4BAF
:1093500005461B68187818B1012800F06781DCE227
:10936000242D984C0CD006D80A2D00F0D8800D2D55
:1093700000F0D58044E12A2D06D02C2D04D03FE109
:1093800020716071A0714DE18F4B617927790020C8
:109390008C4A58542FBB1978D771472921D1597855
:1093A00050291ED19978472907D1D978472904D166
:1093B0001979412901D10121D1719978824A522923
:1093C00003D1D1784D2900F0AA8299787E4A4729A5
:1093D00007D1D178532904D11279562A04BF032228
:1093E000E271E279774E022A38D0032A4BD0012A63
:1093F00040F08380BA1E072A7FD8DFE802F0040815
:109400000F131A257E2A07F00FFDA06075E01B7868
:10941000532B72D1A3685B42A3606EE007F004FD9A
:10942000E0606AE01B78572B67D1E3685B42E3603A
:1094300063E01B78302B654B1A788CBF42F0020238
:1094400022F002021A7058E0002007F04DFD20744F
:1094500053E0002007F048FD60824EE0072F06D061
:10946000082F4AD1012007F03FFDF08245E001209E
:1094700007F03AFD41F2184358434FF47A73B0FBBA
:10948000F3F0B08239E0022F07D0032F0AD1002079
:1094900007F02AFD4E4B18702FE0002007F024FD46
:1094A00030762AE029D93A1F9210337E0132D2B2A7
:1094B000013B02EB8303DBB2102B1ED8F91EC2F175
:1094C000010201EB8202D2B2012A0BD0042A11D18F
:1094D00000205E1E07F008FD3E4B002298553E4BD3
:1094E0009A5507E03D4A5E1E0020935507F0FCFCAC
:1094F0003B4B9855E3690133E361324B2A2D18BF8A
:109500009A7907F101074FF000000CBF0122554086
:10951000277160710CBF83F820209D7182E094F860
:109520002000002847D02F4B13F8012D2E495A70E8
:109530008B42F9D1244A234D13785278402B85BFB2
:10954000373B1B011B01DBB298BF03F0F003402A3D
:109550008CBF373A303AD2B21344A279DBB29A4286
:1095600026D121230B70E8796B6A012803F10103EE
:109570001D4A6B620AD002281CD172231370AA8A7A
:109580001A4B1A80EA8A1A4B1A8013E06723137069
:109590000E4B1B789F070ED5164BAA681A60EA6817
:1095A0005A602A7C144B1A706A8A144B1A8002E0A3
:1095B0003F230B700020002384F8203032E000BFEE
:1095C0002C06002070190020A02E00204818002032
:1095D000E80F00201910002009100020E90F0020DA
:1095E000F90F0020B00200209C0200204A18002041
:1095F000D00F0020501800204E1800204C180020DA
:10960000637994F820000E2B9FBFA94A591C517111
:10961000A84A98BFD554A64A18B993795D40957168
:1096200000E00020003018BF0120F8BDA04B002250
:1096300093F82810082900F27081DFE801F0050C8A
:10964000101A2B3B5E788500B52D40F0668183F8BB
:10965000292001224EE0622D08BF02224AE00322A7
:1096600083F8282083F82A5083F82B5083F82C5055
:1096700053E1042283F8282093F82B2093F82C1030
:109680002A44D2B283F82B200A4483F82C2083F892
:109690002D5042E1052283F8282093F82B2093F8DF
:1096A0002C102A44D2B283F82B200A4483F82C20B1
:1096B000DD8532E1062283F8282093F82B2093F8E9
:1096C0002C102A44D2B283F82B200A4483F82C2091
:1096D000DA8D02EB0525ADB2B5F5AC7F82BF744AD9
:1096E000012182F829100022DD851A86002D40F024
:1096F0001481072283F828200FE193F82B2093F898
:109700002C102A44D2B283F82B200A4483F82C2050
:109710001A8EB2F5AC7F3EBF6549891881F8345086
:109720000132D98D92B291421A86E2D9F5E008222F
:1097300083F8282093F82B30AB4200F0EE805C4B8E
:10974000012283F829200FE05B4C83F8282014F8CD
:10975000012D6270594A9442F9D193F82C10544A61
:10976000A94206D03F232370554A53680133536002
:10977000D3E0516A92F829000131516210B13E23C1
:109780002370CAE02121217092F82D10062941D0C2
:1097900004D8022907D0032923D0F8BD122959D0B3
:1097A000302967D0F8BD502121704649946B4C6038
:1097B000D46B0C60516C4FF47A7491FBF4F1424C11
:1097C000218092F88C11414A19B1117841F00201BF
:1097D00002E0117821F002011170012283F88D213D
:1097E0008DE05321217092F83910CE0705D592F8FB
:1097F0003820D51E6A426A4100E0024602F00101AB
:1098000083F88C11002A7AD130490A7822F00202BA
:109810000A7074E04F21217092F83F10CC0705D5F3
:1098200092F83E20D11E4A424A4100E0024602F030
:10983000010183F88C1122B924490A7822F002022E
:109840000A7093F86310224A1170B3F86010214A2D
:10985000118054E056212170946C1F490C8042F213
:109860001074D16C91FBF4F11C4C2180012182F821
:109870008E1144E04921217092F83810184A1029BD
:1098800088BF10211170174914780022A24233D2E8
:109890000E7A154D56554E7A144D5655CE7A144DB6
:1098A000565511F80C6F134D56550132EEE700BFB7
:1098B00070190020A02E0020B00200209C02002081
:1098C0000C060020501800204C18002048180020DA
:1098D0004E180020460000204A180020D00F00201B
:1098E000E80F0020A4190020E90F0020F90F002044
:1098F0000910002019100020DA690132DA6193F8AA
:109900008D310B4A93B192F88E317BB1002182F8F0
:109910008D1182F88E111846F8BD0020F8BD12791D
:10992000432A7FF452AD0222E2714EE5F8BD00BF3A
:10993000701900200449054B0968002218705A610B
:1099400099611A77704700BF982E00200C060020FE
:10995000F8B5101A0D461F4607F06EFF0446781B37
:1099600007F06AFF174B079E196807F0B9FF2146F9
:109970000546204607F0B4FF29460746284607F06B
:10998000AFFF0146384607F0A3FE0BF045FF0E4936
:1099900007F0A6FF08F090F9069B2946186004F12D
:1099A00000400BF0ADFD094907F09AFF084907F0A8
:1099B0008FFE08F05BF90028BCBF00F50C40A0301A
:1099C0003060F8BD3C0000202C7D8E3FA00CB345DC
:1099D00000A00C4644F25063984203DDA0F50C4011
:1099E000A0387047034B9842BCBF00F50C40A03034
:1099F000704700BFB0B9FFFFF7B50368174C184DAB
:109A000023600B68174E63600068FFF717FC95E84A
:109A10000300154B0196009394E80C00FFF798FFA4
:109A20003668124B60681E606B68114FC01A07F0F1
:109A300003FF104B196807F053FF08F017F92A6865
:109A4000236878609B1A3B600B4B1E600B4B1B68B6
:109A5000DA880B4B1A8003B0F0BD00BFC02D002088
:109A600050180020CC2D0020C82D0020082E0020EA
:109A7000D02D00203C000020002E0020680E002089
:109A8000FC2D002070B50446407907F0D1FE1E4938
:109A900007F0DAFF1D4D1E4E2860E07B07F0C8FE80
:109AA000194907F0D1FFEE606860A07907F0C0FEA9
:109AB000184907F0C9FF184D2860207C07F0B8FE50
:109AC000114907F0C1FF6860A07E07F0B1FE13499D
:109AD00007F0BAFFEE60A860E07907F0A9FE0D4933
:109AE00007F0B2FF0E4D2860607C07F0A1FE06492A
:109AF00007F0AAFF6860E07E07F09AFE074907F0CA
:109B0000A3FFEE60A86070BD0000C842D82D002001
:109B10000000FA4400002041E82D002000007A44B3
:109B20000C2E002010B50C4C23789B0713D50B4B43
:109B30001B78042B0FD90A4A0A4B10685268186028
:109B40005A60FFF77BFB084B1A88084B1A80237872
:109B500043F00103237010BD481800204E18002068
:109B600050180020D40F0020441000201C2E00208C
:109B7000164B13B51B681B0325D5154B154C1B78CD
:109B800015498DF80030154B20681B788DF8013091
:109B900007F0A6FE08F090F811498DF80200606801
:109BA00007F09EFE08F088F88DF80300A06808F022
:109BB00083F80C4B8DF804001B780A2069468DF859
:109BC0000530FEF755FF02B010BD00BF742E002017
:109BD000642E0020882E002000002041842E0020CA
:109BE00000007A44682E0020054A137883F00103B0
:109BF0001370044A00231360034A1360B8E700BFE0
:109C0000682E0020802E00207C2E00200148024972
:109C1000FFF732BB00080040A02C00200148024999
:109C2000FFF72ABB00040040782C00204FF0804052
:109C30000149FFF721BB00BF502C00200148024919
:109C4000FFF71ABB002C0140282C002001480249D4
:109C5000FFF712BB002C0140282C0020254B10B52B
:109C60005A43254B254C1B680139B3FBF2F203889C
:109C7000013AA04289B292B29BB212D004F50064BC
:109C8000A0420ED0B0F1804F0BD0A4F59834A04282
:109C900007D004F58064A04203D004F58064A0429C
:109CA00002D123F070039BB2154CA04206D004F5FC
:109CB0008064A0421CBF23F440739BB203800F4B0F
:109CC0008185984202850FD003F5006398420BD03E
:109CD00003F54063984207D003F58063984203D0B0
:109CE00003F58063984201D1002303860123838218
:109CF00010BD00BF40420F0054000020002C014066
:109D00000010004073B505460068FFF7A7FF2A68FA
:109D10000124138800269BB243F001031380EB7AE1
:109D200001A88DF804308DF805408DF806608DF897
:109D3000074006F0E9FEEB7A1B2B0BD1192301A893
:109D40008DF804308DF805408DF806608DF80740D9
:109D500006F0DAFE02B070BD0C4B800A98420CD0BF
:109D600004D8B0F5801F0CD101207047084B9842F1
:109D700005D04933984206D003E002207047032003
:109D80007047FE2070470020704700BF01001000A0
:109D9000020010002DE9F843046807462046884673
:109DA0009146FFF7D9FF03284BD8BA7A9108B8F14A
:109DB000000F06D1A589AEB202258D4026EA050521
:109DC000A5810A2303FB00131F4A42F823800433B2
:109DD00042F82390B8F1000F07D0BD7AA189AD08F1
:109DE0000223AB400B439BB2A3812823434303F1DF
:109DF00020011144EFF31286502585F3128803F1F8
:109E00000C051C331544134455F8047F17B10F603B
:109E1000296804319D42F7D100230B60F3B283F32C
:109E20001188282303FB0020036A23B1A3899BB276
:109E300043F0010304E0A38923F001031B041B0C7E
:109E4000A381BDE8F88300BF282C0020FFF758BA93
:109E5000FFF756BAFFF754BA014801F057BE00BFEA
:109E6000001B0020014801F051BE00BF541B002020
:109E70000C4B4FF400525A604FF6FE730A48D0F86C
:109E8000182211680B401360D0F80822D0F80C3269
:109E90009A4203D000F5F27001F06ABE012380F807
:109EA0002832704700000240701900202DE9F04F61
:109EB000844B85B01A689B46511C1960032A00F236
:109EC0002683DFE812F0040085000C0317017E4AA8
:109ED0001268140740F11B837C4ADBF804101268F7
:109EE000784C511A0029C0F2128302F5C332A03215
:109EF00062607748E26890477548764A0146127872
:109F000004F0A4FA744A1078114610F0040F13D02C
:109F1000626822610022714C00251444A4F8765135
:109F20006B4C155B6E4C1553063415530232062AE2
:109F3000F1D120F0040008709BF8202082B1644A1F
:109F400066481188B0F87641091B1180B0F8784155
:109F50005188B0F87A01091B51809188091A9180C3
:109F6000DBF810005749002800F0D1824A6801F15F
:109F70001405121A5B4801F11A0482424FF00002E4
:109F800014D8534935F9127031F8121050000EB23E
:109F9000B742C4BF524F27F81210275E0132B742B2
:109FA000BCBF514E8153032AEBD1B0E24F480A6146
:109FB00035F9126034F9121001323144022691FB56
:109FC000F6F1032A20F8021FF2D1FDF777FD9EE299
:109FD0003D4A1268500740F19A823C4ADBF824104F
:109FE0001268384C521A002AC0F2918294F8282044
:109FF0000020012A60620FD002D3022A1DD059E04E
:10A00000626B9047A26B9047012284F82820E18D73
:10A01000626A0A4462624DE0E26B9047226B9047AD
:10A02000A18D626A04F144000A4462623049226CE4
:10A030009047022284F828203CE0276DE16C3F78AD
:10A040004D1CBD4204BF012584F8545084F82800FB
:10A0500008BF0546DBF85800626CA66C441C032C54
:10A0600002BF184C012784F85C700BEB800002667D
:10A070009BF85C0008BF0024124FCBF8584068B131
:10A080003C6E786EBA6E8442DEBF074620463C4680
:10A09000A242A8BF22468242B8BF02460BEB810112
:10A0A000CA660BEB8501C96ECBF84C50711A0A4495
:10A0B000CBF84820FEF788FADBF824201044CBF8D0
:10A0C000240024E2A81B0020441800207030002047
:10A0D0008E0F0020933000204818002054100020DC
:10A0E000BC1B00207FC3C901C21B0020C811002077
:10A0F00048100020B94A1268510702D59BF8541045
:10A1000011B9D20640F1038246F2A711B44ADBF836
:10A110002C711268B34DD71B8F4240F2F881B24CBC
:10A12000C5F82C21228862B32A6DD5F83011127837
:10A13000501EAA6CB2FBF0F2082091FBF0F6891BCE
:10A140000A44C5F8302192FBF0F007F075FBA749EF
:10A1500007F07AFCA6490BF0D5F901464FF07E5086
:10A1600007F0B4FAA34907F0BBFB07F07FFD228894
:10A17000C5F83401013A22800022C5F83821C5F81B
:10A180003C21DBF85050DBF848002A78DFF8809259
:10A19000013AB0FBF2F007F04BFB944907F054FC96
:10A1A00093490BF0AFF901464FF07E5007F08EFA5D
:10A1B000904907F095FB0BF0CBF86D688046D9F815
:10A1C000000007F039FB294607F08AFB0646DBF85A
:10A1D0003401C0EB080007F02FFB294680464FF002
:10A1E0007E5007F073FA0146404607F079FB0146BE
:10A1F000304607F06DFA0BF0ABF87F4A0546B2F92E
:10A200000060B2F90220002EB8BF7642002AB8BF23
:10A2100052429642B8BF1646784AC9F80000126802
:10A220003B2092FBF0F036B2B0F5967FC8BF4FF0FE
:10A23000FF30FA2EDFF8DC8104DD4FF0FF32C8F882
:10A24000002014E007F0F8FA8246304607F0F4FAEE
:10A2500001466B4807F03AFA0146504607F040FBCA
:10A26000674907F0F1FB07F001FDC8F80000D8F8D6
:10A27000006006F1FF38B8F1C60F05D8AD1BCBF86A
:10A280004051C9F800602CE0DBF84021002EA5EB1E
:10A29000020502DCC9F8005023E0C6F5967007F00D
:10A2A000CBFA584907F0D0FB8246304607F0C4FA93
:10A2B000514607F015FB0646284607F0BDFA514601
:10A2C00005464FF07E5007F001FA0146284607F098
:10A2D00007FB0146304607F0FBF907F0C7FCC9F859
:10A2E0000000494A106807F0A3FA4849064607F0FB
:10A2F000F7FADBF84451009075B13A4AD2F85001B0
:10A3000007F09AFA8146284607F096FA0146484631
:10A3100007F09AFB054600E00025DBF854112846BB
:10A3200007F0DEFA314607F0DBFADBF85831384A3D
:10A330004FF07C51D3F80CA001931668039007F0FE
:10A34000CFFA009907F0CCFADBF838910099029027
:10A35000484607F0C5FA029A0146104607F0B8F9D8
:10A36000DBF83C1107F0B4F9514607F0B9FA029056
:10A37000304607F061FA514600904FF07E5007F0EA
:10A38000A5F9009A0146104607F0AAFA029B014679
:10A39000184607F09DF9DDF80CC0CBF83C0161468A
:10A3A0008246484607F094F917490022CBF8482125
:10A3B000CBF84C21CBF85021CBF844210A602288FD
:10A3C0008146CBF83801002A40F0A180B8F1C60FD1
:10A3D000DFF8448022D8C8F8006024E04418002048
:10A3E00070300020A81B00208830002080E6C54780
:10A3F000B1DC423ED048874A6A2E00201C00002073
:10A40000000061440000C84274300020BD3786352A
:10A4100040100020C40F0020C00F0020504607F05D
:10A4200025FCC8F80000DBF85C01744C301A07F01A
:10A4300003FA734907F054FA8246384607F0F8F9F0
:10A440000146504607F000FB07F010FC40F2DC52DA
:10A450009042A8BF1046A2F6B8329042B8BF10464C
:10A460000A21CBF85C61FCF7E5FE019B82469E6801
:10A470004846314607F034FA0746504607F0DCF903
:10A48000314681464FF07E5007F020F9014648469C
:10A4900007F026FA0146384607F01AF9CBF83801DA
:10A4A0000AF056FF05210646FCF7C4FE40F23E6165
:10A4B000544ADBF8607110605348028802F21F3280
:10A4C00092B28A4205D8428802F21F3292B28A4280
:10A4D00025D90020CBF86C01CBF8605117E04B4A2E
:10A4E0001268D30613D54A4A44491068DBF8702134
:10A4F0003C3290420BD3D1F87451464C2A88C1F8B3
:10A50000700122610B20FEF77BF82A886261DBF87C
:10A510000030042B6FDD394B00221A606BE094F899
:10A52000782112BB3C4AD8F8000012680A21121A9E
:10A53000B2F5FA7F3948A8BF4FF4FA729042B8BF1B
:10A540001046FCF777FED4F864214FF0800E1279A4
:10A550003349504390FBFEF2B2F5967FA8BF4FF40B
:10A5600096728A42B8BF0A4601E02E4A1268DBF8AA
:10A570006401C6EB020E847A20260EFB04F494FBE1
:10A58000F6F6017DDBF86821B6F5967F0EFB012219
:10A59000A8BF4FF496762449B2F5C81FA8BF4FF460
:10A5A000C8128A42B8BF0A464FF40054CBF868215B
:10A5B00092FBF4F21A4C807FA642ACBF9419141996
:10A5C00007F03AF939460646284607F081F8014671
:10A5D000304607F085F94FF06C5107F081F907F02C
:10A5E00045FB9628A8BF96206FF095029042ACBF1D
:10A5F000201AA01A6EE705B0BDE8F08FA81B002056
:10A60000002474493C1000206A2E002044180020C9
:10A61000982E0020000C0140E40F00200CFEFFFFEC
:10A62000D4FEFFFF783000200000E7FF2DE9F04F57
:10A6300097498BB00B7813F0010F03F0040200F080
:10A640008181002A40F08B819248066816F080666E
:10A6500040F08581980700F1758143F004030B7089
:10A660008D4B8E4C1A888E4B1A8023681B0340F149
:10A670004A818C4B80201E7003F038FC08B105F035
:10A68000D7FB894F97F87951012D40F03C81874BDA
:10A6900093F8D61721B193F8D7270AB1914203D383
:10A6A000012283F8D62711E096460846BEF1000F36
:10A6B00006D090FBFEFC0EFB1C0C7046E646F5E750
:10A6C00091FBF0F192FBF0F283F8D61783F8D727CD
:10A6D00093F8D8271AB1754A002182F8D81741F6A5
:10A6E0006901D7F87C2193F8D89702EBC2028A421D
:10A6F00084BF40F2E241B2FBF1F26D498CBFD2B2AD
:10A7000004220A70B9F1000F21D18020FDF732FE3A
:10A710008046E0B18021FDF709FE98F80620654BE0
:10A72000022153F8223087F88001B3F5613F0CBF56
:10A730000222002298F900008DE8060080214A4696
:10A74000FDF7AFFFDFF86081C7F8840118B9002377
:10A7500087F87931D7E0494608F5C47014220AF029
:10A76000EAFB08F5D473C8F89C3108F509734F4922
:10A77000C8F8A03108F52873C8F8A4314E4B91F8F9
:10A78000940122681B880028A8F81C33C2F3C03348
:10A7900018BF012391F886010593C2F3402C02F4FF
:10A7A0000063C2F34008454A04901068C0F3800279
:10A7B000C0F3C0094879A0F119077C427C41012807
:10A7C00014BF20460120039091F8D60791F8D717BF
:10A7D00088422CBF002101210691394939488A4617
:10A7E0000078D1F800B002906F1EFFB2791E1329D5
:10A7F00045D8DFE801F00C0C0C0C0C0C0C0C0AAE6C
:10A80000B031333D3F12121241470399A4E002993F
:10A81000B942B4BF0024012430E09BF800100229A3
:10A8200013D1B91E5BF821000021CDF824C0089394
:10A83000079207F0E9F907AA4FF0010492E80C101B
:10A8400008B14FF00004E4B218E00BEB07014C79BB
:10A85000003418BF012411E041467DE023B1049982
:10A86000481E4142414100E0194601F0010173E0F8
:10A87000614671E005996FE006996DE014B1012120
:10A88000B9400E43142D1FD80135EDB2ACE700BF1F
:10A8900092300020680F002044100020742E002009
:10A8A000620E0020312A0020A81B00205410002036
:10A8B000480000208C840108AC2A002044180020A5
:10A8C000A40F0020F72B0020DAF80000254C793087
:10A8D0001921C4F82063FDF7D9FD0023C4F82833FB
:10A8E000A4F82C33A4F82E33C4F838331E4BD4F814
:10A8F00034231B6884F82403C4F83C330223C4F8CF
:10A90000302384F87931184B184A1B6892F8E221F9
:10A910004FF47A7101FB0233154A1360154B1B6823
:10A920001A0609D5144B1B789B0705D5134B1B78CA
:10A93000042B01D9062000E005200BB0BDE8F04F44
:10A94000FDF708BE5AB901200BB0BDE8F04FFDF786
:10A9500023BE494600E01146002990D194E70BB090
:10A96000BDE8F08FA81B0020982E00205410002076
:10A97000140E0020742E0020481800204E180020CD
:10A9800010B5164A1378590727D523F0040313701E
:10A99000134B1B681B031BD5124C94F87931A3F1A0
:10A9A0000802012A0BD8FF200021FEF761F80E4BA8
:10A9B0001B68C4F83C3305F0C1FF0A2306E0012BF5
:10A9C00006D90A2B04D005F09FFF012384F87931C2
:10A9D0000420BDE81040FDF7BDBD10BD9230002041
:10A9E000742E0020A81B0020982E002038B50024CB
:10A9F0000B4D6059254405F00BFB696811B10948FE
:10AA0000FCF7F9FBA96811B10748FCF7F4FB07480C
:10AA1000103405F0FDFAB4F5D87FE9D138BD00BF98
:10AA20007C800108789C01087E9C010873A40108C1
:10AA3000F0B585B004460AF0C2FA082826D1621E95
:10AA4000E01D1F4912F8013F09681944497801F0D7
:10AA50000301022908BF203B82421370F1D1254631
:10AA600004F1080715F8016B164831460AF099FA07
:10AA700020B1284631460AF094FA10B1FDF7D6F815
:10AA80001CE0BD42EED1204603F0B8F90E4805F0B7
:10AA9000BFFA00230D4A04A91A4492F88A210A44F5
:10AAA0000849595C0133082B02F80C1CF2D1002331
:10AAB000074801A98DF80C30FCF79DFB05B0F0BDEF
:10AAC000580000201EA30108849C01085410002097
:10AAD000B5A3010808B5184B184C1D682068FDF790
:10AAE0002CFE2846FDF729FE206841798B0703D408
:10AAF00041F00201FDF7D2FD206804F0C2F968B10F
:10AB00000E4B186804F0BAF90646FEF71FFC08B1B0
:10AB100004F014FD2846314604F0B6F9284604F046
:10AB2000B0F90028E8D02846266804F0A7F90146C5
:10AB3000304604F0A9F9DFE73C2E0020EC1E00208F
:10AB40002DE9F04705460AF03AFA2F4E0446D6F8AA
:10AB5000088090B92D4805F05BFA2D4B53F824106E
:10AB600049B10123A34013EA080F02D02948FCF79A
:10AB700042FB0134F1E7284822E0284627492246D3
:10AB80000AF026FA58B9264805F042FA254C54F83E
:10AB9000041F0029EFD01F48FCF72DFBF7E72B78A7
:10ABA0004FF000092D2B03BF013504F1FF344FF0A6
:10ABB000010A4FF0000A164B53F8297027B91A48BA
:10ABC000BDE8F04705F024BA2846394622460AF087
:10ABD000FFF9A8B9012000FA09F0BAF1000F03D07B
:10ABE000FCF79CFC114803E040EA0800B060104804
:10ABF00005F00EFA3946BDE8F0470E48FCF7FBBAFF
:10AC000009F10109D7E700BF541000208A9C010810
:10AC10002C820108949C010873A40108989C0108E7
:10AC20009D9C010828820108BF9B0108A99C01087E
:10AC3000B29C0108B4A3010810B5084805F0E8F972
:10AC4000074B00241C715C63064B1C7004F0BEFAB9
:10AC500005F0B6FB044B1C6010BD00BFBA9C010898
:10AC6000EC1E0020943000203C2E002070B50646DB
:10AC700000240B4BE518AA8816420AD0E15809486F
:10AC8000FCF7B9FA2846002105F053F9064805F00B
:10AC9000BFF940F6BC4314349C42EAD170BD00BFFA
:10ACA00064860108E69C010873A40108F0B50478E5
:10ACB0008BB005460CB1002436E04B4B19680E23CF
:10ACC00003FB0411B1F91D51B1F91921B1F91B317F
:10ACD000009591F8205101F58C70019591F8215162
:10ACE00001F59071029590F90700039091F9021017
:10ACF0003E48049121460134FCF77DFA082CDCD152
:10AD000070E02D2B14D1072C1BDC28460AF0ACF97F
:10AD10000AAB661C03EB440424F8100C15F8013F41
:10AD2000303B092BFAD934462B78002BE9D104E0CB
:10AD3000A3F13002092A09D8E5E7082CBDF818204C
:10AD400009D00BB0BDE8F040FCF770BF202BF8D164
:10AD500001352646E7E7072AF3D840F2DC55BDF86F
:10AD60001A00214BA0F2EE2189B2A9421B68E8D853
:10AD7000BDF81C10A1F2EE24A4B2AC42E1D8BDF89B
:10AD80001E6004B237B2A742DBDB0DB2AF42D8DCA3
:10AD9000A542D6DBBDF8247007F16404A4B2C82C28
:10ADA000CFD8BDF826E00FFA8EF4112CC9DCBDF81F
:10ADB0002050B42DC5D8BDF82240B42CC1D812B251
:10ADC0004FF00E0C0CFB0233A3F81901A3F81B1172
:10ADD000A3F81D6183F8205183F8214183F81F7186
:10ADE00083F822E10BB0F0BDA40F0020F09C010815
:10ADF000F0B504468FB020460AF0E1F8C5B21DBB9D
:10AE0000AB4805F005F9AB4C94F8D61009B9AA483F
:10AE100053E049B294F8D42094F8D530009194F8D6
:10AE2000D710A648019194F9D8100734029194F9EB
:10AE3000D210039194F8D310049129460135FCF700
:10AE4000DAF9102DE0D1E2E720469D4905220AF00B
:10AE5000BFF80546B8B929469A4870220AF06BF83F
:10AE60002846994B19680E2303FB0013013000227A
:10AE7000082883F8232183F8242183F8252183F8E7
:10AE80002621F0D112E12046904904220AF0A0F8D0
:10AE900005462046002D4AD120210AF082F80028DC
:10AEA00000F00481461C30460AF089F82C4607461B
:10AEB000874B53F824502DB986480FB0BDE8F040B9
:10AEC000FCF799B930462946FAB20AF081F8013404
:10AED0000028EDD1774A164602F17001002382F86E
:10AEE000DA3082F8D63082F8D53082F8D4300732A2
:10AEF0008A42F3D1784901EBC40191F808229342C8
:10AF000010DAD1F80C72C3EBC302B0183A441768D8
:10AF100000F1D401C0F8D470908801338880927910
:10AF20008A71E7E729466D48FCF765F98FE06C49BF
:10AF300007220AF04DF805462046002D49D1202170
:10AF40000AF02FF806460AF03AF8C4B26CBB65481E
:10AF5000FCF751F9214664480134FCF74CF90E2CFA
:10AF6000F8D15548FCF747F9002460482146FCF722
:10AF700042F90025544A012311680E2202FB0412F3
:10AF8000D2F82321AB401342594B5A495A4808BFC3
:10AF900019460135FCF72FF90E2DEBD14648013447
:10AFA000FCF729F9082CE0D180E0304653490AF03B
:10AFB0005FF82C4600284CD0022C4FD00AF054F8F1
:10AFC00006AB43F824004D4900200AF051F8013443
:10AFD000F0E74A490AF04CF8002460B1082C38D058
:10AFE0000AF042F806AB43F82400444900200AF076
:10AFF0003FF80134F1E7082C2BD1069B0F2B28D802
:10B00000DDF81CE0BEF1070F23D8089F0D2F20D8D4
:10B01000099E06F16402C82A1BD80A9DFF2D18D884
:10B020000B98642815D80C99642912D8884210DA34
:10B030000D9C032C0DD8324AC3EBC303134483F891
:10B0400004E05F719E71DD71187259729C722D4C13
:10B05000D1E60FB0BDE8F040FCF7E8BD069B072B3A
:10B0600020D807990D291DD80278722A0DD06E2A92
:10B0700018D1154A0E20126800FB032301228A40D2
:10B08000D3F8231121EA020209E00F4A0E201268C8
:10B0900000FB032301228A40D3F823110A43C3F89B
:10B0A000232101E0FCF7C2FD0D4CA4E60FB0F0BD7A
:10B0B000189D01085410002073A40108439D010845
:10B0C0008F9B010828110020A40F0020BA9B0108C3
:10B0D00020930108BF9B01087C800108CE9B0108DA
:10B0E000109D0108829C01085F9D0108CDA3010805
:10B0F0008EA80108D4A70108649D0108689D010875
:10B1000024110020FB9801082DE9F7430478054637
:10B110008CB9324D95F8AB12B5F8A82295F8AA3241
:10B120002F48009121460134FCF765F8102C05F1F9
:10B130000405EFD14EE009F097FF0F28044636DCF6
:10B140002846202109F02DFF264EE4B2D6F838809B
:10B15000451CA4000027284609F086FF5FFA87F9FE
:10B16000B9F1010F83B208D0B9F1020F0BD0B3F5DA
:10B17000B47F24D2B26B13530AE0FF2B1FD8B36BFA
:10B180002344987004E0FF2B19D8B36B2344D87084
:10B1900028462C2109F005FF054608B1013502E0DB
:10B1A000B9F1020F0BD10137032FD4D112E00E48B1
:10B1B00000210F2203B0BDE8F043FCF7B4BC08EB5C
:10B1C00004000021042209F0B6FE03B0BDE8F043FC
:10B1D000FCF72CBD03B0BDE8F08300BF5410002085
:10B1E0006A9D0108EC1E0020689B01082DE9F043D0
:10B1F00004788FB00546002C59D17C4B00211422D5
:10B2000009A807AED3F83C8009F095FE0722304626
:10B21000002109F090FE00231A46A70005A8059317
:10B2200008EB070583807249B5F802E031F813C0D6
:10B230001CEA0E0F0AD00E310DF1380C595C02F1E8
:10B24000010E624402F81C1C5FFA8EF20133072BD8
:10B25000E9D100210B46674AB5F802E011F802C0B7
:10B260001CEA0E0F0AD006320DF1380C8A5C03F18D
:10B27000010E634403F8242C5FFA8EF30131062992
:10B28000E9D118F807308DE841006A785A490292EE
:10B2900009A81A0903F00F0305F04CFE2146574890
:10B2A00009AA0134FBF7A7FF202CA6D19BE009F0E7
:10B2B000DBFE1F28044600F3898028462021E4B2E3
:10B2C00009F06FFE1F2C02D9FCF7B0FC8BE0474B56
:10B2D000451CDB6B002103EB84042046042209F0AB
:10B2E0002AFE0027464B09AE304600210A2217F8F5
:10B2F00003905FFA87F809F01EFE002315F8012B72
:10B3000032B10A2B04D04A4502D0F2540133F5E79A
:10B310004A4561D108F1FF33032B09D8DFE803F078
:10B32000100502420DF1230037E00DF123011FE06B
:10B33000304609F099FE2378C0B243EA001006E0D7
:10B34000304609F091FE237800F00F00184320707A
:10B3500034E00133062B0BD02A4800F2F3269E5D21
:10B360009642F6D1034493F8ED2263881343638039
:10B3700011F8012F12B30023EEE70133072B0CD095
:10B38000204A02F2E6269E5D8E42F6D102EB43038E
:10B39000B3F8D82263881343638010F8011F69B1A2
:10B3A0000023EDE7304609F05FFE0F2804DC30464D
:10B3B00009F05AFE607001E0002363700137052F29
:10B3C00090D1012404F060F86CB97DE70E480021AB
:10B3D0001F22FCF7A8FB06E020460021042209F00A
:10B3E000AAFD0024EEE70FB0BDE8F083EC1E0020BC
:10B3F00054830108698301087E9D01088D9D010821
:10B40000758301087C800108689B01082DE9F04FD5
:10B41000AB498BB0044609F097FDAA4900282046A5
:10B420000CBF0125072509F08FFDA74900282046FC
:10B4300008BF022509F088FD002808BF0425E90798
:10B4400040F1E680A14804F0E3FD002004F0F0FBA9
:10B450009F4CA04804F0DCFD9F4804F0D9FD6379BF
:10B460009E4A013B52F823109D48FBF7C4FE9D48BD
:10B47000FBF7C1FE26460027D6F81480002140467F
:10B4800006F0C2FB20B19848FBF7B5FE002669E044
:10B4900039469648D6F818B0D6F81CA0D6F82090B1
:10B4A000FBF7A9FE4046002106F0B8FB10B12020B2
:10B4B00004F0A6FD06A94046FBF738FD01468C487E
:10B4C000FBF799FE5846002106F0A8FB10B120209A
:10B4D00004F096FD06A95846FBF728FD014684486E
:10B4E000FBF789FE5046002106F098FB10B12020A2
:10B4F00004F086FD06A95046FBF718FD01467C487E
:10B50000FBF779FE4846002106F088FB10B12020A9
:10B5100004F076FD06A94846FBF708FD0137014611
:10B520007448FBF768FE0C2F06F11006A4D1AAE7B9
:10B5300049B294F8D42094F8D530009194F8D710FB
:10B540006D48019194F9D8100734029194F9D21002
:10B55000039194F8D310049131460136FBF74BFE6A
:10B56000102E03D094F8D6100029E1D1634804F0DE
:10B570004FFD574B624C9F6854F8041F19B1614846
:10B58000FBF739FEF8E70E465F4B53F826404CB107
:10B590000123B3403B4203D05C482146FBF72BFE1E
:10B5A0000136F1E75A4804F033FD2146484B0AAA18
:10B5B0000B4493F88A311344564A8A5C01310829B6
:10B5C00003F8102CF2D1002306A953488DF820303F
:10B5D000FBF711FE514804F01BFD5148FCF704FE37
:10B5E000504804F015FD4E48FFF700FE4E4804F0A9
:10B5F0000FFD4B48FFF788FD4C48FBF7FCFD402052
:10B60000FFF734FB4A4804F003FD4548FCF72CFDE6
:10B61000AA0739D5474804F0FBFC474804F0F8FC7A
:10B620003F4804F045FB454804F0F2FC3C48FCF779
:10B6300087FA434804F0ECFC3948FCF767FC4148C2
:10B64000FBF7D9FD3648FCF7F7FA3F4804F0E0FC79
:10B650003348FFF72BFB00260E27774300243B4A95
:10B660000123126CA3403A44D2F80A2013421ED19F
:10B6700001340E2CF3D10136082EEDD12B48FBF707
:10B68000BAFD8020FFF7F2FA6B0716D5304804F0B8
:10B69000BFFC304804F0BCFC214804F0E3FA234826
:10B6A000FBF7A9FD4FF48070FFF7E0FA05E03146A3
:10B6B00022462948FBF79FFDDAE70BB0BDE8F08F83
:10B6C000999D0108A9A10108A09D0108A69D010856
:10B6D00054100020B49D0108C69D01082093010864
:10B6E000D29D0108DD9D0108EA9D0108F79D010832
:10B6F000819C0108B5A301080F9E0108FF9D010868
:10B70000288201082E9E01082C8201083C9E010817
:10B71000499E01081EA30108559E01085E9E01086E
:10B72000FB9801086D9E0108799E010873A4010829
:10B73000879E0108949E0108A79E0108B59E0108F6
:10B74000BF9E0108CE9E0108DC9E0108EC1E002071
:10B75000E89E0108F99E01080B9F0108026B034651
:10B76000C16810B5406942B11A6C8C1A013A08BF21
:10B770000A46005D1A64C0B210BD1A6A805C0132CC
:10B780008A4228BF0022C0B21A6210BD436B13B1B7
:10B7900090F844007047836A406A1B1A5842584127
:10B7A0007047036B13B15B68016C01E0C369016A08
:10B7B0008B423CBFC2689B18581AC0B27047426A9D
:10B7C000806A131A58425841704741717047437953
:10B7D0009B070AD5436A8269D154436A01690133E0
:10B7E000B3FBF1F201FB123343627047437913F06C
:10B7F00001031FBFC36803F1FF32C369006A1DBFA5
:10B80000181A1040C0B218467047437910B513F0AB
:10B81000010304460DD0FFF7E9FF58B1236A6269BE
:10B82000E168D05C0133B3FBF1F201FB1233236218
:10B8300010BD184610BDF0B5046D8279A389467914
:10B8400023F4005312F0020F4FEA03434FEA13436D
:10B850000CBF00214FF4005112F0040FA38114BF5C
:10B860004FF4806E4FF0000E16F0010F876805460A
:10B8700014BF04200020B307238A48BF40F0080209
:10B880009BB223F4405343EA01032382A18948BFBA
:10B8900090B289B221F4B05121F00C014EEA0101BD
:10B8A00040EA0102A281A38A87B023F440731B04FB
:10B8B0001B0CA38201A802F0E1FB049E039B204A1B
:10B8C000944218BF1E46A389192272431BB2002B53
:10B8D000B4BF7E00BE00B2FBF6F66427B6FBF7F0FD
:10B8E0000001010907FB1163A28912B2002AADBF52
:10B8F0001A01D90032313232ABBFB2FBF7F3B1FBE0
:10B90000F7F203F00F0302F00702B4BF104318432D
:10B910002A6DAB7980B2208113F0080F938A0BBF98
:10B9200023F008039BB21B0443F0080308BF1B0C61
:10B93000938293899BB243F40053938107B0F0BD87
:10B9400000380140417176E7816074E703460A469A
:10B9500090F84602D96A9B7901F010BF38B5A0F57E
:10B9600013746379A579DB0746D594F8383205F06E
:10B970000105F3B1226B1068838DC3F34E038384FA
:10B9800094F83C3223B1B4F842320133A4F8423285
:10B99000917A6A0001F051FD012384F83B320023C3
:10B9A00084F8393284F83A3284F83832A4F84032D4
:10B9B00038BD94F83B322046012B04BF94F839324D
:10B9C00084F83A3201F024FD94F83B22236B3AB913
:10B9D000012284F83B221868997A05FA02F207E0FE
:10B9E000002284F83B2295421868997A08BF022207
:10B9F000BDE8384001F021BD38BD10B5A0F5127486
:10BA000094F83C22BAB9A36A616A994228D0591CB9
:10BA1000A069A162C35C2069DBB25B0043F40073E0
:10BA20008142A4F83E324FF00A0384F83D3228BF29
:10BA3000A262012312E094F93D327BB1B4F83E12C8
:10BA400020464B08A4F83E3201F0010101F008FD48
:10BA500094F83D32013B84F83D3201E084F83C32F9
:10BA600094F83832002B50D194F839320133DBB2DC
:10BA7000092B84F8393204D12046BDE8104001F08A
:10BA8000C7BC0A2B41D194F83B322BB9B4F84032F1
:10BA900043F00103A4F840326379D9071CD5B4F808
:10BAA0004002820501D4C30705D4B4F844320133FF
:10BAB000A4F8443210E0E36AC0F347000BB19847A2
:10BAC0000AE0E3696269D054E369E1680133B3FBDA
:10BAD000F1F201FB1233E361012284F8382294F879
:10BAE0003B220023012A84F839320ED1A27984F84E
:10BAF0003B32236B12F0010F1868997A0CBF0222B7
:10BB00000022BDE8104001F098BC10BD026D70B578
:10BB100015880446ADB2A90613D5036B8BB9C36A69
:10BB20001BB1908880B298470BE0E1699288406928
:10BB30004E1CD2B2E6614254E169E268914228BFEC
:10BB4000E3612B0613D5636AA26A9A42236D0AD079
:10BB5000511CA069A162825C9A802369994206D334
:10BB60000023A36270BDDA6822F08002DA6070BD43
:10BB7000836A8169426B1944D160416A994297BFD7
:10BB80000169CB1ACB1A536096BF002353608362BE
:10BB90004FF0000380F84430136888BF816243F09F
:10BBA000010313607047436A8269D154436A026992
:10BBB0000133934228BF00234362436B1BB11B68D0
:10BBC000DB0705D4D4E7026DD36843F08003D3606C
:10BBD00070472DE9F0431E46944B8DB0984289463C
:10BBE00090469DF8507051D1914B924A92491A60FB
:10BBF000924AC3F808805A6102F580729A614FF444
:10BC00008072DA601A618E4A18651A63A2F548429A
:10BC1000543ADA649A6459638A4B9A6942F48042CE
:10BC20009A615A6942F001025A6102238DF8033089
:10BC30003A074FF40073ADF8003001D51C230FE034
:10BC4000B30706D51823804869468DF8023001F005
:10BC500063FDF5070AD54FF48063ADF80030482343
:10BC6000794869468DF8023001F056FD0E238DF8B3
:10BC700004300022012301A88DF805308DF806203C
:10BC80008DF807306A4C04F03FFF4EE06F4B98424E
:10BC900040F0C7806E4B674AC3F808801A604FF4C3
:10BCA0008072DA601A616B4A18655A6102F5807217
:10BCB0009A61694A3C079A64DA64624BDA6942F431
:10BCC0000032DA615A6942F001025A614FF0020310
:10BCD0008DF803304FF00403ADF8003001D51C237C
:10BCE0000EE0B00706D51823574869468DF8023094
:10BCF00001F012FDF10709D50823ADF80030482303
:10BD0000514869468DF8023001F006FD26238DF872
:10BD100004300022012301A88DF805308DF806209B
:10BD20008DF8073004F0F0FE494C0025012384F81B
:10BD300044302562E561A5626562C4F82C906671A5
:10BD4000C4F80880A7712046FFF775FDF20731D5CA
:10BD5000206B002826D0E36C039501934FF48053A9
:10BD60000A9380230693E36805950493202309939F
:10BD700063690795029308950B9502F007F901A9ED
:10BD8000206B02F0E5F8226B216D136843F001038C
:10BD900013608B8A9BB243F040038B8253689BB243
:10BDA000236407E04FF6DF72236D1A80DA6842F0F1
:10BDB0002002DA60B3072CD5606B28B3A36C002592
:10BDC00001934FF480530A938023069323690295CD
:10BDD00004931023039305950795089509950B95F2
:10BDE00002F0D4F8606B01A902F0B2F8636B1A6834
:10BDF00042F002021A60226D5D605D60938A9BB220
:10BE000043F08003938204E0226DD36843F0800303
:10BE1000D360226D204693899BB243F400539381F3
:10BE200000E000200DB0BDE8F08300BF0038014005
:10BE3000541B00203884010844000240301F0020B9
:10BE40005800024000100240000801400044004039
:10BE5000001B002030210020044400402DE9F74F52
:10BE6000FCF7B2FBA64C804626686568A768861B6F
:10BE7000F643451BC71BED43FF43F60FED0FFF0FC6
:10BE80002EB93FB9002D00F08782B9462CE04FF063
:10BE9000000929E0B14627E003EB8A0BBBF802302A
:10BEA0001A050ED413F4805F1DBF964A9BF801104B
:10BEB0001268954A954B14BF52F82120126843F836
:10BEC0002A20BBF80230D80516D499050AD5904B24
:10BED0001B7813F0040F0CBF8E4A8F4A8B4B1268ED
:10BEE00043F82A2009F10109207B5FFA89FA8B497E
:10BEF00082450B68D0D326E0894A5046594603F064
:10BF000053FA884B1B885A0603D550465946864A31
:10BF100016E0580703D550465946844A10E01907E1
:10BF200003D550465946824A0AE09A0703D550463F
:10BF30005946804A04E0DB07D4D5504659467E4A2C
:10BF400003F032FACEE7DFF808E20093BEF90630DC
:10BF50007822A3F57A7353434FF47A7293FBF2F38A
:10BF6000F34603F22B13019300225FFA82FE86450B
:10BF700017D2009B03EB820EBEF802E01EF4806F26
:10BF80000DD040F2671ADFF88491019B39F822E066
:10BF90009E449EFBFAFC0AFB1CEE29F822E00132CB
:10BFA000E3E74DB308F5C333A0336360637B544AC2
:10BFB00013BB9373614B1B6813F0020F0AD0DFF8B9
:10BFC00094E19EF800E0BEF1000F03D04FF0010EA7
:10BFD00082F80EE0DA0506D5594BDB781BB1A37B5E
:10BFE00043F00203A3734A4B1B7813F0050F02BF03
:10BFF000A37B43F00403A37394F80EE0BEF1000F9B
:10C0000003D13F4B5B7B002B4FD094F80DC01CF04D
:10C01000010FACF10C031DD1BCF1030F07D8DFF801
:10C02000E8901EF0040F3B4A08BF4A4600E0364A3B
:10C03000ACF1040CBCF1070F05D8DFF81CC11EF0F1
:10C04000010F18BF6246DBB2032B0ED81EF0020FA1
:10C050003C4B06E0DBB2032B06D82F4B2A4A1EF0DE
:10C06000020F18BF1A4600E0274A4FF0000C5FFA93
:10C070008CF383420DD20B6803EB8C035B881B06A9
:10C0800042BFD2F80090214B43F82C900CF1010CE8
:10C09000EDE785B1BEF1000F08D0637B184A01338C
:10C0A000DBB2142B06D1002304E025B1637B002B07
:10C0B000F3D100E05373002E52D0234A3223B2F959
:10C0C0000250B2F90020002DB8BF6D42002AB8BF5F
:10C0D000524295FBF3F592FBF3F2EDB2D3B2AB42D1
:10C0E00038BF2B46194A13B192FBF3F300E0134615
:10C0F00043442360E37B024A83BB01232FE000BF5C
:10C1000030230020241F0020A0950108DA0C002015
:10C1100092300020A894010898940108281F00205C
:10C12000508401080C190020568401085C84010821
:10C1300062840108688401086E840108742E00205E
:10C1400044300020B09401084C100020400D030042
:10C150006C2F002094180020B89401080023D3739A
:10C160008F4D904B2D78E27BADB9002F00F00F8101
:10C170008D4B267B1A788D4B02F0040293F800C099
:10C180008B4BD2B2D3F800E00B680021894D03EB52
:10C1900086060F46B5E01AB9874A1A61002508E0FD
:10C1A000864AFAE70A68AB00D6187688760604D481
:10C1B0000135EBB28342F5D3D7E7814EB6F9006083
:10C1C000192E25DD12F803E094F814C00EF00F09C3
:10C1D000E14526690CDCDFF8CCC19CF815C0BCEB4E
:10C1E0001E1FDEBFD6F800C0DFF8D8E143F80EC04E
:10C1F00012F803E094F816C00EF00F09E14533DBA6
:10C20000DFF8A0C19CF815C0BCEB1E1F2CDC26E09B
:10C21000193629DA12F803E094F814C00EF00F0969
:10C22000E14526690CDCDFF87CC19CF817C0BCEB4B
:10C230001E1FA2BFD6F800C0DFF888E143F80EC089
:10C2400012F803E094F816C00EF00F09E1450BDB7D
:10C25000DFF850C19CF817C0BCEB1E1F04DBD6F8FA
:10C2600000E0584E43F806E0554EB6F90260192E2C
:10C270001BDD12F803C094F814E00CF00F09F1452F
:10C2800026690CDCDFF81C9199F81590B9EB1C1F9E
:10C29000DEBFD6F80090DFF82CC143F80C90D25CDA
:10C2A00002F00F0CF4451EDD82E7193680DA12F831
:10C2B00003C094F816E00CF00F09F14526690CDB79
:10C2C000DFF8E09099F81590B9EB1C1FDEBFD6F8A7
:10C2D0000090DFF8F0C043F80C90D25C02F00F0C35
:10C2E000F445FFF665AF94F817E0BEEB121FA2BF4E
:10C2F0003668344A9E505BE75888000504D40433FE
:10C300000435B342F8D122E04AB101EB0C0A062011
:10C310009AFBF0F900FB19A001280DDC01E057B9E8
:10C32000012793F801900EEB89003EF829A090F8C0
:10C330000290C07803E01746002081468246013112
:10C3400025F802AC85F800906870C9B2D7E7174AA3
:10C350001378013B13F0FF0308BF06231370124B41
:10C360001B785B0741BFBBF906304FF47A72A3F527
:10C370007A7303EBC30348BF93FBF2F3124A46BF41
:10C380000133DBB2012392FBF3F34344A36003B018
:10C39000BDE8F04F01F0E2B803B0BDE8F08F00BF98
:10C3A0008B0D002030230020923000202000002040
:10C3B000241F0020DC0C0020B4940108A095010883
:10C3C0004C100020DA0C0020400D0300064B1B78B7
:10C3D00003F0040303F0FF001BB1044B1888C0F303
:10C3E000C01000F001007047923000200C190020AE
:10C3F0002DE9F04F89B00593BE4B0026B3F90290AA
:10C40000B3F90030B9F1000FB8BFC9F10009002B32
:10C41000B8BF5B429945B8BF99468046B24634469C
:10C42000B9F5FA7F04910392A8BF4FF4FA7901900D
:10C4300000960296B04D2B88990754D0AD4B610001
:10C4400033F91420AD4B33F9143003EB4202039B54
:10C450005B429A4203DB039B9342A8BF1346A84A60
:10C460008F5E059ADB1B32F914001F18FFF7AEFF31
:10C4700090B1A44B384613F804A005F0DDF9A249A9
:10C4800005F0E2FA0146504604F05CFB9E4905F0D7
:10C4900027FA05F0EBFB074698F8083064227B4347
:10C4A00093FBF2F398F81C206FF0040A0AFB02FADF
:10C4B000534504DB02EB820A9A45A8BF9A4642F232
:10C4C0001072924B53F8240038449042A8BF104693
:10C4D0008F4A9042B8BF104643F8240098F81230B3
:10C4E0005843031302932D8805F00303012B38D022
:10C4F000804B884933F91430A6000093019B51F812
:10C50000247093F801E0844B33F9140080EAE0735F
:10C51000A3EBE073B3F5206F16DC009A50235A4367
:10C5200092FBFEF3042290FBF2F0181A0744B7F5D1
:10C530007A5F7A4BA8BF4FF47A579F42ACBF41F85D
:10C54000247041F8243002E0002341F824308B5954
:10C550007D2693FBF6F6019BDB7A7343402693FB23
:10C56000F6F6AA0712D5009A09FB06F509FB02F7B1
:10C570000298C9F5FA7303FB0A7703FB00534FF4E3
:10C58000FA7297FBF2F193FBF2F505E0EB0755BF6A
:10C59000354651460099029D5F4B042733F914300C
:10C5A0005F4A93FBF7F3A25C6FF04F07534393FB93
:10C5B000F7F398F851204FEA440BCF1872B1384680
:10C5C000069205F039F95749574B01EBC401069A19
:10C5D0001B68FAF7E5FB05F049FB07464E4B534A4B
:10C5E0003BF803003BF9021003B25B1A042193FBF2
:10C5F000F1F102F1040E5EF824302BF802000C3247
:10C6000052F8240042F8243098F8502018444FEA99
:10C61000840C08444EF8241082B1CDF81CC0069258
:10C6200005F00AF94249404B01EBC401069A1B6828
:10C63000FAF7B6FB05F01AFBDDF81CC03D4BDFF83E
:10C6400010E11B5D7A195843202390FBF3F3D21AB3
:10C650002BF80E20384A5B424CF80230019B3748D9
:10C66000374901334CF801504CF80070019375467E
:10C670000CB90124DEE61F4B0427B3F90440049BE8
:10C68000244E9B79D6F808E00F335B006343224CBD
:10C690005B11B4F90440002B94FBF7F7A3EB0707F9
:10C6A000B8BF5B42322B98F80D400BDC04FB07E46B
:10C6B000244BA342A8BF2346234CA342ACBFB36084
:10C6C000B46001E00023B36098F8034004FB07F373
:10C6D0001E4C9B112478032C3DD9B8F84E40B4F57C
:10C6E000FA7F38D26742BB4234DBA342A8BF23465D
:10C6F00031E000BF4C1000200C1900208C300020CD
:10C700006A2E0020C0840108000020414823002038
:10C71000F0D8FFFF582B0020880F002080C1FFFFBA
:10C72000E02B00203C2B0020542B00205023002025
:10C73000882B0020F42B0020C02B0020A82B0020E9
:10C74000B42B0020FEFFFF0F020000F0F72B0020AB
:10C75000A02B00203B46B4686FF0FF0644F34F3433
:10C76000B4F5807FA8BF4FF48074B442B8BF34469C
:10C7700083601E190023AE808C60936009B0BDE811
:10C78000F08F2DE9F04F87B00393B44B81461D889D
:10C79000029105F00205ADB2019295B1B04BB3F92B
:10C7A0000250B3F90030002DB8BF6D42002BB8BF66
:10C7B0005B429D42B8BF1D46B5F5007FA8BF4FF450
:10C7C0000075CB460026A64BA64933F91620A64B8A
:10C7D0004FEA460A33F91630520083EAE374A4EBB9
:10C7E000E374B4F5206F4FEA860851F8260011DC97
:10C7F000042493FBF4F3D31A0344B3F57A5F9B4804
:10C80000A8BF4FF47A538342ACBF41F8263041F8B9
:10C81000260002E0002341F8263051F808709BF80A
:10C820000B30FF119BF801405F438C4B54431B8836
:10C83000BF119B074FEAA41456D08D4B3AF9033031
:10C840001A44019B5B429A4203DB019B9342A8BFBF
:10C850001346884A3AF902209B1A039A32F91620A5
:10C860001A440492FFF7B2FD049A98B1824B104625
:10C870009B5D049304F0E0FF804905F0E5F8049B1C
:10C880000146184604F05EF97C4905F029F805F0E8
:10C89000EDF9024642F21070794958F8013013441C
:10C8A0008342A8BF034677488342B8BF034648F88F
:10C8B000013099F8081099F81C004A4300EB8000F9
:10C8C000D21141428A4203DB8242A8BF024611468E
:10C8D00099F81220641A53431B13FF1A6F436C43D9
:10C8E00003EB672701EB64245F4B04223AF9033022
:10C8F00093FBF2F2644B9B5D534399F85120A4EBF8
:10C90000A31472B12046049204F096FF5F49604B75
:10C9100001EBC601049A1B68FAF742FA05F0A6F982
:10C92000044651495B4B3AF801003AF903E002B280
:10C93000CEEB02024FF0040E92FBFEF22AF8030047
:10C940009E440C3358F80EC058F8030048F80E20E7
:10C950006044104499F8502048F803C08C467AB1DE
:10C960000591049204F068FF4B49494B01EBC60165
:10C97000049A1B68FAF714FA05F078F9DDF814C088
:10C98000464BDFF834E19B5DE21943435B11D21A59
:10C990002AF80E2042484349434A5B4248F8004087
:10C9A00048F8017048F802300BF1010B74460EB9DB
:10C9B000012608E72A4B0427B3F90450029B294EAD
:10C9C0009B79D6F808E00F335B006B43BCF9045049
:10C9D0005B1195FBF7F7002BA3EB0707B8BF5B4292
:10C9E000322B99F80D500BDC05FB07E52F4BAB42C2
:10C9F000A8BF2B462E4DAB42ACBFB360B56001E083
:10CA00000023B36099F8035005FB07F3294D9B11F0
:10CA10002D78032D0CD9B9F84E50B5F5FA7F07D211
:10CA20006F42BB4203DBAB42A8BF2B4600E03B4654
:10CA3000B5686FF0FF0645F34F35B5F5807FA8BFA9
:10CA40004FF48075B542B8BF354683605E19002348
:10CA5000A6808D60936007B0BDE8F08F0C190020B0
:10CA60004C100020582B0020880F002080C1FFFFB1
:10CA70008C3000206A2E0020C08401080000204174
:10CA800048230020F0D8FFFFE02B00203C2B0020A3
:10CA9000542B002064230020882B0020F42B00203E
:10CAA000A82B0020B42B0020C02B0020FEFFFF0F7E
:10CAB000020000F0F72B0020A02B00202DE9F04F02
:10CAC00089B00593AE4B0027B3F90280B3F900306B
:10CAD000B8F1000FB8BFC8F10008002BB8BF5B4227
:10CAE0009845B8BF98468246B946BB463C46B8F51D
:10CAF000FA7F0492A8BF4FF4FA7802900397A14DF1
:10CB00002B88990757D0022C55D09D4B610033F9E3
:10CB100014209D4B33F9143003EB4202049B5B421B
:10CB20009A4203DB049B9342A8BF1346974A8E5E4A
:10CB3000059A9B1B32F914001E18FFF747FC90B1B1
:10CB4000934B304613F804B004F076FE914904F09C
:10CB50007BFF0146584603F0F5FF8E4904F0C0FE06
:10CB600005F084F806469AF808306422734393FB74
:10CB7000F2F39AF81C206FF0040101FB02FB5B4505
:10CB800005DB02EB82029342A8BF13469B4642F2AA
:10CB90001072814B53F8240030449042A8BF1046D5
:10CBA0007E4A9042B8BF104643F824009AF81230EB
:10CBB000584303130393298801F00303012B01D188
:10CBC000022C3DD16E4B764D33F91490029BA000A0
:10CBD00093F801E0734B55F8247033F9146086EA3A
:10CBE000E673A3EBE673B3F5206F1CDC022C14D0C4
:10CBF000502303FB09F292FBFEF3042296FBF2F6AC
:10CC00009E1B3744B7F57A5F674BA8BF4FF47A573E
:10CC10009F42ACBF2F502B5007E089EAE973A3EB8A
:10CC2000E973642BE4DD00232B505D4B7D27C35853
:10CC300093FBF7F7029BDB7A7B43402793FBF7F7E5
:10CC40008A0713D5022C11D008FB07F508FB09F65B
:10CC50000398C8F5FA7303FB0B6603FB00534FF40C
:10CC6000FA7296FBF2F193FBF2F508E0CB0704D5DC
:10CC7000022C02D0039D594601E03D46494663001F
:10CC80000193484B042633F91430484A93FBF6F3DA
:10CC9000A25C6FF04F06534393FBF6F39AF85120D2
:10CCA000CE18E2B1022C069230460BD104F0C4FD3E
:10CCB000069A530803D09A42A8BF1A4600E0012200
:10CCC0003B4905E004F0B8FD3A49069A01EBC4017E
:10CCD000394B1B68FAF764F804F0C8FF0646314B7D
:10CCE000019A0198D15A354B0AB2C05E4FEA840CC2
:10CCF000121A042092FBF0F20198C15203F10801CC
:10CD0000143351F824E053F8240041F824207044EF
:10CD100010449AF8502043F824E082B1CDF81CC0AA
:10CD2000069204F089FD2649234B01EBC401069AC3
:10CD30001B68FAF735F804F099FFDDF81CC0214BA9
:10CD4000214A1B5D01995843202390FBF3F073198E
:10CD50001B1A8B521D4B40424CF803601C4B013494
:10CD60004CF803501B4B032C4CF80300029B03F1BF
:10CD7000010302937FF4C3AE09B0BDE8F08F00BF9A
:10CD80004C1000200C1900208C3000206A2E00204E
:10CD9000C08401080000204148230020F0D8FFFF94
:10CDA000582B0020880F002080C1FFFFE02B0020BF
:10CDB0004C2B00203C2B0020542B002078230020FB
:10CDC000882B0020F42B0020A02B0020A82B002073
:10CDD000B42B0020C02B00202DE9F04F89B0059323
:10CDE0009D4B80461B880C469B0702924DD540F216
:10CDF000E631129B994AD889B2F900301B1A03F226
:10CE0000F3158D4203D8002BB8BF5B4201E04FF40D
:10CE1000FA73B2F90220101A40F2E63200F2F3116E
:10CE2000914203D80028B8BF404201E04FF4FA70A5
:10CE300098F84C503DB39842B8BF1846C0F5FA7008
:10CE400004F0FAFC864904F0FFFD4FF07E5104F037
:10CE50003DFC0646642090FBF5F004F0EDFC014635
:10CE6000304604F03DFD4FF07E5104F031FC0021CE
:10CE7000074604F0D3FE30B938464FF07E5104F037
:10CE8000EBFE20B101E0002701E04FF07E57E31CEC
:10CE90000393CDF800800024039B022C13F8015F5C
:10CEA000704E039309D1B6F904000A35684304F0C3
:10CEB000C3FC6D4904F0C8FD74E036F9140004F0B9
:10CEC000BBFC8146029804F0B3FC654904F0BCFD4C
:10CED0000146484604F004FD644B814633F91400D2
:10CEE00004F0AAFC0146484604F0F2FB029B81468E
:10CEF000584204F0A1FC8346484659464FEA440A8A
:10CF000004F08CFE48B9029804F096FC834648462B
:10CF1000594604F0A1FE00B9CB46554B33F90A003F
:10CF200004F08AFC0146584604F0D0FB059B81467C
:10CF300033F9140004F080FC0146484604F0C8FBB5
:10CF40004C4904F081FD8146FFF740FA28B14A4B75
:10CF50004946185D03F0F6FD81463F4BB3F800B03B
:10CF60001BF0010F05D04846D8F8441004F0B8FC77
:10CF700018E036F90A001435684304F05DFC3A49BC
:10CF800004F062FD1BF0020F05460CD0D8F84810E3
:10CF9000484604F0A5FC394604F0A2FC01462846A8
:10CFA00004F096FB054663000493344B344E33F98A
:10CFB000140004F041FC334B196E04F091FC01465F
:10CFC000284604F083FB009B8246196A04F088FC23
:10CFD0002D4B0546185D04F02FFC0146284604F051
:10CFE0007FFC2A4904F030FD98F85120814692B127
:10CFF000022C09D1530803D09A42A8BF1A4600E078
:10D0000001224846224902E0224901EBC40133686B
:10D01000F9F7C6FE8146336850461946019304F07D
:10D020005FFC009BDFF878B0D96A04F059FC114925
:10D0300004F056FC5BF8241004F04AFB1649A500E6
:10D04000064604F0EBFD68BB3046144904F004FECC
:10D0500048B3124E27E000BF0C1900206C2F0020AF
:10D060000000FA434C100020000048428C300020A1
:10D070006A2E002000002041C0840108880F002093
:10D08000542B002048230020382B00200000C842E9
:10D090004C2B00203C2B002000007AC300007A4378
:10D0A000D42B0020444E4BF80560DFF83CB15046CD
:10D0B00055F80B1004F00AFB45F80BA006900199F7
:10D0C0004FF07E5004F0C0FC069B0146184604F069
:10D0D00007FC82460BF10C03EA580BF1180B1046C3
:10D0E00055F80B100793069204F0F2FA514604F03B
:10D0F000EFFA069A079B45F80B2098F85020014656
:10D1000045F803A032B12D49019B01EBC401F9F7A9
:10D1100047FE014608462A4904F096FC009B996B9D
:10D1200004F0DEFB274B8246185D04F085FB0146C8
:10D13000504604F0D5FB244904F086FC234982467E
:10D1400004F06CFD38B95046214904F085FD20B14A
:10D15000DFF87CA001E0DFF874A03146484604F017
:10D16000B7FA514604F0B4FA08F0F2F8194BB0F5EA
:10D170007A7FA8BF4FF47A709842B8BF1846049AD5
:10D18000154B0134D052484604F070FD134B5851F2
:10D19000304604F06BFD124B5851504604F066FDCA
:10D1A000104B032C5851009B03F1040300937FF4B0
:10D1B00073AE09B0BDE8F08F00007AC3882B002061
:10D1C00000004040382B00200000C842000096C3F9
:10D1D0000000964318FCFFFFA02B0020A82B002086
:10D1E000B42B0020C02B0020AC230020044B0022D5
:10D1F0001A605A60034B00221A605A60704700BFE1
:10D2000048230020CC2B002010B50C4C0123E370E8
:10D210004FF48060022384F82030FAF76FF9084A4F
:10D22000084BD2F888201B685278642101FB023336
:10D23000636123880133238010BD00BF4430002088
:10D2400048230020982E002010F80A3C0133DBB25E
:10D250000A2B84BF10F8131C044A00F80A3C82BF52
:10D26000002322F8113000F80A3C7047902F00206C
:10D27000334A70B5136C9068194440F68C23081A31
:10D2800098429160D060516013463BD9127893F96F
:10D29000451010468A420BD1111F082908D893F86F
:10D2A0004610182901D8013103E083F8442002E038
:10D2B000002183F8461093F944402149A24219D134
:10D2C00091F84740B4B10C310024944206DA51F889
:10D2D000046F1C4D25F814600134F6E70C2805D0C6
:10D2E0001849002421F810400130F7E7164801786A
:10D2F0000131017083F84520002201211A7083F862
:10D30000471070BD92F84710C9B140F2DA51A0F24F
:10D31000EF248C4208D811780B2905D80B1D013158
:10D32000117042F8230070BD002283F84720074B9C
:10D3300003F13002002143F8041F9342FAD170BD7B
:10D34000F4000020902F002004060020000100209F
:10D35000024A136C0133194411647047F400002031
:10D36000024B53F820301B6819807047F82B0020BF
:10D37000074BA1F57A7153F820301A681B8959437D
:10D380004FF47A7391FBF3F189B21180704700BFBB
:10D39000F82B002037B5044603211E2006226B46D9
:10D3A000F7F760FD78BB9DF801309DF80000174D40
:10D3B00043EA002000B204F03FFA296804F090FA32
:10D3C00004F054FC9DF8033020809DF8020043EAED
:10D3D000002000B204F030FAA96804F081FA04F0E9
:10D3E00045FC9DF80530A0809DF8040043EA00202C
:10D3F00000B204F021FA696804F072FA04F036FC15
:10D400006080012000E0002003B030BD2400002037
:10D4100090F83B3210B57BB990F83A3290F8394227
:10D42000A34209D2B0F8401201229A400A430133C4
:10D43000A0F84022DBB2F3E710BD1FB50123ADF821
:10D440000830ADF80410002301A9ADF80A30ADF89A
:10D450000C30ADF8062000F072FE05B05DF804FB5C
:10D460008379DB0748BFB1FA81F1D0F8343148BF86
:10D4700049095A681B8909B11361704753617047A4
:10D480001FB50123ADF808300023ADF80C30ADF81E
:10D490000A30094BADF804101B7801A9012B08BF15
:10D4A0000323ADF8062008BFADF80C3000F047FEAE
:10D4B00005B05DF804FB00BFF000002038B510F89F
:10D4C0000E2C044650F8043C52B9012200F80E2CF0
:10D4D00020F80C1C997A18680222BDE83840CFE782
:10D4E00030F80C2C20F80A1C891A89B220F8081C84
:10D4F000074A10F80F0C002522F8101004F80E5CF3
:10D500001868997A2A46FFF7BBFF04F8065C38BD15
:10D51000902F0020044B53F820301BB107289CBFEC
:10D520001B681980704700BF1C020020084A13685E
:10D530009B020BD5074B002119704FF6FE7306496D
:10D54000086803400B604FF400135360704700BF3E
:10D5500000000240913000206C0002402DE9F047AD
:10D56000664D2B686649581C0A788E4602F0FF0605
:10D570000AB10346F6E737462B60687BAB6895F83F
:10D580000C80AA7B39B2202900F09C80DFF880C192
:10D590000CEB8103DC789B783CF82110C3F1FF038E
:10D5A0009BB2002B65D04FF03C0CB1FBFCF9C3F1F2
:10D5B000FF0363431B12B9F1050F5DD8DFE809F0E3
:10D5C000030B1A293A4AE01A4143B1FBFCF0DAB2E4
:10D5D0001044C0B251E0B1FBFCF00CFB101189B259
:10D5E000DAB2C1F13C01E31A4B43B3FBFCFC204629
:10D5F00094442CE0B1FBFCF00CFB1011E21A89B250
:10D600004A43B2FBFCF25FFA83F84244D2B22046AE
:10D6100032E0B1FBFCF90CFB191189B2E01AC1F13F
:10D620003C014843B0FBFCF05FFA83F84044C0B2D1
:10D63000224621E0B1FBFCF80CFB1811D8B289B2EC
:10D64000E31A01FB03F2B2FBFCFC224684445FFABE
:10D650008CF412E0B1FBFCF80CFB181189B2D8B2C3
:10D66000C1F13C01E31A4B43B3FBFCF20244D2B2DA
:10D6700003E02246204600E044464FEA042C4CEAF0
:10D68000004C4CEA020C17234FF0010808FA03F88B
:10D6900006F1170118EA0C0FA1EB0301DFF8748003
:10D6A00014BF4FF011094FF0090989B213F1FF338C
:10D6B00008F80190E8D218360137B6B2BFB2114B64
:10D6C000A0465FE7AB6001238EF8003040F22A33BA
:10D6D000AA730D4AE9800D4985F80C806873AE8005
:10D6E000536000238B840B889BB243F001030B80B3
:10D6F000136843F001031360BDE8F087D4230020D2
:10D7000091300020E02300206C0002400004004023
:10D71000DA0C0020B1020020F0B5B1F800E00023DF
:10D720004EFA03F2D50725D58E784FEAD30CF406CE
:10D7300048BFCC7806F00F0203F0070748BF22432A
:10D74000BF0050F82C500F24BC4025EA0404BA4016
:10D750002243282E40F82C2005D1C46801229A408B
:10D7600024EA020205E0482E04D1C46801229A404E
:10D770002243C2600133102BD2D1F0BD2DE9F04F0E
:10D780001E464FF414734343554D85B005F1100404
:10D7900080469146E718A24610B92B44514A03E04F
:10D7A000012805D1504A2B441A641032C3F8442191
:10D7B0004FF4147303FB08F34C48EC180AEB030214
:10D7C00003F59C73343253442061E1636262A362C7
:10D7D00000224FF480714FF0010BD4F84431032044
:10D7E000E1612263E2622162A263626384F84C22F7
:10D7F00084F848B284F84922A4F85222A4F85422AA
:10D80000C4F818906075A67584F8568258681B890C
:10D8100004F5A0724FF0020CADF80C3003A91023F0
:10D8200001928DF80E308DF80FC0CDF800C0FFF7D3
:10D8300073FF236CDDF800C0597B58681B898DF895
:10D840000E1003A9ADF80C308DF80FC0FFF764FF80
:10D8500059463846FFF704FE3220FAF7DCFE244B27
:10D86000019A1B68D2F804B01A46B2FBF9F1B1F57F
:10D87000803F03D3012AF8D95208F6E71D4A4FF436
:10D880001474B3FBF2F204FB08F8584689B2D2B222
:10D89000FCF738FA05EB0809174B08F512780AEB84
:10D8A00008040022C9F8583258462146FCF772FA9B
:10D8B000D9F8405016F0010F0CBF02220022286850
:10D8C000A97AFFF7BAFD0D4B2846C9F85C32211D35
:10D8D0000022FCF75FFA384605B0BDE8F08F00BFC4
:10D8E000D4230020009501082095010874840108C4
:10D8F0005400002040420F00FBB900085DB9000849
:10D900002DE9F7438E460546DFF8A092114699F8B7
:10D91000B0440068164698467246631C89F8B034D5
:10D92000FCF79CF92B8901A9ADF8043018238DF878
:10D930000630686802238DF80730FFF7EDFEAB7AFA
:10D9400009F2B447240127442A6849460C2B00F207
:10D95000F680DFE813F00D00F400F400F40051004D
:10D96000F400F400F4008A00F400F400F400C200B3
:10D97000138CDFF83CC223F001031B041B0C13843F
:10D98000138CB2F804E0108B624520F073004FEA6C
:10D9900000404FEA10409BB21FFA8EFE40F070002C
:10D9A00014D00CF5006C624510D00CF5406C62454B
:10D9B0000CD00CF5806C624508D00CF5806C62458B
:10D9C00004D023F0020343F0030307E023F00E0327
:10D9D0002EF4407E43F003034EF4807EA2F804E070
:10D9E0001083A2F834801384138B23F008031B04E4
:10D9F0001B0C43F0080336E0138CDFF8B4C123F0AE
:10DA000010031B041B0C1384138CB2F804E0108B5E
:10DA1000624520F4E6404FEA00404FEA10409BB2D6
:10DA20001FFA8EFE40F4E04008D00CF5006C624511
:10DA300004D023F0200343F0300307E023F0E00399
:10DA40002EF4406E43F030034EF4806EA2F804E0F2
:10DA50001083A2F838801384138B23F400631B0413
:10DA60001B0C43F40063138369E0138CDFF840C19F
:10DA700023F480731B041B0C1384138CB2F804E092
:10DA8000908B624520F073004FEA00404FEA10404F
:10DA90009BB21FFA8EFE40F0700008D00CF5006CAF
:10DAA000624504D023F4007343F4407307E023F489
:10DAB00060632EF4405E43F440734EF4805EA2F83F
:10DAC00004E09083A2F83C801384938B23F0080336
:10DAD0001B041B0C43F0080330E0138CDFF8D0C0AC
:10DAE00023F480531B041B0C1384108CB2F804E045
:10DAF000938B20F4005023F4E6431B0400041B0C1A
:10DB0000000C62451FFA8EFE43F4E04340F440509F
:10DB100003D00CF5006C624503D12EF4804E4EF418
:10DB2000804EA2F804E09383A2F840801084938B87
:10DB300023F400631B041B0C43F4006393832B7BCF
:10DB400043B1B2F844306FEA43436FEA53439BB2A8
:10DB5000A2F8443013889BB243F001031380AB7AE0
:10DB60000C2B19D8DFE803F0071818180B18181831
:10DB70000F18181813000B1902F134000AE00B19E2
:10DB800002F1380006E00B1902F13C0002E00B192B
:10DB900002F14000C3F8B40438460C44A4F8BC6455
:10DBA000C4F8B82403B0BDE8F08300BFD42300203C
:10DBB000002C0140084BDA68D10709D4DA68520713
:10DBC00008D4DB6813F0100F14BF03200420704743
:10DBD000012070470220704700200240704701205A
:10DBE0007047704703788B4286BF024B33F81100B1
:10DBF000002070474829002008B50021062207F0C0
:10DC00009AF9012008BD08B50021062207F093F912
:10DC1000012008BD70B50546FAF7D6FC324CA36961
:10DC2000A061C31AB3F5FA5FE36182BF002384F8F1
:10DC3000203084F8213094F820302BB9A12D02BF78
:10DC4000294A012182F8211094F82110264A31B185
:10DC5000D118EDB2013381F8225082F8203094F8C7
:10DC6000205094F84330AB423CD11F4B93F84430E2
:10DC7000052B02D0062B03D02FE0002003F04EFC32
:10DC800094F823301E2B28D100200246C1B26B1E0F
:10DC900099421ADA214491F822300821DBB283EA52
:10DCA0000206F60744BF83F01803C3F3460301F1ED
:10DCB000FF3154BF5B0843F0800311F0FF01C2F352
:10DCC0004702ECD101301A46E0E7234493F82230B2
:10DCD0009A4202D1032003F021FC002384F8213072
:10DCE00084F8203070BD00BF4829002010B50446DC
:10DCF000B0F9000002F002FFB4F9020002F0FEFEEB
:10DD0000B4F90400BDE8104002F0F8BE10B50446B6
:10DD1000006802F0F3FE606802F0F0FEA068BDE863
:10DD2000104002F0EBBE2DE9F74F0120FAF722FB7D
:10DD3000002488B3012C2FD84FF04C0909FB04FABA
:10DD4000174E06EB0A0808F19007BD7815B10134AB
:10DD5000E4B2EEE790F9003090F804E01846114B79
:10DD600003228DE8240001212A4653F82E30FAF7C9
:10DD700098FC834660B106F14800504429464A4663
:10DD800007F0D9F801231C44C8F848B0BB70E4B2CE
:10DD90000120FAF7D5FACCE703B0BDE8F08F00BF59
:10DDA000482900208C8401080021222210B5104847
:10DDB00007F0C1F80F4B002219460F480424105CED
:10DDC000013283F8F60183F8FB4105200024042A80
:10DDD00083F8FA0183F8FD4183F8FC0103F108039D
:10DDE000EBD10123A1F8F831522381F8F43110BDB1
:10DDF00048120020541000201AA3010870B50646EE
:10DE0000441E14F8011F89B1094D284607F0C9F8CE
:10DE10000028F6D005F1080398423FBF054B401B90
:10DE2000C018A31B38BF80F88A31EAE770BD00BF75
:10DE30001EA3010854100020031EB8BF2D2210B5E8
:10DE4000B8BF58420C46B8BF01F8012B0A22F9F7B7
:10DE5000D3F800230370204610BD07B51C4B03F117
:10DE6000E402C3F8E0201B4A92F892215AB1012A39
:10DE700014D1032183F8E610072183F8E82083F802
:10DE8000E7100C2208E0022183F8E610032183F852
:10DE9000E82083F8E710072283F8E4200E4A0F4BAE
:10DEA00040201A60FAF766FA70B10122002390F957
:10DEB000000040218DE80C00094A4FF4E133FAF7E5
:10DEC000F0FB003018BF012003B05DF804FB00BF79
:10DED0004829002054100020D512010830000020ED
:10DEE000891301080120002101F0F0BF174AF0B5A5
:10DEF000164692F8E930D2F8ECE0032B10D85C1CFF
:10DF00000EEBC3039D1CE4B208D09A88D10705D557
:10DF1000104203D008E00131042907D12346ECE781
:10DF200086F8E9300020F0BD9F7800210C2202FB2A
:10DF300001F3064D05F1F00C1CF803209742EAD1DD
:10DF40002B4485F8E940D3F8F400F0BD48290020BF
:10DF50008A6810B50C6A036814430A6923F4FF4306
:10DF600014434A6923F0700314438A691443CA694D
:10DF700014434A6A14438A6A224313430360CB68FA
:10DF800043600B6883604B68C36010BD4FF6FE733F
:10DF90000268134003600023036043608360C36032
:10DFA000284B984201D1284A27E0284B984201D1BA
:10DFB000254A2AE0264B984201D1234A2DE0254BE1
:10DFC000984201D1204A30E0234B984201D11E4AA9
:10DFD00033E0224B984204D11B4A536843F4700348
:10DFE0002EE01F4B984204D1174A536843F07063E8
:10DFF00026E01C4B984204D11B4A536843F00F03A0
:10E000001EE01A4B984204D1174A536843F0F003BC
:10E0100016E0174B984204D1134A536843F47063D7
:10E020000EE0144B984204D10F4A536843F47043F6
:10E0300006E0114B984204D10B4A536843F4702315
:10E040005360704708000240000002401C0002407C
:10E050003000024044000240580002406C00024080
:10E060008000024008040240000402401C040240F8
:10E07000300402404404024058040240224A10B5D1
:10E08000536803F00C03042B03D0082B04D01F4B60
:10E0900014E01F4B5B6811E053685168C3F383437E
:10E0A000C90303F1020301D41A4906E0516811F4CF
:10E0B000003F1749496818BF49084B43036053683C
:10E0C000154CC3F30313234493F820100368CB408B
:10E0D00043605168C1F30221214491F8201023FAD2
:10E0E00001F181605168C1F3C221214491F82010EF
:10E0F000CB40C3605268C2F38132224492F8302090
:10E10000B3FBF2F3036110BD0010024000127A006D
:10E110003000002000093D008C84010810B5044641
:10E12000FFF748FD012806D11CB1FFF743FD013C74
:10E13000F8E7052010BD002C08BF052010BD0A8897
:10E14000F0B54B888E88B1F808E0CC88002A3AD127
:10E15000028C43F0010322F001021204120C02842B
:10E16000058B078CADB225F0F30545EA0E1189B297
:10E1700041EA06027A49BFB2884212D001F5006135
:10E1800088420ED0B0F1804F0BD0A1F59831884273
:10E1900007D001F58061884203D001F58061884293
:10E1A00002D127F0020701E027F00A071F4302838C
:10E1B0000784038B23F00C031B041B0C0383038BCA
:10E1C0009BB21C4344E0042A44D1028C22F010028A
:10E1D0001204120C0284018B058C21F4407212058A
:10E1E000120D42EA0E325E4992B242EA062288429B
:10E1F000ADB292B212D001F5006188420ED0B0F1FA
:10E20000804F0BD0A1F59831884207D001F580618D
:10E21000884203D001F58061884207D125F02001B2
:10E2200041EA03139BB243F0100304E025F0A00180
:10E2300043F010030B4302830384038B23F44063F6
:10E240001B041B0C0383038B9BB243EA0424A4B27C
:10E250000483F0BD082A028C3ED122F4807212049D
:10E26000120C0284828B3E4D92B222F0F307018C95
:10E2700047EA0E1292B2A84289B242EA060212D0CE
:10E2800005F50065A8420ED0B0F1804F0BD0A5F582
:10E290009835A84207D005F58065A84203D005F55A
:10E2A0008065A84207D121F4007141EA03239BB2A3
:10E2B00043F4807304E021F4206143F480730B4342
:10E2C00082830384838B23F00C031B041B0C838346
:10E2D000838B9BB21C4341E022F480521204120C47
:10E2E0000284858B018C25F440752D052D0D45EAA2
:10E2F000062545EA0E321A4D89B2A84292B212D0D2
:10E3000005F50065A8420ED0B0F1804F0BD0A5F501
:10E310009835A84207D005F58065A84203D005F5D9
:10E320008065A84207D121F4005141EA03339BB232
:10E3300043F4805305E047F6FF5543F480530D4006
:10E340002B4382830384838B23F440631B041B0CC5
:10E350008383838B9BB243EA0424A4B28483F0BDFD
:10E36000002C0140CA78F0B5D40648BF8C780D88DF
:10E3700002F00F0348BF234315F0FF0F1DD00168C3
:10E3800000240126A64006EA0507B74211D14FEA4C
:10E39000840E0F2606FA0EF621EA0601282A03FA51
:10E3A0000EF641EA060101D1476102E0482A08BFA2
:10E3B00007610134082CE4D10160FF2D1FD94168A9
:10E3C000002404F108070126BE4006EA0507B7420B
:10E3D00011D14FEA840E0F2606FA0EF621EA060145
:10E3E000282A03FA0EF641EA060101D1476102E04C
:10E3F000482A08BF07610134082CE2D14160F0BD12
:10E400000F4B1A6842F001021A6059680D4A0A401F
:10E410005A601A6822F0847222F480321A601A68F4
:10E4200022F480221A605A6822F4FE025A604FF4E5
:10E430001F029A60044B4FF000629A60704700BF61
:10E44000001002400000FFF800ED00E02DE9F84365
:10E450005B4C0368013AC4F8203183880D46A4F868
:10E460002431072A42D8DFE802F0040A10182229D2
:10E470002F35B4F820310B80B4F8223113E0B4F812
:10E4800022310B80B4F8203105E0B4F820315B4232
:10E490000B80B4F822315B4205E0B4F822315B42D4
:10E4A0000B80B4F820316B80B4F824311DE0B4F84F
:10E4B00020315B420B80B4F8223112E0B4F82231F3
:10E4C0000B80B4F820310CE0B4F820310B80B4F8A4
:10E4D000223105E0B4F822315B420B80B4F82031E0
:10E4E0005B426B80B4F824315B42AB80354B1B7AC6
:10E4F000002B62D1B5F9000003F09EF98046B5F912
:10E50000020003F099F90746B5F9040003F094F905
:10E51000D4F828110646404603F0E2F9D4F8341145
:10E520008146384603F0DCF90146484603F0D0F84E
:10E53000D4F840118146304603F0D2F901464846EE
:10E5400003F0C6F806F004FFD4F82C1128804046EA
:10E5500003F0C6F9D4F838118146384603F0C0F903
:10E560000146484603F0B4F8D4F8441181463046D9
:10E5700003F0B6F90146484603F0AAF806F0E8FEB3
:10E58000D4F830116880404603F0AAF9D4F83C1161
:10E590008046384603F0A4F90146404603F098F857
:10E5A000D4F848110746304603F09AF90146384638
:10E5B00003F08EF806F0CCFEA880BDE8F88300BF1B
:10E5C000482900203000002044F6FB71084B1A68EF
:10E5D000137803EB431300FB03135078C0EB0030B8
:10E5E000B3FBF0F39078B3FBF0F080B2704700BF5C
:10E5F0003018002008B50A480A2290F84D3100EB87
:10E600004303B3F85C1100F5B47089B220F8041C20
:10E6100000F03DFC80B2FFF7D7FF024B188008BD29
:10E6200048290020341800202DE9F04F89B00593C7
:10E63000A04B80461B880492980737D540F2E632FB
:10E64000129B9D48DC89B0F900301B1B03F2F315C7
:10E65000954203D8002BB8BF5B4201E04FF4FA7338
:10E66000B0F9022040F2E630121B02F2F3148442A9
:10E6700003D8002AB8BF524201E04FF4FA72934225
:10E68000B8BF13460522C3F5FA7393FBF2F30A22CF
:10E69000643B534398F81C20D2105343642293FBED
:10E6A000F2F3134423EAE373DBB200E06423C146D0
:10E6B0000193CB1C03930024039B022C13F8016FDE
:10E6C0007E4F03934FEA440A05D1B7F904301B3655
:10E6D0005E4376114AE07A4B37F9142033F914304F
:10E6E00003EB4202049B5B429A4203DB049B93428E
:10E6F000A8BF1346734A32F90A50059A5B1B32F9D8
:10E70000145003EB050BFDF761FE88B16E4A5846C5
:10E71000155D03F091F86D4903F096F9014628461E
:10E7200002F010FA694903F0DBF803F09FFA834620
:10E73000604A1288D10714D437F90A501B366E4349
:10E7400093074FEA261611D598F812509DF9042028
:10E7500005FB0BF35343642293FBF2F306EB231602
:10E7600004E098F8085005FB0BF52E11584B0425D2
:10E7700033F90A30574F93FBF5F5751B99F8016093
:10E78000E35D6E435E430293642396FBF3F698F8D1
:10E7900051B0F611BBF1000F1BD0022C30460CD14A
:10E7A00003F04AF85FEA5B0304D05B45A8BF5B4611
:10E7B0001A4600E00122484905E003F03DF85A46B8
:10E7C000391D01EBC401FB69F8F7EAFA03F04EFAD0
:10E7D0000646424B99F80B7019883E4B01FB05F237
:10E7E00003F1200E5EF82400D21207FB02073C4A18
:10E7F000B7F5001FA8BF4FF40017974203F12C0094
:10E80000B8BF174650F8242040F824504FF6FF7048
:10E810000909B0FBF1F1AA1A4A4303F1380103F1E7
:10E8200044054EF8247051F824E055F8240045F8CA
:10E8300024E098F85050921170444FEA840C7F13F2
:10E84000104441F824208DB1CDF818C0079302F090
:10E85000F3FF079B2A4603F1500101EBC401DB697A
:10E86000F8F79EFA03F002FADDF818C099F81530AF
:10E87000F2195843029B013443431846642390FB2A
:10E88000F3F0184B0012024423F80A2003F10802A7
:10E890004CF80260032C03F1140203F120034CF83E
:10E8A00002704CF8030009F101097FF405AF09B0CB
:10E8B000BDE8F08F0C1900206C2F00204C100020B8
:10E8C0008C3000206A2E0020C08401080000204106
:10E8D000880F0020382B00204C2B0020640F0020D4
:10E8E0000000E0FFA02B00202DE9F04F054690F836
:10E8F00050008DB008910592099318B13228A8BF35
:10E90000322000E0012002F097FF0146AA4803F000
:10E910009BF8AA4B04461888002808BF012002F083
:10E920008BFFA749069002F0DBFF0190019920467A
:10E9300002F0CEFE0146019803F086F8A14B079045
:10E940001B889A0724D5A049B1F90030B1F902001B
:10E9500083EAE37280EAE071A2EBE372A1EBE0717B
:10E9600091420C46B8BF1446B4F5E17F12DA9142E9
:10E9700003DD0028D8BF404203E0002BCCBF18467F
:10E98000584202F059FF914903F05EF8064603E051
:10E99000002601E04FF07E564FF00009CA4603956D
:10E9A0000024630004938A4B33F9140002F044FFFF
:10E9B000884902F095FF03F059F902F03DFF8649BE
:10E9C00002F08EFF804B029033F9140002F034FF06
:10E9D0007C4B07461B889B077ED0014602F078FEE1
:10E9E0007E4B804633F9140002F026FF0146404674
:10E9F00002F06EFE03F03AF9059B5B42984203DB9E
:10EA0000059B8342A8BF0346754A0499885E099A0C
:10EA10001B1A32F91400184402F00EFF8046FDF76D
:10EA2000D5FC70B16F4B40466F4914F8039003F06A
:10EA30000BF80146484602F085F86B4902F050FF9A
:10EA40008046287F02F0F4FE684902F049FF8246C2
:10EA5000287A02F0EDFE0146404602F041FF64498B
:10EA600002F03EFF03F002F981460AF1004003F094
:10EA7000FDF8814505DB504603F0F8F84845A8BF8E
:10EA8000484602F0D9FEDFF88C9101998246404653
:10EA900002F026FF59F8241002F01AFE55494FEAF9
:10EAA000840B804603F0BAF838B94046524903F067
:10EAB000D3F820B1DFF8408101E0DFF8388149F870
:10EAC0000B80A87C02F0B4FE0146404602F008FF2D
:10EAD0004A4902F005FF81463A4BB3F800B01BF0FB
:10EAE000010F40F099803A4B049ADFF82081D35E01
:10EAF000002BB8BF5B42B3F5206F4FEA84030A9343
:10EB000003DD002348F824302AE03D49384602F06E
:10EB1000E7FE039B0B90587802F08AFE0B9A0146A1
:10EB2000104602F091FF029902F0D0FD019902F027
:10EB3000D7FE58F8241002F0CBFD3249804603F08E
:10EB40006DF838B94046304903F086F820B1DFF857
:10EB5000B88001E0DFF8AC802C4A0A9B42F80380C1
:10EB6000039BD87A02F064FE284B53F8241002F07D
:10EB7000B7FE274902F0B4FE1BF0020F80464DD0CD
:10EB80003846514602F0A2FD0146304602F0A8FE8A
:10EB90000146504602F09CFD49460746404602F0B9
:10EBA00095FD0146304602F09BFE0146484602F0C4
:10EBB0008FFD804632E000BF83F9223E640F0020C3
:10EBC000BD3786350C1900204C1000200000E143B1
:10EBD000880F00200000A03ECDCC4C408C3000209F
:10EBE0006A2E0020C0840108000020410000A040DF
:10EBF0006F12033C0000F0C10000F0410AD7A33DB2
:10EC00000000A043000040C300004043D42B00207C
:10EC10000AD7233CCC2B0020C8465746DFF83CB22D
:10EC20000BF1A803185D02F007FE0146029802F0FE
:10EC300057FE894902F054FE0146384602F046FD6F
:10EC400095F85120034642B10BF10401DBF81C306A
:10EC500001EBC401F8F7A4F80346804F029807F1CE
:10EC6000AC0B5BF824100A9302F030FD019902F01E
:10EC7000EBFE029B07F1B4024BF8243052F824B0AB
:10EC80000292594602F022FD0146079802F028FE42
:10EC90000146584602F01CFD029A834642F82400C1
:10ECA00007F1BC02105D02F0C7FD0146584602F0B4
:10ECB00017FE6B4902F014FE83460A9B4146184634
:10ECC00002F006FD594602F001FD06F041FB049BEF
:10ECD00007F16802D0520A9B07F1700218460292AF
:10ECE00002F0C4FF029A07F17C0342F82400404678
:10ECF000029302F0BBFF029B07F1880843F824004F
:10ED00000BF1004002F0B2FF039B48F824000133EE
:10ED100003930CB9012444E6089A524B9479B3F951
:10ED20000430640028345C434F4B6411B3F9040091
:10ED300002F082FD4FF07A5102F0D2FD06F008FB9E
:10ED4000201A02F079FD002CB8BF6442322C06462E
:10ED500002DD0023BB6224E0069802F087FF20F06A
:10ED6000030002F069FD8046687B02F061FD014608
:10ED7000304602F0B5FD3D490446404602F064FECF
:10ED80000146204602F0ACFD02F070FFBB6A184459
:10ED9000374B9842A8BF1846364B9842ACBFB86272
:10EDA000BB62BB6A6FF0FF005B13B3F5807FA8BF47
:10EDB0004FF480739842B8BF184602F03DFD80467C
:10EDC000304602F053FFEB785843801102F034FDD7
:10EDD00097F8BF300446032B11D9B5F84E60B6F54D
:10EDE000FA7F0CD202F042FF7342984203DBB0423A
:10EDF0000346A8BF3346184602F01EFD044695F8A8
:10EE0000512062B1530803D09A42A8BF1A4600E0CD
:10EE1000012220461849FB69F7F7C2FF0446414624
:10EE2000204602F055FC02F021FF00B202F004FD82
:10EE300006F08EFAA7F86C00204602F017FFB867BC
:10EE4000404602F013FF0023C7F88400C7F8903053
:10EE50000DB0BDE8F08F00BFA69B443B382B0020CF
:10EE6000F7CC92384C100020880F002000803B45E2
:10EE7000FEFFFF0F020000F04C2B002003689B6890
:10EE8000184703685B68184703681B681847B0F9A0
:10EE900002302DE9F74F93421CBF0023037090F816
:10EEA00000A004460E469146BAF1000F40F0AB8038
:10EEB000104602F0C1FC864902F012FD854902F0BD
:10EEC0000FFD4FF07C5102F00BFD06F0A1FA014658
:10EED000054602F005FD80498346284602F000FD04
:10EEE000034658461946019302F0F2FB4FF07E515B
:10EEF00002F0EEFB01464FF07E5002F0A5FD2946E0
:10EF0000804602F0EDFC294602F0EAFC0746014685
:10EF1000606002F0DDFBE7604FF07E572946A0609D
:10EF20002761284602F0D4FB294602F0D9FC4FF0B5
:10EF3000804102F0CBFB0146404602F0D1FC019B30
:10EF400060611946584602F0C1FB394602F0C0FB29
:10EF50000146404602F0C4FC40F2DC53A04627467E
:10EF6000554663651023A4F852301823A061A4F815
:10EF700050304FF09741D8F8100002F0B1FC00215A
:10EF8000824602F04BFE28B150464FF07C5102F011
:10EF90009DFB04E050464FF07C5102F099FB02F0DB
:10EFA000C7FEC7E90E014FF09741D8F8040002F000
:10EFB00097FC0021824602F031FE28B150464FF006
:10EFC0007C5102F083FB04E050464FF07C5102F08C
:10EFD0007FFB02F0ADFE0135032DC7E9080108F102
:10EFE000040807F10807C4D1A6F2DC531B04236709
:10EFF000E3676367C4F88030A367C4F884300123F3
:10F00000A4F802902370D4F85490B4F95280C9EB5C
:10F010000606636A06FA08F67343276A4FEAE67B38
:10F02000206F07FB0B332667A7FB0667E26F1F44C1
:10F03000636CD4F840C053434FEAE27B0CFB0B3EB9
:10F04000D4F88010C4F88020ACFB02237344B61AB5
:10F0500067EB0307E36AA26A43434FEAE07B02FBE4
:10F060000B3EA2FB00237344B6185F41E36C656F4F
:10F070004B436067A06C4FEAE17B00FB0B33C4F8A5
:10F080008410A0FB01011944636B361A05FB03F3DE
:10F09000206B4FEAE57B00FB0B3367EB0107A0FB1E
:10F0A0000501801919447941B4F95020A56702F08F
:10F0B000FBFA08F1FF3201239340E067C01841EBEF
:10F0C000E371424602F0F0FA484403B0BDE8F08F25
:10F0D0006F12833ADB0F4940F404B53F2DE9F84342
:10F0E0000024254BE0B293F8BF60B0420DD203EB91
:10F0F0008003224AD3F8C03032F810101BB10B281D
:10F1000001D8DB6898470134EBE71D4B1B685B03B4
:10F110002FD500242346E2B2B2422AD2DFF858901B
:10F120004FEA840809F1C00757F8242055689D422A
:10F1300017D02846FAF710FEEFF31283502282F31D
:10F1400012882821AA8C01FB009092B20132C0F8EB
:10F150001421AA8ADBB292B242F00102AA8283F39E
:10F16000118857F8083000221B6801341A802B469A
:10F17000D1E7BDE8F88300BF382B0020A80F00209E
:10F18000742E002008B50E4B1B6813F4805F0D4BE6
:10F1900014BFD3F89021D3F8942193F8BF1092882C
:10F1A0000023D8B2884204D2074820F81320013344
:10F1B000F7E7FFF793FFBDE808403220F9F72BBAD5
:10F1C000742E0020382B0020A80F00200A4B30B5E9
:10F1D0001A680A4B02F48052D3F89041D3F8945144
:10F1E00000230AB1A18800E0A988054820F813107F
:10F1F00001330C2BF5D130BD742E0020382B0020AC
:10F20000222E002070B5124D0024214605F29910DF
:10F21000702285F8984105F08EFE2146D5F80C3213
:10F220000B4A0B4493F9020088B11E6802F299144C
:10F230000E5108199C88073184809B79702983714D
:10F2400092F8983103F1010382F89831E6D170BD4C
:10F25000382B0020094B1A680E2303FB0020437A49
:10F26000FF2B07D0064A12789A4203D9054A32F892
:10F27000130000E0808800B2704700BF2C1F002000
:10F280002C2A00206C2F00202DE9F74F304C05462A
:10F29000D4F810723846F8F74FF806463846F7F7B4
:10F2A000D8FFD4F8147281463846F8F745F8019033
:10F2B0003846F7F7CEFFD5F804A00746314650464A
:10F2C00002F00EFBD5F8088083464946404602F01E
:10F2D00007FB0146584602F0F9F9019B296883466D
:10F2E000184602F0FDFA49460546504602F0F8FA83
:10F2F000394602F0F5FA0146284602F0E9F93946A6
:10F300000546404602F0ECFA314602F0E9FA0146C1
:10F31000284602F0DDF90146584606F0F1F80D499D
:10F3200002F0DEFA0C4902F08FFBD4F8181202F05A
:10F33000CFF90A4902F088FB06F00AF883B21A04F2
:10F3400044BF00F5B47083B218B203B0BDE8F08FCB
:10F35000382B00200000E144DB0F49400000204131
:10F3600001380A4B042804D8DFE800F00507090B30
:10F370000D00074A08E0074A06E0074A04E0074A8A
:10F3800002E0074A00E0074A1A6070474C0000207C
:10F39000BDCA000829E60008D9CD000883C70008C7
:10F3A000F1C30008E9E8000810B54B88DC0641BF4E
:10F3B0002F4B14791B6853F8244044BF2D4B43F85E
:10F3C00020404B889B0641BF294B54791B6853F85A
:10F3D000244044BF274B43F820404B881C070ED5E0
:10F3E000254B0C781B78B3EB141FA1BF204BD478AE
:10F3F0001B6853F82440A4BF1E4B43F820404B88A1
:10F400009B070ED51D4B0C781B78B3EB141FDFBF89
:10F41000174B54781B6853F82440DCBF154B43F856
:10F4200020404B88DC070FD5154C0B78247803F06F
:10F430000F03A342DFBF0E4B14781B6853F8244020
:10F44000DCBF0C4B43F820404B885B070FD50B7893
:10F450000C4903F00F0309788B42A1BF044B92784B
:10F460001B6853F82220A4BF024B43F8202010BD94
:10F47000241F0020DA0C0020472300204523002011
:10F480004423002046230020254A0023F0B51568B8
:10F490001C461A462348244903700B702E1976889F
:10F4A0004EB92F5D3FB9037000230A704B70077887
:10F4B0001C461A460CE0360548BF013204F104042C
:10F4C00003F1010348BFD2B2802CDBB2E6D1EAE7F8
:10F4D000E0B2B8420CD215F82400013406099E426D
:10F4E00000F00F00A8BF731C9042A8BF421CEFE7BA
:10F4F0008A704B70C2F3470102F001020A444C1EAD
:10F500000A490B480A70C3F3470203F0010313448E
:10F5100004700849501E084A08701370F0BD00BFFF
:10F52000281F00203C230020542D002046230020CB
:10F53000442300204723002045230020924B2DE93F
:10F54000F04FDA68914D1A612A6891B0DA60904AFA
:10F550000295136843F0200313608E4B1A78012A3A
:10F560000CBF002201221A708B4B1A78910740F1D0
:10F570004D838A490978042940F2488388490978EB
:10F5800001F0040101F0FF0011B922F001021A702C
:10F590001B78DB0702D408B1FAF7C4FA8149CA78AC
:10F5A000531C052293FBF2F202EB82029A1A7E4B65
:10F5B000CA701F7892000023DFF81082DFF81092E3
:10F5C00058F82310794C91FBF9FE04F1080040F83B
:10F5D00023E0774844F8231000FB0E1142F210702C
:10F5E00091FBF0F004F1100680B226F813004FF002
:10F5F000140C04F114060CFB036C04F13C0A5AF8D9
:10F6000023605CF802504CF80210761B314405264A
:10F610004AF8231091FBF6F109FB0E114434012F37
:10F6200044F823104FEA830B444605D10238B0F565
:10F63000797F98BF4BF808100BB90123BCE7594EEE
:10F64000029BB2461868336DC01A02F0F1F85949AE
:10F6500002F0FAF9029B4FF07E511B6807463365B2
:10F6600002F0DCFA08B94FF07E574B4BCAF85470E1
:10F670001B78514E13F00103504D12D00DAA009289
:10F680004F4B0EAA01920CCB94E80300FAF760F9F5
:10F690000D9A6421B2FBF1F20E9B328093FBF1F3E1
:10F6A00000E033802B809AF858303E4D002B35D047
:10F6B000696D4FF07E5002F0C7F90746EB6D206888
:10F6C000C01A02F0B9F8394602F00AF902F0CEFA8F
:10F6D0002B6E86B2606836B2C01A02F0ADF8394BB4
:10F6E000196802F0FDF8394602F0FAF802F0BEFAA5
:10F6F000B5F9662000B28118B5F964200220B3186C
:10F7000091FBF0F193FBF0F389B29BB2A5F86A107C
:10F71000A5F86830A5F86610A5F8643001238AF8CA
:10F720005830294B61681B88206803F030031D4E58
:10F73000264DCAF86010CAF85C00002B00F0668203
:10F7400006F17403009306F178030193F26E336FB0
:10F75000FAF7FEF86B68306FC01A02F06DF8194BBB
:10F76000196802F0BDF802F081FAF36E2A68C6F853
:10F7700080009B1AF3670C4B1B78012B2AD0022BBD
:10F7800000F0E68042E200BF0C060020982E002028
:10F7900044180020D20F0020481800204E180020E6
:10F7A00092300020542D0020640E0020582D00209F
:10F7B000806967FF00007A44C2180020C418002046
:10F7C000D40F00203C0000200C190020501800200D
:10F7D00080969800D6F88430D6F8A0400293D6F8E8
:10F7E000943004F100400393D6F89830776D059378
:10F7F00002F03CFA8146204602F038FAD6F89C30F6
:10F80000BB4C0493BB4B06901B684FF0000B079357
:10F81000B94E4FEA4B0356F82B80A6F1140240462E
:10F8200032F81B50089302F007F8029902F058F8DA
:10F8300002F01CFA401B1FFA80FA283626F81BA09B
:10F840000FFA8AFA504601F0F7FF039902F048F8E0
:10F8500002F00CFA86B20AEB080001F0EDFF059900
:10F8600002F03EF8394602F03BF8216801F030FF23
:10F8700002F0FCF9484504DB069B9842A8BF1846F5
:10F8800000E0484601F0D8FF206002F0EFF9079B46
:10F89000304486B2987801F0CBFF984902F020F806
:10F8A00001464FF07E5002F0CFF8394601F010FFCC
:10F8B0000146384602F0C8F809906068D4F808A0FC
:10F8C000C0EB080001F0B8FF394602F0BDF8514620
:10F8D00001F0FCFE099A0146104602F001F80146CB
:10F8E000504601F0F5FE3135ADB2622D0146206182
:10F8F000C4F80480A0600ED9049801F0F1FF02F072
:10F90000B5F97F4AB0F5FA6FA8BF4FF4FA6090429C
:10F91000B8BF104600E0002040F6B832064436B2C8
:10F920009642A8BF1646774A089B9642B8BF16462D
:10F93000754A54F8140B9E52142202FB0BF27349C1
:10F940005050BBF1000F40F061814FF0010B5FE7B9
:10F95000684BB6F8A8401F68736F3D8902935B0837
:10F960009D4228BF1D4623B29D4202DC1FFA85F945
:10F970000AE06749706D01F0B3FF02F077F92044A7
:10F980001FFA80F9A6F8A890DAF87860DAF8AC40A7
:10F99000341B2046FAF71EF841F293130028D8BF13
:10F9A00040429842CCBF0020012078B3204601F0AD
:10F9B00043FF584901F094FFF7F74BFC04460298C7
:10F9C00001F036FF0146204601F08AFF02F04EF9B1
:10F9D00040F6B83380B2AAF8B00000B29842A8BF8F
:10F9E0001846484B9842ACBF3018F01848F6A04370
:10F9F000984203DDA0F50C40A03804E00028BCBF0D
:10FA000000F50C40A030CAF8B40001E0CAF8B460B8
:10FA1000DAF8B4300026C3F50C502830039301F017
:10FA20000BFF3C4901F05CFF0446F7F785FC0F90A3
:10FA30002046F7F70EFCDAF8B830DAF8C440059340
:10FA4000DAF8BC300E9004F10040089302F00EF991
:10FA50000490204602F00AF9DAF8C030DAF854804F
:10FA60002A4C09900793730048460A9301F0E4FE7C
:10FA70000EAB53F8261001F033FFDFF8A0A00546C7
:10FA80003AF9160001F0D8FE0146284601F01EFEA4
:10FA900002F0ECF805B2204BB5F57A7FA8BF4FF421
:10FAA0007A759D42B8BF1D460AF13C0AA8B22AF8F1
:10FAB000160000B201F0C0FE0599824601F010FF69
:10FAC00002F0D4F8089983B25046069301F008FF7B
:10FAD000414601F005FF216801F0FAFD02F0C6F889
:10FAE000049B98421CDB099B9842A8BF184618E06B
:10FAF000A00E0020680E0020D02D0020DB0FC94092
:10FB000030F8FFFF48F4FFFF720E0020C80E0020FF
:10FB10000000C842D302373918FCFFFFBC2D00207B
:10FB2000049801F089FE20608346B87801F080FED9
:10FB3000384901F0D5FE01464FF07E5001F084FFB8
:10FB4000414601F0C5FD0146404601F07DFF0B90A6
:10FB50006068D4F808A0281A01F06EFE414601F052
:10FB600073FF514601F0B2FDDDF82CC0014660463E
:10FB700001F0B6FE0146504601F0AAFD656001465F
:10FB80002061A060079801F0ABFE02F06FF8069BC1
:10FB90001434034458469A4602F068F840F6B832E6
:10FBA000504400B29042A8BF10461B4A0A9B9042A4
:10FBB000B8BF1046194A1A4998521422724342F8A3
:10FBC00001B00EB901264EE73B792BB1039A6423AD
:10FBD00092FBF3F3134A13803B88029A124C9A4229
:10FBE0000DD9D4F8AC30A06FC01AF9F7F3FE42F289
:10FBF000107380EAE072A2EBE0729A4206DD0B4BD2
:10FC000001221A70B4F8C820064B1A8011B0BDE862
:10FC1000F08F00BFDB0FC94048F4FFFF720E0020D9
:10FC2000A00E0020600E0020542D0020640E002045
:10FC300007B5064B06490093064B074A0193074850
:10FC4000074BF7F7D8FA03B05DF804FB04960108F8
:10FC500053A30108D99501085DA3010833A3010846
:10FC6000F895010808B5037833B90C4B0C4819789E
:10FC7000BDE80840F7F7BFBA05F0F6F902280CD83E
:10FC8000064B0C221870074B02FB0030064B02306B
:10FC90001860F7F71BFD0548E5E708BD202E00209A
:10FCA00064A3010804180020CC0F0020FB98010871
:10FCB00008B503783BB90B4B0B4893F8B017BDE878
:10FCC0000840F7F798BA05F0CFF9022808D8054B95
:10FCD00083F8B007F7F754FCF7F71CFD0348E8E793
:10FCE00008BD00BF5410002068A30108FB9801085C
:10FCF00038B5037803BB214B1B6801330F2B07D8A2
:10FD00001F490C2202FB031295681C462DBB00E024
:10FD10001C4601340F2C01DD002400E005D81849F1
:10FD20000C2202FB04129568BDB99C42F1D1154822
:10FD3000BDE83840F7F75FBA05F096F90F2804469A
:10FD400005D80F4A0C2303FB00239D682DB92146DB
:10FD5000BDE838400C48F7F74EBA084B1C60F8F77E
:10FD6000E9FB21462A460948F7F745FA0C235C438C
:10FD7000034B185DBDE83840F8F7ECBB40000020AD
:10FD8000C484010875A301088BA30108A3A301087B
:10FD900073B5037813B9F7F749FF3DE01F4901AA8E
:10FDA00005F0C3F9002401462646254699B134B131
:10FDB000012C08D1084605F057F9064603E008462D
:10FDC00005F052F905461549002001AA05F0ADF9E4
:10FDD00001340146EAE70B2D02D911480C220BE051
:10FDE000022C10D1A6F57A73B3F57A7F07D90D48A6
:10FDF0004FF47A714FF4FA62F7F795FE0CE00A4B74
:10FE000003EB45035E80084B084803EB4503294696
:10FE1000B3F90220F7F7EFF902B070BD689D010851
:10FE2000689B0108CBA00108202E0020BAA301087E
:10FE300038B50D4C05462368834206D1F8F7ACF976
:10FE4000204600214C2205F076F8E36CAB4209D144
:10FE50002846F8F7A1F9BDE83840044800214C22B3
:10FE600005F069B838BD00BF90290020DC290020CA
:10FE7000034B1A68D379591C1344D171187A70470F
:10FE8000EC18002010B5FFF7F3FF84B2FFF7F0FF86
:10FE900004EB002080B210BD10B5FFF7F3FF04465D
:10FEA000FFF7F0FF04EB004010BD10B50446054B12
:10FEB00021461868FEF7E8FF034B1B6898796040FD
:10FEC000987110BDF0180020EC18002038B50446D9
:10FED0000D462420FFF7E9FF4D20FFF7E6FF002C39
:10FEE000084C14BF21203E20FFF7DFFF23680022CB
:10FEF00028469A71FFF7D9FF236893F84900BDE8B7
:10FF00003840D2E7EC18002001460020DEE710B5AB
:10FF10000446C0B2FFF7C9FF200ABDE81040C4E79D
:10FF200010B5044680B2FFF7F2FF200CBDE8104088
:10FF3000EDE737B582888368044610060D4641BF59
:10FF400029494FF4CC7091F8B01700FB0133D1056B
:10FF500042BF26490C20097802F03F0248BF00FB4F
:10FF60000133042A12D006D8012A0DD0022A2FD13B
:10FF700093F900102DE0102A0AD0202A0AD0082A6E
:10FF800026D1B3F9001024E0197822E0198820E086
:10FF900019681EE069461868F6F7C8FF014614485C
:10FFA000F7F729F9F5B1E06801F046FC6946F6F784
:10FFB000BDFF01460F48F7F71EF9206901F03CFC30
:10FFC0006946F6F7B3FF01460A48F7F714F909E066
:10FFD00000210948F7F70FF925B10848E1682269BF
:10FFE000F7F709F903B030BD54100020202E00208F
:10FFF000819C01087A9C0108CDA30108C9A30108CE
:020000040801F1
:10000000024B0146D869FEF73FBF00BF202E0020FB
:1000100010B5441E14F8011F21B1034BD869FEF737
:1000200033FFF7E710BD00BF202E0020F7B52A49A7
:100030002A4B08782A4D1C682A4B05EB80001A8849
:10004000D0F8C010284B29481B7800914FF47A71E2
:10005000B4FBF1F1F7F7CFF8254B26481968264B8A
:100060000026B1FBF3F1F7F7C6F8244B1F68F3B293
:1000700005EB8302D2F8D010E9B101249C403C4248
:1000800017D0220715D01E4A0B20D25C00FB032399
:10009000134A1C4802EB8303D3F8F020F7F7ABF8C0
:1000A000022C06D1184B93F8281011B11748F7F716
:1000B000A2F80136DBE71648FFF7AAFF154B1648F2
:1000C0001A88164B92B2198840F2DC7303B0BDE86F
:1000D000F040F7F790B800BF94180020982E002049
:1000E000C48401083418002044000020D0A3010873
:1000F0005400002013A4010840420F0044180020BF
:100100005000002023A40108202E00202BA4010869
:1001100073A40108660F00202FA40108640F0020BB
:100120002DE9F0410024804625460F4E4146A7594F
:10013000384604F081FF58B139460C48F7F75BF8B0
:1001400030190021FFF7F5FE0948FFF761FF01357F
:1001500040F6BC4314349C42E7D11DB9BDE8F041E0
:10016000044855E7BDE8F08164860108EA9C01086F
:1001700073A40108BF9B01082DE9F74F824604F0E4
:100180001EFF054628B1012819D19AF800302A2B04
:1001900015D15948FFF73CFF0024584E5848A15943
:1001A000F7F729F830192946FFF7C3FE5548FFF73E
:1001B0002FFF40F6BC4314349C42EED198E05046E9
:1001C0003D2104F0EEFE002800F08D8003461D4620
:1001D00013F8012D202AFAD0441C204604F044FFD5
:1001E00081462046F6F70CFE0746CAEB05054FF0A0
:1001F000000B142404FB0BF4DFF8208108F5D07306
:10020000E6580193304604F0DAFE844631466246F1
:100210005046CDF800C004F0DBFEDDF800C0019BC5
:10022000002856D1EAB2624553D11D194444D4F88E
:10023000AC0101F001FB0146384601F003FD002846
:1002400045D0D4F8B00101F0F7FA0146384601F084
:10025000EFFC00283BD0B4F8A4319A0658BF4F46B3
:10026000142202FB0B881C0648BF2748D8F8A82197
:1002700042BF90F8B0074FF4CC7404FB0022D805BD
:1002800042BF22480C24007803F03F0348BF04FB20
:100290000022042B39460BD004D8013B012B0CD88B
:1002A00017700AE0102B05D0202B05D0082B04D1A5
:1002B000118002E0176000E0176031461448F6F73D
:1002C0009AFF2846002103B0BDE8F04F31E61148FF
:1002D00005E00BF1010BBBF1A30F8AD10E4803B06F
:1002E000BDE8F04F94E6504603B0BDE8F04F17E785
:1002F00003B0BDE8F08F00BF61A401086486010867
:10030000EA9C010873A4010854100020202E00204C
:1003100076A4010881A40108BF9B0108C4840108D8
:1003200070B50546284604F04AFE064658B9194BF2
:1003300019485A79194BBDE8704003EB8203D3F892
:10034000581EF6F758BF28461549324604F040FEBD
:1003500060B91448FFF75CFE134C54F8041F19B140
:100360001248F6F748FFF8E7114805E00024114B62
:1003700053F8241019B91048BDE8704048E62846E3
:10038000324604F025FE01340028F0D1014B0B4D1C
:100390005C71C7E754100020A1A40108C4840108BF
:1003A000989C0108ADA401081C930108949C0108C5
:1003B00073A4010820930108BF9B0108FB98010862
:1003C00008B50748FFF724FE064BD869F8F7B5F9DA
:1003D000FEF7D8FEF7F7AAF8034A044BDA6008BD27
:1003E000C0A40108202E00200400FA0500ED00E062
:1003F00008B50548FFF70CFE00F036F8F7F7C0F82F
:10040000BDE80840DCE700BFCCA4010808B50448FB
:10041000FFF7FEFDF7F7B4F8BDE80840D0E700BFEE
:10042000E2A401080E4B1A78692A16D140F2DC7258
:100430005988914211D11A79BE2A0ED193F8D92741
:100440000020EF2A0BD113F8012B5040054A9342AC
:10045000F9D1B0FA80F0400970470020704770472A
:1004600000F80108DCFF01082DE9F74FEA4C0021F4
:1004700040F2DC72204604F05EFDE84B04F53A726F
:100480001A60E74B00221A70E64B04F2B271196051
:1004900069232370032363714FF48073A3604FF4C7
:1004A0001673A4F86631FA23A4F86831BC23A4F8C3
:1004B00064314FF4FA73A4F86E31012384F8623189
:1004C00084F87E3184F88631052384F8273240F29F
:1004D000DC53A4F8983140F24C43A4F89A3140F22E
:1004E0006C73A4F89C3140F27533A4F89E3140F649
:1004F0004303A4F8A0312346202184F86A116E2119
:1005000084F87C110A2184F87D112B2184F87F1155
:10051000212184F88011232184F881114FF4C871BE
:10052000A4F88211032ACCBF0121002102F10102AB
:1005300083F8A21114BF1E217521122A83F8A3117A
:1005400003F10203EED140F27E41A4F8441140F2DF
:100550003A71A4F8461140F27E51A4F84C1140F2D1
:10056000EA5140F2DC50A4F84E1140F2B4514FF47D
:10057000FA63A4F8C831A4F8CC31A4F8D031A4F8B7
:10058000D431052384F8E231C82301264FF47A7769
:100590004FF0320BA4F8E631DFF880924FF4C873C5
:1005A0004FF01E0A1922A4F8EA31A4F84A01A4F86F
:1005B0005011A4F8C671A4F8CA71A4F8CE71A4F8B9
:1005C000D27184F8E46184F8E56184F8E861A4F804
:1005D0004871A4F852B184F895A184F8E3210092FF
:1005E0000190A4F8543184F8E16184F8EE61A4F834
:1005F00056B184F8F161FDF7D7FBD9F80030009AC5
:1006000000254FF00F0E2674E673A573A58183F8BD
:1006100005E0DA714FF0220E2122172183F806E05F
:100620005A744FF00E0E53225975997583F810E0E5
:10063000DA7655210A224FF0350E4FF02808D9708E
:1006400083F81AE02D214FF05A0E9A7400924FF061
:10065000780C642283F80BA083F80CA0597383F8FC
:1006600008E01A771D7083F8018083F80280DD7539
:1006700083F804B09D731D76DD735D7683F8098081
:1006800083F80AC019754FF4FA71A3F84E103C2193
:1006900083F85110112183F850106349DFF8A8C185
:1006A0009963D9636149C3F82CC099626049C3F862
:1006B00030C0DFF898C159634FF07F5A5D49019807
:1006C000C3F820A0C3F824A0C3F848C04FF0000A24
:1006D0004FF04B0C59649E7783F85250C3F840A0FA
:1006E00083F84CC084F8B2E7A4F8BC074FF0410E81
:1006F000042084F8B3E784F8B4B784F8B55784F8D5
:10070000B95784F8BA5784F8B65784F8B75784F8BD
:10071000B85783F85C00A3F85850A3F85A50A3F8D0
:1007200056501966152183F8681043494348D96625
:10073000434983F864801967424983F865805967A3
:1007400083F87860FDF75AFBD9F80030009A184614
:100750004FF4487183F8115183F8125183F81381D3
:1007600083F8146183F81851A3F8161184F8D8217E
:10077000C82284F8D9216422A4F8DA7184F8DC5103
:10078000A4F8DE210E2202FB05326FF0170482F876
:100790001941032482F81A416FF02F0482F81B419B
:1007A000072482F81C416FF0230482F81D410524C0
:1007B00082F81E4101355A2480F8204180F82141F9
:1007C0006422FF24082D80F81F2180F822414FF079
:1007D000000100F10E00D5D1C820A3F88A01142031
:1007E00083F88C01A3F890211E204FF4967283F8B1
:1007F0008D01A3F892210120282283F8891183F822
:100800008E01A3F894210B46034D5A191033C02BC7
:10081000C2F814A01CE000BF54100020A40F002058
:10082000202E0020CC0F00208FC2F53C000060403D
:100830006666663F0000A0409A99193FC8AF01085C
:10084000F6287C3F3D0A773FCDCCCC3E00004040AF
:10085000DAD105F52A700021402204F06CFB002358
:10086000264EEA18995904330868382B244CC2F8EC
:10087000A802F5D104F50A700021802204F05BFB88
:1008800006F13801702204F50A7004F049FBFEF706
:10089000FBFDD9F8006000230125314604F5906086
:1008A0004FF4CC7284F8D83784F8D65784F8D757E9
:1008B00004F036FB04F5C36031464FF4CC7204F00B
:1008C0002FFB104B1B681A68C4F8BE275A68C4F87F
:1008D000C2279A68C4F8C6271A68C4F8CA275A6893
:1008E000C4F8CE279A680223C4F8D22784F8D454D7
:1008F00084F86C3603B0BDE8F08F00BFE4930108C4
:1009000054100020CC0F002038B5094B93F8D8576D
:1009100065B9084C2068F7F73FFC074B25601B784A
:10092000022B03D1BDE83840FDF7FDB938BD00BF4B
:10093000541000202C1D0020281D0020044B93F88B
:10094000D8371BB9034B1868F7F7F4BE002070477F
:10095000541000202C1D002038B5054604462046C2
:1009600014F8011B21B1034B1868FEF78DFAF6E766
:10097000401B38BD2C1D00200FB407B504AB53F845
:10098000042B054900200193F6F74AFB03B05DF8FC
:1009900004EB04B0704700BF050B0108024B014691
:1009A0001868FEF771BA00BF2C1D0020F8B5011FB2
:1009B00006460023083051F8042F02F120043F2C92
:1009C0003AD802F108040F2C06D80232032A04D9BF
:1009D000002B08BF012300E002238142EBD1012B51
:1009E00030680ED0022B1AD0736800F0030003F0B9
:1009F00003039B0043EA0010B36803F003031843AA
:100A000017E000F00F0040F04000FFF7C7FFB068AC
:100A1000736800F00F0040EA0310C0B209E000F074
:100A20003F0040F08000FFF7B9FF3079FFF7B6FFD5
:100A3000307ABDE8F840B1E706F10C0734463A4693
:100A4000002552F8043DAD0003F18001FF2910D9C3
:100A500003F50041B1F5803F02D245F0010508E001
:100A600003F50003B3F1807F34BF45F0020545F084
:100A70000305B242E5D165F03F00C0B2FFF78EFF3B
:100A800005F00303022B207807D0032B0CD0012B99
:100A900013D1FFF783FF60780FE0FFF77FFF6078E7
:100AA000FFF77CFFA07808E0FFF778FF6078FFF79A
:100AB00075FFA078FFF772FFE0780434FFF76EFF50
:100AC000BC424FEAA505DBD1F8BD10B50446C0B263
:100AD000FFF764FFC4F30720BDE810405EE710B5E0
:100AE00004467F2C06D964F07F00C0B2FFF756FFA2
:100AF000E409F6E7E0B2BDE810404FE7430083EABF
:100B0000E070ECE7084649E70C4B0D49DA6843789A
:100B1000D243C2F30222C2F10402934002781B01C5
:100B2000DBB20A4482F8003303780122580903F04B
:100B30001F0302FA03F341F82030704700ED00E094
:100B400000E100E02DE9F74FAE4C2378013B012B8B
:100B500000F253816678864240F04F81A378022BE1
:100B600000F04B81A84B9B5D7600E37023791BB1AD
:100B7000A319B3F9060007E0E36803F10043E3605B
:100B8000A319B3F90600404200F056FE9F4900F059
:100B90005BFF2369074618039A4D2BD5E86801F0DF
:100BA00065F88DF80200686901F060F897498DF8E2
:100BB0000300384600F094FE04F006FC01F07CF8D7
:100BC0009249ADF80000A86900F08AFE04F0FCFB31
:100BD00001F072F88D49ADF80400E86900F080FE7C
:100BE00004F0F2FB01F068F86946ADF806000C204D
:100BF000F7F73EFFD4F81C8000214046814D01F0FC
:100C000003F8002860D0D5F818803846414601F036
:100C100023F818B1EB68AF616B61DAE04046002160
:100C200001F01AF8002800F0D48095F820303BB18C
:100C3000022B00F2CE806B6BEF61FA33AB63C8E03E
:100C4000E968384600F042FD4FF07E514FF0010553
:100C500000F0F8FF00B90546EDB28DB16C49A06A0D
:100C600000F03EFEDFF8BC81664F4146814600F051
:100C7000D5FF10B9C7F8289007E0C7F8288004E02E
:100C8000A06A644900F02CFEA06223695D4A190342
:100C900011D5116BD3788DF800500B445A780B2086
:100CA0008DF80120DA7A69468DF802205B7D8DF897
:100CB0000330F7F7DDFE0123226B84F82030E37860
:100CC00013440022DA7282E03846414600F0A6FF63
:100CD00000B1EF61D4F81890D4F81CB048465946DA
:100CE00000F0F4FC636BA56B82465D1B6FEA0508A0
:100CF0004FEAD878B8F1000F0BD14FF07E5100F0D9
:100D0000ABFF002865D03846594600F0A5FF002803
:100D10005FD0484661694FF0010500F09DFF00B9C2
:100D20000546EDB23DB1606A394900F0D9FD394957
:100D30006062E06A07E050464FF0804100F08CFFAF
:100D400028B1E06A324900F0CBFDE06204E0606A5D
:100D5000304900F0C5FD60622C49606A00F0C0FDBA
:100D600000F0AAFFD4F830A0E7785FFA80F9574482
:100D700087F80190E06A00F09FFF2369C0B21B036F
:100D800078750ED545EA48058DF800508DF801902C
:100D9000FB7A69468DF803000B208DF80230F7F7D7
:100DA00067FE94F82020174B022A0DD1002283F809
:100DB00020201D6BDA78986A1749154400F090FDE1
:100DC00000F07AFFE87202E0022283F82020F8F7B0
:100DD0000BFF22790B4B0AB1104A00E0104A26445F
:100DE000DA60B6F9060000F027FD084900F02CFE95
:100DF0000146E06800F06AFC00E0084603B0BDE888
:100E0000F08F00BF642E0020BC9401080000204138
:100E1000EC51783F0AD7833F00007A440000A0419C
:100E20000000A0C16F12833A2B4BF0B52B4D1E680A
:100E300005F110002F782C46F3195978013501F08F
:100E4000040101F0FF0219B18542F3D10020F0BD89
:100E5000224D631B022B0ADD1AB102EB8202520003
:100E6000D2B215F8013B303B1A44D2B2F1E700216F
:100E7000AC420AD919B101EB81014900C9B215F898
:100E8000013B303B1944C9B2F2E72E2F16D1013491
:100E900004200023257803EB830377197F785B0018
:100EA0007F079BB244BF303D5B1900F1FF3044BF68
:100EB00001349BB210F0FF00ECD100E000230848A1
:100EC0004143642000FB03130620B3FBF0F3054805
:100ED00000FB0230F0BD00BF58000020A02E002013
:100EE00040420F008096980000231A4630B5104902
:100EF0008C1894F83C40BCB12E2C06D1013298B12C
:100F00008C180444002584F83C500A24114463439F
:100F100091F83C10A1F13004092C9CBF303B5B18C8
:100F20000E2A03D80132E2E7184630BD002030BD5A
:100F3000642E00200EB40FB5074906AB0190074A96
:100F400001A80393F6F76CF8019B00221A7004B015
:100F50005DF804EB03B07047356D00087E9D010815
:100F60000028114AB8BF404290FBF2F330B50F4C55
:100F70003C2504FB030068430D4D90FBF2F22D6805
:100F80002D7B25B903EB830303EB830301E0C3EB64
:100F9000031302EB830304FB02020B804FF47A730A
:100FA00092FBF3F24A8030BD80969800806967FF1B
:100FB00038180020022803D0431E58425841704779
:100FC000064B1B681B7823B1054B1868C0F3C04063
:100FD0007047044B1878C0F380007047DC05002090
:100FE000680F00209230002010B50A4C5E280146A0
:100FF000206805D15D21FDF747FF20683E2105E00F
:101000005D2903D1FDF740FF20683D21BDE8104078
:10101000FDF73ABFB02E002010B50446C0B2FFF76E
:10102000E3FFC4F30720BDE81040DDE7024B5E217B
:101030001868FDF729BF00BFB02E002038B505465F
:10104000054C5E212068FDF71FFF20682946BDE89A
:101050003840FDF719BF00BFB02E002013B504467D
:1010600001A90068FFF77CFF1320FFF7E7FFBDF938
:101070000400FFF7D1FF1B20FFF7E0FFBDF90600DA
:10108000FFF7CAFF2320FFF7D9FF2368002BB4BF67
:1010900053204E20FFF7C0FF01A96068FFF760FFF3
:1010A0001220FFF7CBFFBDF90400FFF7B5FF1A20B0
:1010B000FFF7C4FFBDF90600FFF7AEFF2220FFF7E0
:1010C000BDFF6368002BB4BF57204520FFF7A4FF86
:1010D00002B010BD674B73B51878FFF76BFF664D14
:1010E00004462B78834220D0C8B1644B1B68E3B11F
:1010F00093F9000002230093614B04211B68002236
:101100005B78003318BF012301934FF41653F7F7B0
:10111000C8FA5C4B186040B101232B7005E0594EB2
:101120003068F7F739F834602C70574B574D187802
:10113000FFF740FF2B780446834218D088B1544B08
:101140001B68A3B10022012493F9000008214FF489
:10115000964300940192F7F7A4FA4E4B186028B911
:1011600005E04C4E3068F7F717F834602C704A4BA6
:101170004A4D1878FFF71EFF2B78044683422E460F
:1011800043D0002838D0464B1A68002A3DD0D37986
:1011900092F90000002B4FF00202424C08BF0223DC
:1011A0000092002254F8233001921021F7F779FAC7
:1011B0003D4B0546186040B33C4C94F84A30022B36
:1011C0000BD094F89620022A01D14C3405E023B1CB
:1011D000002A04F14C0418BF0024354B1C6044B1B4
:1011E000204600214C2203F0A6FE0223256084F84D
:1011F0004A300123337008E02B4E3068FEF718FEAA
:101200003068F6F7C9FF34602C702A4B2A4D1878E5
:10121000FFF7D0FE2B780446834229D000B3274B3A
:101220001B682BB3264A93F90000126803235278F7
:101230002021002A0CBF08220922009301924FF4BA
:1012400061430022F7F72DFA1E4B186080B11E4A49
:10125000012313702B701D4B1A681D4B1A6007E099
:10126000184E3068F6F798FF174B34601C702C70DE
:1012700002B070BDE40500202C100020E005002025
:1012800038180020B02E0020E50500205818002056
:10129000DC180020CC180020F0050020E218002007
:1012A000EC0500208C840108E4180020902900201F
:1012B000E8180020FC050020F8180020F8050020A0
:1012C000F4050020FC18002000190020982E0020B2
:1012D0000419002003788B420AD9064B1A78064B72
:1012E00053F8210002B1400800F5777080B27047D2
:1012F00000207047302A0020B42E002007299DBF0F
:10130000024B03EB8101088E00207047B42E0020B1
:10131000034B03EB4101B1F85000C008704700BF18
:10132000B42E002008B5084B03EB8101086F00F0D4
:101330007FFA064900F0D4FA054900F0C9F900F037
:10134000BBFC80B208BD00BFB42E00200000203FCF
:1013500000005C44024B03EB4101B1F8B800704758
:10136000B42E0020024B03EB4101B1F8DC007047C2
:10137000B42E0020024B03EB4101B1F8DC007047B2
:10138000B42E00200020704710B50446F7F71CF972
:1013900041F288310E4BE4B2D3F8F420C3F8F400E4
:1013A000821A8A42C3F8F82084BF002283F8FC2006
:1013B00093F8FC2006490F2A134418BF013283F822
:1013C000FD4012BF81F8FC20012381F80D3110BDD2
:1013D000B42E002010B50446F7F7F6F841F2883134
:1013E0000E4BD3F81021C3F81001821A8A42C3F8B9
:1013F000142184BF002283F8182193F8182107498B
:10140000142A134418BF013283F8194112BF81F81E
:101410001821012381F82E3110BD00BFB42E002009
:1014200038B50446F7F7D0F8274A2749D2F83031C3
:10143000C2F83001C31AB3F57A6F84BF002382F873
:10144000343192F8343133B9A82C3BD181F835319D
:10145000A1F8363106E0022B02D181F8384101E0D3
:10146000242B02D8D11881F8394192F83811013370
:101470000231DBB249008B42134D82F8343118DA65
:10148000B5F83631E0B283EA0020082310F4004FAB
:101490004FEA400018BF80F4815003F1FF3318BFBA
:1014A00080F0010013F0FF0380B2EFD1A2F8360103
:1014B00038BD01318B4201BF002385F8343101234F
:1014C00085F8353138BD00BFB42E002010B5044674
:1014D000F7F77AF840F6AC510F4AD2F86031C31AE8
:1014E0008B42C4BF002382F8643192F86431D11872
:1014F00081F8654123B90F2C0DD10749C1F860016E
:101500000133DBB2192B044982F864310CBF01238B
:10151000002381F87E3110BDB42E00200022134636
:1015200070B5214C1118615C83EA0123082113F482
:10153000004F4FEA430318BF83F4815301F1FF3199
:1015400018BF83F0010311F0FF019BB2EFD101320C
:10155000192AE6D100F11902A55C00F11A02A25C79
:1015600002EB052292B29A421DD1104E96F87F519D
:10157000CAB2AA4214D2431C03EB4203DBB2E25CC0
:101580000133E35C03EB02239BB24FF4AF6253439E
:10159000074A1B1303F5487322F811300131E7E7BE
:1015A000012386F8803170BD6A290020B42E002006
:1015B0004829002030B5114A4300D2F88411CC18D4
:1015C000257E15B1022D10D00BE0022805D9032885
:1015D00007D10B4B1B68DB0401D5C88930BD888A55
:1015E00030BD1344B3F8B80030BD607E00EB80001E
:1015F00000EB800000F2EE2080B230BDB42E00205F
:10160000742E002008B5F6F7DFFF074B022283F89F
:101610008C21064AC3F888011268C3F89821012278
:1016200083F8B12108BD00BFB42E0020982E002001
:1016300008B5F6F7C9FF084B022283F88C21D3F8CE
:10164000982100F5B71000F5587002F2DC52C3F88B
:101650008801C3F8982108BDB42E002042F201028F
:10166000034B1B681A420CBF01200020704700BFCB
:10167000742E002008B5F6F7A7FF044B00F5F42000
:1016800000F59070C3F8B40108BD00BFB42E00206F
:1016900008B5044B1B7803F00503052B01D1FDF7BA
:1016A00071FDFEE76C300020D0400B1C1141203A48
:1016B00003D49C4613411843634652429340184357
:1016C000704700BF80F0004002E000BF81F00041A1
:1016D00042001FBF5FEA410392EA030F7FEA226CD8
:1016E0007FEA236C6AD04FEA1262D2EB1363C1BF68
:1016F000D218414048404140B8BF5B42192B88BFD7
:10170000704710F0004F40F4000020F07F4018BFF9
:10171000404211F0004F41F4000121F07F4118BF19
:10172000494292EA030F3FD0A2F1010241FA03FCC1
:1017300010EB0C00C3F1200301FA03F100F00043A9
:1017400002D5494260EB4000B0F5000F13D3B0F171
:10175000807F06D340084FEA310102F10102FE2AE0
:1017600051D2B1F1004F40EBC25008BF20F0010050
:1017700040EA03007047490040EB000010F4000FFE
:10178000A2F10102EDD1B0FA80FCACF1080CB2EB91
:101790000C0200FA0CF0AABF00EBC25052421843F0
:1017A000BCBFD0401843704792F0000F81F4000195
:1017B00006BF80F400000132013BB5E74FEA410368
:1017C0007FEA226C18BF7FEA236C21D092EA030FD4
:1017D00004D092F0000F08BF0846704790EA010F4E
:1017E0001CBF0020704712F07F4F04D1400028BF7B
:1017F00040F00040704712F100723CBF00F500005D
:10180000704700F0004343F0FE4040F40000704792
:101810007FEA226216BF08467FEA2363014642023E
:1018200006BF5FEA412390EA010F40F48000704751
:101830004FF0000304E000BF10F0004348BF4042F7
:101840005FEA000C08BF704743F0964301464FF033
:1018500000001CE050EA010208BF70474FF000038F
:101860000AE000BF50EA010208BF704711F00043D0
:1018700002D5404261EB41015FEA010C02BF8446A0
:101880000146002043F0B64308BFA3F18053A3F5FF
:101890000003BCFA8CF2083AA3EBC25310DB01FA46
:1018A00002FC634400FA02FCC2F12002BCF1004FCA
:1018B00020FA02F243EB020008BF20F0010070475B
:1018C00002F1200201FA02FCC2F1200250EA4C00AF
:1018D00021FA02F243EB020008BF20EADC707047F5
:1018E0004FF0FF0C1CEAD0521EBF1CEAD15392EA03
:1018F0000C0F93EA0C0F6FD01A4480EA010C4002DF
:1019000018BF5FEA41211ED04FF0006343EA501038
:1019100043EA5111A0FB01310CF00040B1F5000F7A
:101920003EBF490041EAD3715B0040EA010062F129
:101930007F02FD2A1DD8B3F1004F40EBC25008BF13
:1019400020F00100704790F0000F0CF0004C08BF31
:1019500049024CEA502040EA51207F3AC2BFD2F1FE
:10196000FF0340EAC250704740F400004FF000030C
:10197000013A5DDC12F1190FDCBF00F00040704746
:10198000C2F10002410021FA02F1C2F1200200FA84
:1019900002FC5FEA310040F1000053EA4C0308BF4B
:1019A00020EADC70704792F0000F00F0004C02BF9C
:1019B000400010F4000F013AF9D040EA0C0093F017
:1019C000000F01F0004C02BF490011F4000F013B71
:1019D000F9D041EA0C018FE70CEAD15392EA0C0FDF
:1019E00018BF93EA0C0F0AD030F0004C18BF31F04A
:1019F000004CD8D180EA010000F00040704790F020
:101A0000000F17BF90F0004F084691F0000F91F0C3
:101A1000004F14D092EA0C0F01D142020FD193EA89
:101A20000C0F03D14B0218BF084608D180EA010011
:101A300000F0004040F0FE4040F40000704740F0ED
:101A4000FE4040F4400070474FF0FF0C1CEAD052BB
:101A50001EBF1CEAD15392EA0C0F93EA0C0F69D017
:101A6000A2EB030280EA010C49024FEA402037D082
:101A70004FF0805343EA111143EA10130CF0004079
:101A80008B4238BF5B0042F17D024FF4000C8B4269
:101A900024BF5B1A40EA0C00B3EB510F24BFA3EB49
:101AA000510340EA5C00B3EB910F24BFA3EB910319
:101AB00040EA9C00B3EBD10F24BFA3EBD10340EA73
:101AC000DC001B0118BF5FEA1C1CE0D1FD2A3FF6B9
:101AD00050AF8B4240EBC25008BF20F0010070476E
:101AE0000CF0004C4CEA50207F32C2BFD2F1FF0311
:101AF00040EAC250704740F400004FF00003013A42
:101B000037E792F0000F00F0004C02BF400010F4E5
:101B1000000F013AF9D040EA0C0093F0000F01F0F9
:101B2000004C02BF490011F4000F013BF9D041EA1B
:101B30000C0195E70CEAD15392EA0C0F08D142024E
:101B40007FF47DAF93EA0C0F7FF470AF084676E721
:101B500093EA0C0F04D14B023FF44CAF08466EE7FA
:101B600030F0004C18BF31F0004CCAD130F00042C8
:101B70007FF45CAF31F000437FF43CAF5FE700BF20
:101B80004FF0FF3C06E000BF4FF0010C02E000BF49
:101B90004FF0010C4DF804CD4FEA40024FEA4103EB
:101BA0007FEA226C18BF7FEA236C11D001B052EAA1
:101BB000530C18BF90EA010F58BFB2EB030088BF67
:101BC000C81738BF6FEAE17018BF40F001007047D6
:101BD0007FEA226C02D15FEA402C05D17FEA236CB8
:101BE000E4D15FEA412CE1D05DF8040B704700BFFF
:101BF000844608466146FFE70FB5FFF7C9FF002896
